:1000000000400020DD8000001D8100001F810000F5
:1000100000000000000000000000000000000000E0
:10002000000000000000000000000000218100002E
:100030000000000000000000238100002581000076
:1000400027810000495B00008984000027810000AF
:1000500027810000000000002781000027810000A8
:10006000B53900005D88000027810000278100006D
:1000700027810000278100002781000027810000E0
:10008000278100000D8500002781000027810000E6
:1000900027810000278100002781000027810000C0
:1000A0002781000027810000000000000000000000
:1000B0000000000000000000000000000000000040
:1000C00010B5064C2378002B07D1054B002B02D02E
:1000D000044800E000BF0123237010BD700200201F
:1000E000000000003CF60000044B10B5002B03D0CC
:1000F0000349044800E000BF10BDC04600000000F6
:10010000740200203CF60000164B002B00D1144B6B
:100110009D46402292029A1A924600218B460F4633
:100120001348144A121A0CF0CDF90F4B002B00D0D3
:1001300098470E4B002B00D0984700200021040068
:100140000D000D48002802D00C4800E000BF0CF064
:1001500079F92000290008F0E9F90CF04DF9C046C2
:100160000000080000400020000000000000000027
:1001700070020020CC2F00200000000000000000D2
:1001800002000120104011D1042A0ED91368180969
:1001900080B2002809D001388000031D11180979A8
:1001A000002902D001309842F8D170470020FCE7C6
:1001B0000378002B03D05AB2002A01DB01307047CC
:1001C0003F229343C03B59424B41C01803789343AD
:1001D000802BF4D10130F9E710B500240378002B0F
:1001E00001D1200010BDFFF7E3FF0134F6E770B541
:1001F000002204000D00411C092003F003FF002829
:1002000006D001236200134343600023A34200DBB6
:1002100070BD9A00A958821891600133F6E770B555
:10022000012803DC1C2001F06FFA70BD01230D686A
:1002300011201D42F7D04868184206D1042804D97D
:100240000F2302681340042B01D00E20EBE703F0CC
:1002500037FD6D100400002D03DDFFF7BDFFA84240
:1002600006DA1220DFE72000FFF7A2FF0400013DBD
:10027000012DF8D120787F2809DDDF280BDCF82359
:100280003F22DB00800118406378134018430123AC
:1002900040001843C9E7EF280BDCFC226378120109
:1002A0009B0113403F220007000C0343A07810403D
:1002B000ECE7F72812DCFC22637892021B03134060
:1002C000E0228004520310403F221843E378134099
:1002D000FC220343A07812018001E8E7012040429C
:1002E000D5E7F8B54D680F00EB0706D4042D04D907
:1002F0000F232E683340092B03D00B2001F004FAA2
:10030000F8BD6B683609B6B25C10731EA3420FD8F5
:100310000321200009F092FF6421642803DC01001E
:10032000032800DA03212800891903F09DFE050047
:100330002B6800201B099BB2013B9C42E0D23A682B
:10034000A31C9B005A510123013464001C436C60C0
:10035000D6E7F0B585B0012803DC1C2001F0D4F904
:1003600012E001274B683A000093022806D08B6800
:100370003B4203D05F10002F00DC17000125009BDB
:100380002B4203D00120404205B0F0BD009B042B5E
:10039000F8D91B680C680F261900314004292DD1AB
:1003A0002C4205D1042C03D923681E40042E01D011
:1003B0000E20D3E70098FFF7E3FEB842E2DB009897
:1003C00003F07EFC0600200003F07AFC03780100B5
:1003D000002BD7D0781E30180CF02AFC041ED1D088
:1003E0003378002B01D0A64202D36800012521E01A
:1003F0003000FFF7DDFE01350600F1E709293ED1A7
:10040000009B5B685B1001939F42BBDC2C422ED1AA
:10041000042C2CD923683340042B28D1200003F06E
:100420004FFC039602907E1C009AB300D058844281
:1004300002D178002843A7E728420ED104280CD91E
:100440000368039A1340042B07D103F039FC010021
:1004500002980CF0B7FB0028EBD0019B37009E42BE
:10046000E1DD8FE71F00019B9F4200DD8AE77B1CD7
:1004700000999A008A58A242F4D17800B6E703297D
:1004800000D07FE71A0992B25B0F92000B40D31A9B
:1004900001939F4200DD75E72C4229D1042C27D916
:1004A00022681640032E19D1100980B2520F800025
:1004B0003240251D801A019B2E181B1A0193009BA8
:1004C000781E0433019A904200DD5BE72A00191878
:1004D000B2420FD316D10130400087E7042E07D176
:1004E000200003F0EDFB05002000FFF749FEE2E7E6
:1004F0000F2033E70C78A4461478A44502D10131CB
:100500000132E5E70130DDE7F0B50D0085B00128E7
:1005100004DC1C2001F0F8F805B0F0BD01270868E4
:10052000384206D1042804D90F2102680A40042A5F
:1005300001D00E20EEE76A681740FAD1042AF8D9F4
:1005400013680B40042BF4D103F0BAFB0400686875
:1005500003F0B6FB02900CF03FFB039000280FD194
:100560002000FFF739FE0190019B0122591C092050
:1005700003F048FD364E3060002815D10020CBE74F
:10058000029920000CF054FB001B43424341200021
:100590000193019B5E1C0028E6D0039B0299C018C2
:1005A0000CF046FB0196F4E70122019B5B0013432C
:1005B0004360039B002B18D12000FFF7F9FD019B3E
:1005C0000500BB4201DC3068A6E7291B200003F0D0
:1005D00097FD0028D2D0BB1C32689B0098502800A1
:1005E000FFF7E6FD01372C00E9E7019B012B02D163
:1005F0002B68836090E7029920000CF019FB01251D
:100600000700019B002F13D0AB42DCDB391B20001D
:1006100003F076FD0028B1D032680135AB00985068
:10062000039B0299FC1820000CF002FB0700E8E78E
:10063000AB42C8DB20000CF0CFFA0100200003F031
:100640005FFD00289AD001353368AD00E850BAE765
:10065000E40F002010B503F017FB430001201843FE
:1006600010BD0000C30711D404280FD90F2302685E
:100670001340032B0AD119400133591AC0234907EB
:10068000DB051940024B1A40114301607047C04618
:10069000FFFFFF9F70B5002805DC1C2001F034F837
:1006A0000500280070BD01220C68144201D10D2004
:1006B000F4E701281CD04B681342F8D05B101320DC
:1006C000FF2BEBD81A0619040A431A431B021343E3
:1006D0006410E243D2171440E11C89101A00032071
:1006E00003F090FC051EDCD02100FFF7BBFFD8E72C
:1006F0000023EDE7F7B507000E001C20012F06DDF3
:100700004C68012322001A40009203D10D2000F012
:10071000FBFF53E0022F02D08A681A42F6D0012371
:1007200035681D4200D0A9E0042D00D8A6E01C4188
:10073000002C00DC1C000F2029680840092828D163
:100740006B685B100093022F05D0B368009A5B10B2
:100750009A4200DD0093009B01221D1B0135EB43F3
:10076000DB171D40691C092003F04CFC071E09D053
:1007700001236D001D430300326808334560009972
:10078000A14201DA3800FEBD0134A100515802C374
:10079000F5E7042845D1280003F092FAFFF71CFD85
:1007A0000190022F04D0B3685B10984200DD0193E2
:1007B000019BA34204DA002003F096FC0700E1E766
:1007C000280003F07DFA0700009BA34221DB2800EC
:1007D000009703F075FA05003800FFF7E9FC019B6C
:1007E00001340700A342F7DA009BC41A200003F08B
:1007F0007BFC071EC6D003F063FA0190306803F05B
:100800005FFA2200009B591B411801980BF03EFE35
:10081000B8E73800FFF7CCFC009B070001330093DA
:10082000D2E703282AD10B099BB2490F9B00014054
:10083000591A022F04D0B2685210914200DD110003
:10084000A14205DA00220320110003F0DBFBB5E72B
:1008500003200E1B331DD9170140C918891000222F
:1008600003F0D0FB071E00D18CE7013631000334C2
:10087000FFF7F8FE381D29193200C7E7212046E7A7
:10088000F7B5002804DC1C2000F03EFF040014E053
:100890000D6801272E003E4011D03D41FF2D01D9AA
:1008A0001320F1E700223900032003F0ABFB041E04
:1008B00003D03900FFF7D6FE25712000FEBD042DC0
:1008C000EED90F232A681340042B1BD12800FFF711
:1008D00057FCC31C07000320D9170140C918891011
:1008E000320003F08FFB041EE7D03900FFF7BAFE99
:1008F000280003F0E5F9231D01003A0018000BF071
:10090000C5FDDAE7092B1FD103206B6832005B10AD
:1009100001930333D9170140C918891003F072FB02
:10092000041ECAD00199FFF79DFE019B9E42C4DAC6
:10093000B300EB189B683B4204D05B10FF2BAFD891
:10094000A21913710136F0E7032BA9D12C00B4E7EB
:1009500010B57F2902DC0170013010BD1A4B99429D
:100960000CDC40238A115B42134303703F230B408E
:1009700080214942194341700230EEE7134B9942FE
:1009800010DC20230A135B4213433F2480220370B0
:100990008B1152422340214013430A43437082701B
:1009A0000330DAE70A4B9942D7DCF0230370603B4F
:1009B0004370113B8A11FF3B1A4382703F22114062
:1009C0001943C1700430C8E7FF070000FFFF0000B3
:1009D000FF0F0100F0B50D0085B0002803DC1C20DE
:1009E00000F092FE0DE009680122080010400AD0D4
:1009F00002AC11412000FFF7ABFF011B200003F008
:100A00007FFB04001AE004293FD90F230C68234020
:100A1000092B3AD14B685B10019303239C46019B41
:100A20009A420EDD03F060FB041E07D02E680125FC
:100A300003F046F92F00019B9D421DDD200005B00B
:100A4000F0BD01329300CC580123234001D127206F
:100A5000C6E764107F2C0DDD0D4E0223B44209DD84
:100A60000C4E6346B44205DD00270B4EE30FA64251
:100A70007B419B00C018D2E70135AB00F1583942E9
:100A8000E5D04910FFF764FFD5E70B20A8E7C04683
:100A9000FF070000FFFF0000FF0F010010B5012459
:100AA000044002D04410200010BD042810D90F23A8
:100AB00002681340042B07D103F002F921000A2237
:100AC0000CF052F90400EEE7032B01D10430F5E7F6
:100AD0000D2000F019FEE6E710B5040001200840E3
:100AE00010D104290DD90F230A681340042B08D113
:100AF000080003F0E5F8010020000CF063F8434221
:100B0000584110BD0020FCE7F7B50E00012803DCBA
:100B10001C2000F0F9FDFEBD4D68EB0706D4042D46
:100B200004D90F222B681A40092A01D00B20F0E7C4
:100B30006A681B099BB25410A34200D85C1E0127AF
:100B400031680F404810002F35D12648FFF7C4FF09
:100B500001230190002813D131682348FFF7BCFF1F
:100B6000002811D0002C0DD00122631C013C9440C0
:100B70009B005A5114436C6004E00137BA00AB503B
:100B8000BC42FADA0020C6E701233068184223D1BC
:100B9000042821D902680E331340042B1CD1FFF71F
:100BA0007DFF002807D131681048FFF795FF002826
:100BB00012D01220ADE70028FBDD8442F9DB830070
:100BC000EB180433844209DC0123621C013C9C4085
:100BD000920053511C43CEE711209AE75A68013026
:100BE0001A60EEE767DB00006BDB000070DB0000E3
:100BF000002310B50C000B70C30705D50D4942103A
:100C000020000BF0A3FF08E00B49002802D00428C5
:100C100004D10A4920000BF0B9FF10BD0428FCD90B
:100C20000F2302681340042BF7D103F049F804495D
:100C30000200E5E70CE7000072DB000078DB000053
:100C40007DDB0000F0B593B0060002911C20012E60
:100C50001DDD029B01251B681C002C4000D0ADE06F
:100C6000042B00D8E6E01A680F231A40092A4AD15B
:100C70000394039A029992008A5817002F4005D1D5
:100C8000042A03D910681840092806D0222000F051
:100C90003BFD0190019813B0F0BD52685210A418AA
:100CA000039A013203929642E3D1611C012203F0C0
:100CB000A9F90190002802D100230193EAE7019BE2
:100CC0006400190025435D600831029ABB00D058CA
:100CD00002684368120992B25B109A4200D8531E10
:100CE0000022934209DCDA43D21713409B00C91853
:100CF000039B01379F42E8DBCCE794000519AD6800
:100D000001320D51EDE72700032A59D10193029AD0
:100D1000BB00D3582B42B9D1042BB7D9186801991D
:100D20000140032939D1020992B2430F92000B40CE
:100D3000D31A1C190137BE42E9D10320E31CD9178D
:100D40000140C9188910002203F05CF901900028C5
:100D5000B2D000252100FFF785FC019B1E1D029AE1
:100D6000AB00D45801231C421FD1042C1DD90F21E4
:100D700023681940032918D1180980B25B0F80003D
:100D80000B40C01A0023834213DBC343DB17184018
:100D900001353618BD42E2DB7CE7042900D075E757
:100DA0001800FFF7EDF92418C4E72000FFF7E8F971
:100DB000E8E7E2181279F2540133E4E700273C0037
:100DC0000F25029ABB00D3580122134234D1042BC1
:100DD00032D9186801002940042935D11800FFF7DD
:100DE000CFF924180137BE42EBD1200003F07CF983
:100DF0000190002800D15FE7029FB600BB19041DD7
:100E0000029301233D681D4229D1042D27D90F26C5
:100E10002B681E40042E37D12800FFF7B1F90600D9
:100E2000280002F04DFF0100200032000BF02EFBE5
:100E3000A41922E02700C3E7180005A9FFF7D8FE90
:100E400005A80BF0C9FECCE7032900D01EE7020974
:100E500092B2430F92000B40D31A1C19C2E705A9A6
:100E60002800FFF7C5FE05A80BF0B6FE05A9050092
:100E7000020020000BF00AFB6419029B0437BB42FE
:100E8000BFD10023237005E7032EF6D11A0992B2D1
:100E90005B0F92001E40961B291DC5E7F0B50D00A3
:100EA00097B0002806DC1C2000F02EFC070038005C
:100EB00017B0F0BD0C68012123000B40009306D150
:100EC000042C04D922680F331A40092A01D00B20C0
:100ED000EAE7626852100392002A03DC009803F0EC
:100EE00003F9E3E7504A019201280BD068680842F1
:100EF00008D1042806D902681340042B02D102F05D
:100F0000DFFE019001980BF067FE06000F27039BA0
:100F10000834013B05935E43039B02909B00E3185A
:100F2000049301232068184273D1042871D9016801
:100F30000B003B409C46042B03D1FFF721F9861997
:100F400009E0032B6CD162460B099BB2490F9B0051
:100F500011405A1A9619049B0434A342E1D130007F
:100F600003F0C2F8071EA2D02B680793029B002B48
:100F700003D0686802F0A4FE0190380002F0A0FEE1
:100F80000400009B079A9B00D3189E68300002F073
:100F900097FE0123334005000693002B01D1042E58
:100FA00004D809A93000FFF723FE09AD28000BF093
:100FB00013FE069B0490002B0ED1042E0CD90F219A
:100FC00033681940032907D11A0992B25B0F9200C6
:100FD0000B40D31A351D04932000049A29000BF00E
:100FE00055FA049BE418029B002B0AD0059B009A3B
:100FF000934206DD2000029A01990BF047FA029B0A
:10100000E418009B01330093009A039B9342B8D1EC
:101010004DE709A9FFF7ECFD09A80BF0DDFD8EE710
:1010200002F04EFEF9E7C046A2E0000010B5012232
:10103000002400280BDD0B681A40141E03D05C103E
:10104000E343DB171C400122904200D04A68611C38
:10105000092002F0D7FF002803D0012364001C43BD
:10106000446010BD0A6870B510000125284034D1D5
:10107000042A32D90F24136849681C40092C17D15F
:1010800054681B099BB22C41A34200D85C1E8442C9
:1010900005DC02200133984206DB00200FE08500CA
:1010A0005519A9600130F2E7840011510130F2E7CF
:1010B000032C12D1294203D1132000F025FB70BD6F
:1010C0004910FF29F8D81B099BB204329B00D318A2
:1010D0009342E2D911700132FAE70B2000F014FBC1
:1010E000DBE700000123F7B500254E680C00334014
:1010F0000193AB420ED11D00042E0BD90F22336891
:101100001A40092A26D172681B099BB25510AB42BE
:1011100000D85D1E27687C10FB0746D439003D4887
:10112000FFF7DAFC002826D00BF0ACFC290009F010
:101130006BF94C1C019B002B00D069E0042E67D991
:1011400032680F331340092B3BD10134A400A4595A
:101150002000FEBD042A04D13000FFF711F805007D
:10116000D8E7019D032AD5D11D09ADB25B0FAD00B3
:101170001340ED1ACEE739002748FFF7ADFC0028F1
:101180001DD1042F16D90F233A681340042B11D117
:101190003800FFF783FC041E07D139001F48FFF712
:1011A0009BFC002806D0122005E0002CFBDDA542A8
:1011B000C0DAF8E7112000F0A7FA0400C8E72C0015
:1011C000B8E7042B1CD1300002F07AFD0500012C99
:1011D0000EDCFEF7EDFF461B300002F085FF041E1B
:1011E000B6D002F06DFD320029000BF04FF9AFE7E9
:1011F0002B78013C002BD6D02800FEF7D9FFE5E77D
:10120000032B05D13419E37801245B001C439FE7CD
:101210000B20D0E760DB00006BDB000070DB000020
:10122000F7B54D680E002A0001210A402FD1042D88
:101230002DD90F242B68B7681C40092C14D169687C
:101240001B099BB24C100192A34200D85C1E31686E
:101250003448FFF741FC00282DD00F232A681340A3
:10126000092B1DD1012317E0032C10D10F4203D10C
:10127000132000F049FAFEBD7A100192FF2AF7D838
:101280001A0992B25B0F92001C40141BDFE70B207F
:10129000EFE701339A00AF509C42FADA0020EAE708
:1012A000032BFBD12B0001335A1BA242F6DC6A460A
:1012B0001279DA70F7E736687010F30719D4310045
:1012C0001948FFF709FC002822D1042E1ED90F234C
:1012D00032681340042B19D13000FFF7DFFB0028E0
:1012E00007D131001148FFF7F7FB00280ED012207C
:1012F000BFE70028FBDD8442F9DB0F232A68134097
:10130000092B07D1013080004751C7E71120B0E712
:101310002000F2E7032BC1D16B461B792D18EB702F
:10132000BCE7C04667DB00006BDB000070DB000041
:1013300070B501240868204207D1042805D90F257B
:1013400001680D40092D02D14468200070BD032DB5
:1013500008D10A0992B24B0F92002B40D31A5B00BE
:101360001C43F2E7042DF0D102F0AAFCFEF734FF93
:1013700040000443E9E7000010B5034A0D2103488B
:1013800004F0B6FC10BDC046F8DA0000F0DA000048
:1013900000207047042070470120704710B50020DE
:1013A00002F0A2FE10BD0020704700207047002010
:1013B00070470020704700207047002070470020D1
:1013C00070470020704700207047000010B5034AA6
:1013D0000D21034804F08CFC10BDC04604DC000065
:1013E0006CDC000070470378002B03D05AB2002A4F
:1013F00001DB013070473F229343C03B59424B41D0
:10140000C01803789343802BF4D10130F9E7000032
:10141000F8B50127060014000800394227D1042935
:101420003FD90F230A681A40042A3AD13C4213D10B
:10143000042C11D922681340042B0DD102F040FC7A
:101440000500200002F03CFC010028000BF0BAFB74
:1014500000282EDB1FD127E0E30722D502F030FC65
:101460000A2200210BF080FC0500601010E01740FC
:1014700015D1042A15D90F2312681340042B10D15B
:1014800020004D1002F01CFC0A2239000BF06CFC0D
:1014900085420EDB08DD002E09DC00200CE04D103B
:1014A000E3E70F22054B1A700136022EF5D804200F
:1014B00002E0042076173040F8BDC046B00200209C
:1014C000F8B5060000242B4BE500ED182B79032B13
:1014D00009D00134FF2CF6D1300004F01DFC041EAD
:1014E00046D1013C44E030000BF076FBE3B2020051
:1014F0003100180004F090FC002839D12A685168A6
:101500008842E6D08300D3189B680130F02BF7D1D6
:1015100001238000083012181A42DAD1042AD8D9DF
:101520000F21136819400429D3D11B0998B2012354
:101530000130800010181842CBD10428C9D90F22DD
:1015400003681340042BC4D102F0BAFB0327050043
:10155000092128000BF028FB0028BAD0013F451CC8
:10156000002FF5D1310028000BF062FB8542B0D18D
:101570002000F8BDA025002010B50124044002D0B1
:101580004410200010BD042810D90F230268134016
:10159000042B07D102F094FB21000A220BF0E4FB9C
:1015A0000400EEE7032B01D10430F5E70D22014BD7
:1015B0001A70E6E7B0020020012210B5024018D1EF
:1015C000042802D903681A0992B201230B4012D1F0
:1015D000042902D90B681B099BB20024934206D14F
:1015E00004309B000431C318984206D30124200024
:1015F00010BD0022E9E70023EFE704780A78002C09
:1016000001D1002AF2D0013001319442ECD0002403
:10161000EDE70000F7B50700009101933049314B29
:10162000002A02D002220A70013A00261A601B68C2
:10163000CE54BE4200DBF7BD009AB300D058294B10
:10164000274D1C68C8239B0065191C1B01231842E9
:1016500006D0254A4310210028000BF045FA09E086
:10166000224A002802D004281BD1214A2100280048
:101670000BF03AFA1A4C20000BF0AEFA194A019B13
:101680001060002B0BD07B1EB34208DD194B984233
:1016900005D8431C1360202222540022E254013654
:1016A000C7E7042819D90F2301680B40042B04D184
:1016B00002F006FB104A0300CDE7092B03D1436873
:1016C0000E4A5B10C7E7032B08D10A0992B2490FF3
:1016D00092000B40D31A0A4ABDE70123094ABAE730
:1016E000B1020020D40500200CE7000072DB0000EE
:1016F00078DB00001F0300003BED0000E4DE00008B
:10170000F3DE0000FEDE0000014B18700020704781
:10171000B002002070B502F073F8094C0100251DDD
:101720001F2228000BF070FA28000BF055FA042352
:1017300004308008000118432060200070BDC046BE
:101740008C020020C368F0B59D00836889B05D19E4
:101750000300183306930369069A9F00069B0290C4
:10176000DF19436901939B00D3180393D04B1B7877
:10177000002B26D17F222B68CE491C1213409B00E0
:101780005B58043501929F46029B587804F066FF2F
:101790000023029A137027E0C54B1B78002B10D151
:1017A0002B68019A1C121340C24A9B009B580435B7
:1017B000E9E7069B3A1DD11ABD4BD82928DD1A222C
:1017C0001A70029BBA4C9B6821780193EA1A029B1B
:1017D00092109B7812021A43029B587804F046FF3D
:1017E0000023029A23701370029B069A9B68019350
:1017F000ED1A029BAD10DD60069BFE1A029BB6102F
:101800001E61039B9B1A029A9B10536109B0F0BDA5
:1018100039001B7817000C60002BD2D12B68019A7D
:101820001C121340A34A9B009B580435ABE7069B50
:101830003A1DD11A9E4BD82902DD1A221A70C0E730
:1018400038001B7817002A68291D0260002B01D080
:101850000D00B6E76B68019A1C121340954A9B0075
:101860009B5808358FE7069B3A1DD11A904BD82913
:1018700002DD1A221A70A4E73900A4001B782C1983
:1018800017000C60002B9CD12B68019A1C1213408E
:10189000884A9B009B58043575E7069B3A1DD11A70
:1018A000834BD82902DD1A221A708AE73900170003
:1018B000814AA400A2581B780A60002B00D080E760
:1018C0002B68019A1C1213407A4A9B009B580435DE
:1018D00059E7043F784B3A68A400E250744B1B78F8
:1018E000002B00D06DE72B68019A1C121340714A3F
:1018F0009B009B58043546E76F4BA400E058FFF768
:101900003BFE6B4B06001B78002B09D1043F386867
:10191000FFF732FE0123861976001E43664BE65020
:10192000634B1B78002B00D04BE72B68019A1C12ED
:101930001340604A9B009B58043524E7069B391DE1
:10194000CA1A5B4BD82A02DD1A221A7039E70698A8
:10195000039C0122A04202D222000C3A12683800F5
:101960001B780F000260002B00D02AE72B68019A39
:101970001C1213404F4A9B009B58043503E7069AFC
:101980003B1D991A4A4AD82902DD1A23137018E719
:1019900006990398814218D202000C3A126847490E
:1019A00052106418A41AA40022583A601F00404B39
:1019B0001B78002B00D004E72B68019A1C121340FF
:1019C0003C4A9B009B580435DDE61821117000222B
:1019D000EBE7069B039A934219D213000C3B1B685A
:1019E000364A5B10A418043FE41A3A68039BA4002B
:1019F000E2502F4B1B78002B00D0E2E62B68019AB7
:101A00001C1213402B4A9B009B580435BBE618223E
:101A1000274B1A70EDE7069B039A934228D2274B77
:101A2000043FE61814000C3C23685B10F31A9B007B
:101A30009858FFF7A1FD04903868FFF79DFD2468D2
:101A4000049B6410341B1E18012376001E43039B65
:101A5000A400E650164B1B78002B00D0B1E62B6893
:101A6000019A1C121340134A9B009B5804358AE6C6
:101A700018220F4B1A70EDE7069B3A1DD11A0C4B3A
:101A8000D82902DD1A221A709BE639001700039A42
:101A9000A400A2581B780A60002B00D091E62B68A6
:101AA000019A1C121340034A9B009B5804356AE6B6
:101AB000B0020020E4DC0000982D0020FDFFFF3F75
:101AC000043F039B3A68A400E250D64B1B78002BDE
:101AD00000D076E62B68019A1C121340D24A9B0074
:101AE0009B5804354FE6039BA4001C192368043F50
:101AF00038685E10FFF740FD0123361876001E435C
:101B0000C84B26601B78002B00D05AE62B68019A40
:101B10001C121340C44A9B009B58043533E6069BB5
:101B2000A4003F1BBF4CBB420CD82378002B00D035
:101B300047E62B68019A1C121340BB4A9B009B5836
:101B4000043520E6B94802F0ABF82378002B00D02A
:101B500037E62B68019A1C121340B34A9B009B582E
:101B6000043510E6A300ED18002C00DA3CE6AD4B7E
:101B70001B78002B00D024E62B68019A1C1213401E
:101B8000A94A9B009B580435FDE5043F3B68042BA4
:101B900004D1A300ED18002C00DA25E6A14B1B7838
:101BA000002B00D00DE62B68019A1C1213409E4AB0
:101BB0009B009B580435E6E5043F3B68042B04D0AA
:101BC000A300ED18002C00DA0EE6964B1B78002BD4
:101BD00000D0F6E52B68019A1C121340924A9B0034
:101BE0009B580435CFE501233E1F306818420AD0C8
:101BF00018410138002809DB01234000A4001843E4
:101C00002D193060F0E5FFF7B7FCF2E7854B1B7844
:101C1000002B01D03700D4E52B68019A1C12134029
:101C2000814A9B009B5837000435ACE5FF206100DA
:101C300040000140FE38FF380143396002993B0003
:101C40008968241204916D1A0299AD1089782D02C9
:101C50000D43854005437D6006991700039A521A8B
:101C60009210824002439A60029B029A9C70E4B2F6
:101C70006F4BE400E35893606A4A1278002A03D05D
:101C800008331D0003979CE51D00019A9B680C35E5
:101C90001C121340644A9B009B58039773E53B1F3B
:101CA0001C68039A069B934232D10A20E30711D4A1
:101CB000042C18D90F2322681340042B16D12000BE
:101CC00001F0FEFF0AF088FFC8239B00984200D96C
:101CD00018000630643004F0D3F800280FD1043D1A
:101CE000069B039380E50720042CF3D02000431EBD
:101CF0009841FA234042FF3318400730EAE7029B3D
:101D00002100587804F0C4FC0023029A1370E7E71E
:101D1000039B039A0C3B1B6802995B109B00D31A30
:101D20000C3B1C601F1D1300083B1B685A108A7077
:101D3000D2B23F49D2005B0055589B0A029A9B00E1
:101D40009560ED18039B069A043B1B685B109B0093
:101D5000D3180393334B1B78002B00D031E52B684D
:101D6000019A1C121340304A9B009B5804350AE527
:101D70003B1F1868FFF700FCA40006003F1B1E284D
:101D800027DC00280DDC274B1B78002B00D018E542
:101D90002B68019A1C121340234A9B009B58043560
:101DA000F1E401F013FD033E361801F00FFD214B65
:101DB000801B9842F9D81B4B1B78002B00D000E504
:101DC0002B68019A1C121340174A9B009B5804353C
:101DD000D9E40123029A137001F0F8FC029B0A383F
:101DE00086195E6000E53B1F1868FFF7C5FBA4007D
:101DF00006003F1B00280DDC0A4B1B78002B00D08F
:101E0000DFE42B68019A1C121340074A9B009B5881
:101E10000435B8E4084B984210DD1D22014B1A70BE
:101E2000CFE4C046B0020020E4DC000010DF000078
:101E3000A02500203F420F0080EE36000123029AC9
:101E4000137001F0C3FCFA239B005E430A3E301876
:101E5000029B5860C8E4A300FF1A002320001A0068
:101E60003900FFF7D7FBD74ED74C3168200002F07E
:101E700047F9D64B31681860200004F0C3FA316886
:101E8000200004F00CFCD24B1B78002B00D098E40F
:101E90002B68019A1C121340CE4A9B009B580435B4
:101EA00071E4CB4BA4001B783F1B002B00D088E4CF
:101EB0002B68019A1C121340C64A9B009B5804359C
:101EC00061E4029804F040F8C14B1B78002B00D06D
:101ED00077E42B68019A1C121340BE4A9B009B5862
:101EE000043550E43B1F1B68002B58D13B000126F2
:101EF0000C3B186806402FD046103A0001217300B1
:101F0000083A0B431360002E00DC95E001217300BA
:101F10000B433A1F13603B00083B1B680B419B1BA4
:101F200004933B000C3B186808423BD0049BA40080
:101F30005B188B400B43039AA350A54B1B78002BD7
:101F400000D03EE42B68019A1C121340A14A9B006A
:101F50009B580435FFF717FC04281BD90F23026890
:101F60001340092B02D143685E10C6E7042B08D149
:101F700001F0A6FE0378002BBFD0FFF734FA01363C
:101F8000F8E7032B06D11609B6B2520FB60013407C
:101F9000F61AB2E719228E4B1A70FFF712FC5B108B
:101FA0005E1EB0E7042842D90F2302681340092BB4
:101FB00005D1049BA40002339B001B58BBE7042BF4
:101FC0002BD1039BA4001B19079301F079FE060097
:101FD000049C0134012C10DC3000FFF704FA831B51
:101FE0001800049302F080F8041E0ED001F068FE81
:101FF000049A31000AF04AFA07E03178013C0029DE
:1020000006D112220C00724B1A70079B1C6094E7D9
:102010003000FFF7E8F90600DCE7032B07D10122C7
:10202000049BA400C01803795B00134383E71922C3
:10203000674B1A70FFF7C5FB04357EE7A300069ACD
:10204000FB189B1AD82B08DD1A22614B1A70FFF778
:10205000B8FB01221C003A600437631E002CF8DC38
:102060005B4B1B78002B01D0FFF7ABFB2B68019A71
:102070001C121340574A9B009B580435FFF783FB03
:10208000069A3B1D9B1A524ED82B03DD1A23337040
:10209000FFF797FB069B039AA40093422AD23B1FAB
:1020A0001868FFF769FA011E21DD039B0C3B1A68D3
:1020B000521082421BDB9007801A474B4018C01811
:1020C000039B8000C2583B1B1A60414B3F1B1B788F
:1020D0000437002B01D0FFF774FB2B68019A1C1208
:1020E00013403C4A9B009B580435FFF74CFB2023D0
:1020F0003370EAE71823FBE7344BA4001A683B1B54
:102100001F001A60324B04371B78002B01D0FFF7F9
:1021100058FB2B68019A1C1213402E4A9B009B58B7
:102120000435FFF730FB3A1F1368042B02D13A0045
:10213000A4002D19264B1B78002B02D01700FFF7A7
:1021400040FB2B6801991C120B4022499B005B58F5
:1021500017000435FFF717FB043F3B68042B04D03E
:102160000023A4003B602D190437194B1B78002B6A
:1021700001D0FFF726FB2B68019A1C121340154A69
:102180009B009B580435FFF7FEFAA3009C46F81A03
:10219000002C23DC1C2200260D4B1A706346FF1A0C
:1021A0000B4B06601B780437002B01D0FFF709FBAF
:1021B0002B68019A1C121340064A9B009B58043559
:1021C000FFF7E1FAD4050020B1020020080000204A
:1021D000B0020020E4DC0000FCFFFF3F00210368A8
:1021E0005B1001268A008258164003D10D22D54B80
:1021F0001A70D3E75210934200DD130001318C4274
:10220000EFDC5E0001231E43C8E7A3009C46F81ADA
:10221000002C17DC1C220026CA4B1A706346FF1ADA
:10222000C84B06601B780437002B01D0FFF7C9FAB2
:102230002B68019A1C121340C34A9B009B5804351B
:10224000FFF7A1FA002103685B1001268A0082587B
:10225000164003D10D22BB4B1A70DFE75210934298
:1022600000DA130001318C42EFDC5E0001231E43D3
:10227000D4E73B000122083B1968A40011421DD09D
:102280003B1F1B68134219D0114113410022994290
:1022900000DA04323B1B1A60AA4B3F1B1B78043741
:1022A000002B01D0FFF78DFA2B68019A1C12134006
:1022B000A54A9B009B580435FFF765FA02203B1F97
:1022C0001A684042FFF7A4F83E1B3060E4E73B0089
:1022D0000120083B1968A40001421ED03B1F1A6868
:1022E00002421AD001415010CB0FD21788425341FD
:1022F0003A1B9B001360934B3F1B1B780437002B4A
:1023000001D0FFF75EFA2B68019A1C1213408E4A27
:102310009B009B580435FFF736FA01203B1F1A68D3
:102320004042FFF775F83E1B3060E4E73B00083B96
:1023300018683B1F1968A600BE1B0423814202D007
:10234000042802D80023336016E001231842F9D193
:102350000F2302681A40042AF4D1033A1142F1D142
:102360000429EFD90A681340042BEBD1FFF724F9B5
:10237000431E984180003060724BA4001B783F1BC5
:102380000437002B01D0FFF71CFA2B68019A1C12AE
:1023900013406D4A9B009B580435FFF7F4F93B004E
:1023A000083B18683B1F1968A600BE1B002381422A
:1023B00002D0042802D80423336016E00123184217
:1023C000F9D10F2302681A40042AF4D1033A1142CA
:1023D000F1D10429EFD90A681340042BEBD1FFF7A0
:1023E000EBF84342584180003060564BA4001B7804
:1023F0003F1B0437002B01D0FFF7E3F92B68019A4C
:102400001C121340504A9B009B580435FFF7BBF940
:102410003B000122083B1968A40011421ED03B1F5B
:102420001B6813421AD05B104A10D80FC9179A4282
:1024300041413B1B89001960424B3F1B1B7804370D
:10244000002B01D0FFF7BDF92B68019A1C12134035
:102450003D4A9B009B580435FFF795F93B1F1A68CE
:102460000120FEF7D5FF3E1B3060E5E73B0001226F
:10247000083B1968A40011421DD03B1F1B68134282
:1024800019D0114113410022994200DD04323B1B57
:102490001A602C4B3F1B1B780437002B01D0FFF731
:1024A00090F92B68019A1C121340274A9B009B58F5
:1024B0000435FFF768F93B1F1A680220FEF7A8FFF2
:1024C0003E1B3060E5E73B1F1B68A400043B5A1E1F
:1024D00093413A1B17009B0013601A4B04371B787B
:1024E000002B01D0FFF76DF92B68019A1C121340E5
:1024F000154A9B009B580435FFF745F93B00083B04
:102500001868FFF739F83B1F06001868FFF734F822
:102510000121A4003B1B1F00321852000A431A601D
:10252000084B04371B78002B01D0FFF74AF92B68C2
:10253000019A1C121340044A9B009B580435FFF774
:1025400022F9C046B0020020E4DC00003B00083B5A
:102550001868FFF711F83B1F06001868FFF70CF822
:102560000121A4003B1B1F00321A52000A431A60CB
:10257000EB4B04371B78002B01D0FFF722F92B68B7
:10258000019A1C121340E74A9B009B580435FFF741
:10259000FAF83B00083B1868FEF7EEFF3B1F060009
:1025A0001868FEF7E9FF02000121A4003B1B1F0091
:1025B000724352000A431A60D94B04371B78002B30
:1025C00001D0FFF7FEF82B68019A1C121340D54A80
:1025D0009B009B580435FFF7D6F83B1F1868FEF7A1
:1025E000CBFF061E17D11F23CD4A1370A4003B1B3F
:1025F0001F001E60CA4B04371B78002B01D0FFF769
:10260000E0F82B68019A1C121340C64A9B009B58A5
:102610000435FFF7B8F83B00083B1868FEF7ACFF3D
:10262000310007F00BFE012346001E43DEE73B1F8F
:102630001868FEF7A1FF061E17D11F23B84A1370B2
:10264000A4003B1B1F001E60B54B04371B78002BFA
:1026500001D0FFF7B6F82B68019A1C121340B14A5B
:102660009B009B580435FFF78EF83B00083B186829
:10267000FEF782FF310007F0C7FE01234E001E4324
:10268000DEE73B1F1868FEF777FFC217801850403F
:102690000122A4003B1B1F00400010431860A04B08
:1026A00004371B78002B01D0FFF78BF82B68019AB9
:1026B0001C1213409B4A9B009B580435FFF763F89C
:1026C000A3000793FB1A0493012C2CD11868FEF782
:1026D00053FF01230600C4179C43E418B44202DCF4
:1026E000330026001C000134A41B0AF0CBF92100A2
:1026F00007F08AFE01238E1976001E43049B1E609C
:10270000079BFF1A864B04371B78002B01D0FFF77D
:1027100058F82B68019A1C121340824A9B009B5860
:102720000435FFF730F8022C0AD1049B1868FEF735
:1027300023FF049B04005868FEF71EFF0600CDE748
:1027400064240126CFE7A300FE1A31002000049381
:1027500001F05CFE049B3060FF1A714B04371B785C
:10276000002B01D0FFF72DF82B68019A1C121340A3
:102770006C4A9B009B580435FFF705F83B00083B6B
:102780001868FEF7F9FE3B1F06001868FEF7F4FE16
:1027900002000121A4003B1B1F00324052000A43EB
:1027A0001A605F4B04371B78002B01D0FFF709F844
:1027B0002B68019A1C1213405A4A9B009B580435FF
:1027C000FEF7E1FF3B00083B1868FEF7D5FE060068
:1027D0003B1F1868FEF7D0FE32000121A4003B1B0E
:1027E0001F00024352000A431A604D4B04371B7806
:1027F000002B01D0FEF7E5FF2B68019A1C12134055
:10280000484A9B009B580435FEF7BDFF3B00083B40
:102810001868FEF7B1FE06003B1F1868FEF7ACFE15
:1028200032000121A4003B1B1F00424052000A431A
:102830001A603B4B04371B78002B01D0FEF7C1FF19
:102840002B68019A1C121340364A9B009B58043592
:10285000FEF799FF3B1F1868FEF78EFEC04301226A
:10286000A4003B1B1F004000104318602C4B043792
:102870001B78002B01D0FEF7A4FF2B68019A1C12D5
:102880001340284A9B009B580435FEF77CFF3B0011
:10289000083B1868FEF770FE06003B1F1868FEF73D
:1028A0006BFE320082400121A4003B1B1F0052003E
:1028B0000A431A601A4B04371B78002B01D0FEF72D
:1028C00080FF2B68019A1C121340164A9B009B58EC
:1028D0000435FEF758FF3B00083B1868FEF74CFE36
:1028E00006003B1F1868FEF747FE32000241012137
:1028F000A4003B1B1F0052000A431A60084B043718
:102900001B78002B01D0FEF75CFF2B68019A1C128C
:102910001340044A9B009B580435FEF734FFC04621
:10292000B0020020E4DC00003B000C3B1868FEF71E
:1029300023FE3B00083B06001868FEF71DFEF1175A
:102940000200C317300007F0B1FD3B1F0490059152
:102950001868FEF711FE02000498059907F05AFD69
:102960000123A4003E1B370040001843E54B3060B4
:102970001B780437002B01D0FEF723FF2B68019A48
:102980001C121340E04A9B009B580435FEF7FBFEE7
:10299000A300FE1A310020000493FEF747FB049BBE
:1029A0003060FF1AD74B04371B78002B01D0FEF79D
:1029B00008FF2B68019A1C121340D34A9B009B58B6
:1029C0000435FEF7E0FEA300FF1A39002000FEF7F1
:1029D00049FBCC4B1B78002B01D0FEF7F2FE2B6895
:1029E000019A1C121340C84A9B009B580435FEF7FD
:1029F000CAFEA300FE1A310020000493FEF772FB0A
:102A0000049B3060FF1ABF4B04371B78002B01D0AA
:102A1000FEF7D7FE2B68019A1C121340BA4A9B009E
:102A20009B580435FEF7AFFEA300FF1A39002000C3
:102A3000FEF7F6FBB34B1B78002B01D0FEF7C1FE6F
:102A40002B68019A1C121340AF4A9B009B58043517
:102A5000FEF799FEA300FE1A310020000493FEF752
:102A600067FC049B3060FF1AA64B04371B78002BD1
:102A700001D0FEF7A6FE2B68019A1C121340A24A51
:102A80009B009B580435FEF77EFE3B1F186801F043
:102A900017F93A000121083A12680300A4000A421B
:102AA00029D1042A0CD910680F22104001380828B7
:102AB0000FD807F02FFB052026220E0E0E0E240045
:102AC000924918000AF07EF8434258413B1B8000AF
:102AD00018608C4B3F1B1B780437002B01D0FEF78E
:102AE00070FE2B68019A1C121340874A9B009B586A
:102AF0000435FEF748FE8649E3E78649E1E7864963
:102B0000DFE78649DDE7069B3E1DF31A7D4CD82B97
:102B100003DD1A232370FEF754FE00F061FE01224C
:102B20003B0040001043186023783700002B01D091
:102B3000FEF747FE2B68019A1C121340724A9B0055
:102B40009B580435FEF71FFE069B3E1DF31A6D4C85
:102B5000D82B03DD1A232370FEF733FE00F036FE78
:102B60006F4A4000104001223B0010431860237858
:102B70003700002B01D0FEF724FE2B68019A1C12AF
:102B80001340614A9B009B580435FEF7FCFD069AF2
:102B90003B1D9B1A5B4CD82B03DD1A232370FEF7D9
:102BA00010FE00F01DFE5F4B1A68831A904201D29E
:102BB0005D4A9B1801213A005B000B4313602378A8
:102BC0000437002B01D0FEF7FCFD2B68019A1C1284
:102BD00013404D4A9B009B580435FEF7D4FD00F08E
:102BE000FFFD504BA4001860464B3F1B1B78002B89
:102BF00001D0FEF7E6FD2B68019A1C121340424AF1
:102C00009B009B580435FEF7BEFD00F0F7FDA300C6
:102C1000002810D1FF1A3B4B1B78002B01D0FEF788
:102C2000D0FD2B68019A1C121340374A9B009B5819
:102C30000435FEF7A8FD3E00FF1A012320001A000C
:102C40003900FEF7E7FC394C2068643003F018F9CE
:102C5000002803D1043D3700FEF7C6FD029B216822
:102C60005A78334803F02DFD0123029A137000F0C7
:102C7000ADFD304B22681B68063253431818FFF72E
:102C8000E7F800F0BBFDA300002810D1FF1A1D4B90
:102C90001B78002B01D0FEF794FD2B68019A1C12C3
:102CA0001340194A9B009B580435FEF76CFD3E000B
:102CB000FF1A2000012300223900FEF7ABFC1B4C59
:102CC0002068643003F0DCF80028C3D0184803F013
:102CD00083FAC9E7A4003E1BFEF71CFD3700094B31
:102CE00030601B780437002B01D0FEF76AFD2B689B
:102CF000019A1C121340044A9B009B580435FEF7AE
:102D000042FDC046B0020020E4DC000020DF0000ED
:102D100028DF00002FDF000036DF00003BDF00006F
:102D2000FEFFFF7FDC05002037894100D40500202D
:102D3000B102002004000020FB4BA4001B783F1BC5
:102D4000002B01D0FEF73DFD2B68019A1C121340A9
:102D5000F64A9B009B580435FEF715FDA4003E1B68
:102D6000300000F078FD3700EF4B30601B780437FF
:102D7000002B01D0FEF725FD2B68019A1C12134091
:102D8000EA4A9B009B580435FEF7FDFCA4003E1B5D
:102D9000300000F062FD3700E34B30601B780437F1
:102DA000002B01D0FEF70DFD2B68019A1C12134079
:102DB000DE4A9B009B580435FEF7E5FCA300FE1A93
:102DC00031002000049300F025FC049B3060FF1AC2
:102DD000D54B04371B78002B01D0FEF7F2FC2B6893
:102DE000019A1C121340D14A9B009B580435FEF7F0
:102DF000CAFCA4003F1B380000F032FDCA4B1B7810
:102E0000002B01D0FEF7DDFC2B68019A1C12134049
:102E1000C64A9B009B580435FEF7B5FCA300FE1A7A
:102E200031002000049300F027FC049B3060FF1A5F
:102E3000BD4B04371B78002B01D0FEF7C2FC2B687A
:102E4000019A1C121340B94A9B009B580435FEF7A7
:102E50009AFCA4003F1B380000F048FDB24B1B78E1
:102E6000002B01D0FEF7ADFC2B68019A1C12134019
:102E7000AE4A9B009B580435FEF785FC01212000DB
:102E800000F01CFDA84B1B78002B01D0FEF799FC2D
:102E90002B68019A1C121340A44A9B009B580435CE
:102EA000FEF771FC0021200000F008FD9E4B1B780E
:102EB000002B01D0FEF785FC2B68019A1C121340F1
:102EC0009A4A9B009B580435FEF75DFCA4003E1B0C
:102ED000300000F039FD3700934B30601B78043729
:102EE000002B01D0FEF76DFC2B68019A1C121340D9
:102EF0008E4A9B009B580435FEF745FCA4003E1B00
:102F0000300000F035FD3700874B30601B78043708
:102F1000002B01D0FEF755FC2B68019A1C121340C0
:102F2000824A9B009B580435FEF72DFCA4003F1BF2
:102F3000380000F0F1FC7C4B1B78002B01D0FEF731
:102F400040FC2B68019A1C121340784A9B009B5846
:102F50000435FEF718FCA4003F1B380003F0AAFF5D
:102F6000714B1B78002B01D0FEF72BFC2B68019ACC
:102F70001C1213406D4A9B009B580435FEF703FC5E
:102F8000A4003E1B300004F04FF83700664B306061
:102F90001B780437002B01D0FEF713FC2B68019A35
:102FA0001C121340614A9B009B580435FEF7EBFB53
:102FB000A4003F1B380003F025FF5B4B1B78002B60
:102FC00001D0FEF7FEFB2B68019A1C121340574AF2
:102FD0009B009B580435FEF7D6FBA4003E1B300037
:102FE00003F02AFF3700504B30601B780437002B6A
:102FF00001D0FEF7E6FB2B68019A1C1213404B4AE6
:103000009B009B580435FEF7BEFBA300FF1A390056
:10301000200001F06FFD444B1B78002B01D0FEF720
:10302000D0FB2B68019A1C121340404A9B009B580E
:103030000435FEF7A8FBA300FF1A3900200001F0B9
:1030400079FB394B1B78002B01D0FEF7BAFB2B68BC
:10305000019A1C121340354A9B009B580435FEF719
:1030600092FBA300FF1A3900200001F0FBFB2E4B5E
:103070001B78002B01D0FEF7A4FB2B68019A1C12D1
:1030800013402A4A9B009B580435FEF77CFBA300A3
:10309000FF1A3900200001F00DFC234B1B78002B98
:1030A00001D0FEF78EFB2B68019A1C1213401F4AB9
:1030B0009B009B580435FEF766FBA300FE1A310007
:1030C0002000049304F09AF8049B3060FF1A164B1A
:1030D00004371B78002B01D0FEF773FB2B68019A95
:1030E0001C121340114A9B009B580435FEF74BFB02
:1030F000A300FE1A31002000049304F087F8049B1B
:103100003060FF1A084B04371B78002B01D0FEF704
:1031100058FB2B68019A1C121340044A9B009B58D1
:103120000435FEF730FBC046B0020020E4DC0000AE
:10313000A300FE1A31002000049304F06FF8049BF2
:103140003060FF1AAA4B04371B78002B01D0FEF722
:1031500038FB2B68019A1C121340A64A9B009B580F
:103160000435FEF710FBA300FE1A31002000049383
:1031700003F024FD049B3060FF1A9D4B04371B783D
:10318000002B01D0FEF71DFB2B68019A1C12134087
:10319000984A9B009B580435FEF7F5FAA300FF1AE6
:1031A0003900200001F026FC914B1B78002B01D048
:1031B000FEF707FB2B68019A1C1213408D4A9B00F7
:1031C0009B580435FEF7DFFAA300FF1A39002000F0
:1031D00001F098FB864B1B78002B01D0FEF7F1FA2B
:1031E0002B68019A1C121340824A9B009B5804359D
:1031F000FEF7C9FAA300FE1A31002000049301F083
:10320000FDFA049B3060FF1A794B04371B78002BC2
:1032100001D0FEF7D6FA2B68019A1C121340754AAA
:103220009B009B580435FEF7AEFAA300FF1A390045
:10323000200001F0ABFA6E4B1B78002B01D0FEF79B
:10324000C0FA2B68019A1C1213406A4A9B009B58D3
:103250000435FEF798FA002C79DD3B1F1E68012C1F
:103260000CD1264207D1042E05D90F233268300035
:103270001340042B11D001235B4213E0022CFAD13E
:103280003B00083B186801231842F4D10428F2D906
:1032900002680E331340042BEDD100F011FDFEF750
:1032A0000FF90300A200BF1A5A1C50D00020022CB4
:1032B00011D101223240824223D1042E21D90F2183
:1032C0003068014009291CD171684810C0B28100E2
:1032D000914211D17F18FF2B1BD81C0204433A00E6
:1032E000069B0C32D31AD82B01DCFEF79FFC1A2266
:1032F0003F4B1A70FEF765FAB418A468BC5004324C
:10330000E6E70B223A4B1A7000233B600437FEF7C6
:1033100058FA069A0299BA1A86009210BE1B0A61E0
:10332000310098470022344B371D1A60304B306013
:103330001B78934201D0FEF744FA2B68019A1C12C5
:1033400013402C4A9B009B580435FEF71CFA0023BF
:103350003B60274B3A1D1B78002B02D01700FEF76D
:1033600030FA2B6801991C120B4022499B005B58D4
:1033700017000435FEF707FA069B029AFB1A9B100A
:103380001361A300FF1A3900200002F063FF184BFD
:103390001B78002B01D0FEF714FA2B68019A1C123F
:1033A0001340144A9B009B580435FEF7ECF9069B2A
:1033B000029AFB1A9B101361A300FE1A3100200031
:1033C000049302F047FF049B3060FF1A084B043758
:1033D0001B78002B01D0FEF7F4F92B68019A1C1220
:1033E0001340044A9B009B580435FEF7CCF9C046B5
:1033F000B0020020E4DC0000E40F00200023F7B559
:103400005A1E0192002B07DA01F08AFB03F03AF80A
:1034100003F0B6F91923019300263000194B1968FF
:10342000B14212DD184B1A6801328A420FDAF024D9
:103430001A601D68154F6C43E35D002B1FD0E41923
:10344000022B06D12000FEF77DF9019BD8E7002270
:10345000EDE7012B0DD1002801D100F0B7F9F022E2
:103460006A43BB185B680A49C31A8B4201D802231E
:10347000BB54F0235D43054BEB5C022BE2D00136DD
:10348000CCE7C046D805002000000020401C0020EA
:103490003F420F0080220B4B52001A600121A822EC
:1034A000A920094BD20019649A58C00005321A505D
:1034B00006481A50C122C020920000039850044BC5
:1034C0001970704700E100E0008000404C050000EA
:1034D0000306002004207047F8B550C901232200DC
:1034E0001A40101E2DD03340181E2AD06410002020
:1034F0001C2C26D81D4B761035009E4200DD1D0089
:103500001B4F3B5D012B05D00121200005F0F2F996
:1035100001233B55174B1B78002B01D1FFF7BAFF56
:103520000023154A9E420DDCFF2514491448D65C41
:10353000B44202D15E007052D5540133042BF6D14F
:103540000420F8BDD15C8C4203D10C4A5B009D5233
:10355000F6E70133042BF5D10023D15CFF2901D11B
:10356000D454F2E70133042BF7D1E9E788130000C4
:10357000E4050020030600201C0000200E000020AF
:10358000DC05000070B530C9012322001A40101E6E
:103590001BD02B40181E18D064101C2C00D90024FE
:1035A000154E335D012B05D00121200005F0A2F955
:1035B0000123335569100800104A1038104B90420F
:1035C00004D9012252421A60042070BD1C600D48CB
:1035D00006F034FE0C4B040018800C4B1B78002BBB
:1035E00001D1FFF757FF0122094B9A64A922D200AB
:1035F000995864189C50E7E7E40500209086010084
:103600001800002020A107000C0000200306002065
:1036100000800040F8B501240B6806000D0023422D
:1036200004D10D20FEF770F82000F8BD5B102000DB
:10363000052BFAD80E4A9B009C580E4F3B5D002B81
:1036400005D00021200005F055F900233B55012E3F
:1036500006DD6B68042B03D10221200005F04AF936
:10366000200004F0F5FF012440002043DDE7C046C0
:10367000B0DF0000E405002070B501240D6825428C
:1036800004D10D20FEF740F8200070BD6D101C2DF8
:1036900017D80024012804DD4C68043C63425C41D7
:1036A0006400094E735DA34204D02100280005F098
:1036B00021F97455280005F051F903000420012B6D
:1036C000E3D00020E1E7C046E4050020F8B501267C
:1036D0000D683400B04200DD4C682B003340181EEA
:1036E0000BD023003340181E07D06D10002D05DCD1
:1036F000A12300201E4ADB00D650F8BD6410002034
:103700001C2CFAD81B4F3B5D012B04D0012120005B
:1037100005F0F0F83E552900174806F08FFD0A2104
:10372000053006F08BFD154BA400E258144B120235
:103730001343A2221349D2008B50134C0C4B9C50C4
:10374000124C1951012412495C50124B1969002185
:103750009950114A904200DD1000A8228021D20029
:103760009850012289005A5004201A60C5E7C046CB
:1037700000F00140E405002000B4C404F8F00000AB
:10378000030003000060004040A100401405000059
:103790000405000000A00040FFFF0000030010B57A
:1037A0000120002B02DC1B30FDF7AEFF10BD042012
:1037B000704710B5002803DC1C20FDF7A5FF10BDE5
:1037C0000B680020DB07FAD40D30F6E70122034B2B
:1037D0001A64A822D20098587047C0460080004062
:1037E0000122054B10B51A64A822FA21D20098587C
:1037F000890006F099FC10BD008000400120704750
:1038000000487047C8DF00001D20704770B5054EA6
:103810000400335C0D008B4202D005F06BF8355587
:1038200070BDC046E405002070B50024084D635DFE
:10383000012B09D10021200005F07AF80021200099
:1038400005F058F80023635501341D2CEED170BDEE
:10385000E405002070470D2070473B2070470000B2
:10386000F8B501260568354202D04468344203D1D8
:103870000D20FDF749FFF8BD6D101C2DFBD80A4F38
:103880007B5D012B04D03100280005F033F87E5514
:10389000064964108C4202DCE143C917214028002C
:1038A00004F05CFFE7E7C046E4050020FF030000EA
:1038B00010B50800FFF7D4FF002010BD70B504005C
:1038C0000D001C280ED8084E335C012B04D00121BA
:1038D00005F010F801233355290020004D1EA941A1
:1038E00005F026F870BDC046E4050020036810B559
:1038F000DA0703D40D20FDF707FF10BD416858100B
:1039000004394A425141FFF7D9FFF6E710B50800E4
:10391000FFF7ECFF002010BD37B569460A00064BE3
:1039200030CB30C203680220042B02D100F09AFF92
:1039300037BD00F0BFFFFBE748DF000010B508000F
:10394000FFF7EAFF002010BD10B5084C6379002B8B
:1039500005D00021052004F0CDFF00236371052070
:1039600004F0FCFF43425841800010BDE4050020F4
:1039700010B5084CE37A002B05D000210B2004F091
:10398000B9FF0023E3720B2004F0E8FF43425841E3
:10399000800010BDE4050020A02200230349D200CE
:1039A0008B50034910328B507047C04600F00140E5
:1039B00000600040F7B52F4D2F4EEB6C002B14D05C
:1039C000A9240023E4003759EB642C4B1868002825
:1039D0000BDB2B4B19784A425141C9B2197004F0E4
:1039E000A7FF284B1B88DF1937512B6D002B38D0D0
:1039F0000021254B254FF45829653A780193244D31
:103A00008A4206D02B68032B03D8224AD05C04F0EC
:103A10008FFF2B68204A0133134004D50422013B59
:103A20005242134301331B4900228C462B60042B66
:103A300018D06046C05C591CFF2802D10B0001223F
:103A4000F5E7002A00D02B60012104F071FF01236B
:103A50003B702B68114A5B009B5A0C34E418019BA5
:103A6000F450F7BD01235B422B6000233B700C4BED
:103A7000F4E7C046FC8000400080004018000020B1
:103A8000020600200C0000204C050000010600206A
:103A9000E00500201C000020030000800E00002034
:103AA0005C460000084B094AFF201A805A809A8021
:103AB000DA800023064A07491370074A08704870E5
:103AC0008870C870136070470E000020DC0500008D
:103AD000010600201C000020E00500200122024B0E
:103AE00052421A607047C0461800002010B5034AC1
:103AF0000C21034802F0FCF810BDC04650DF000066
:103B000043E80000E12170B54902194804F016FBB2
:103B1000002401220320174B17491A615C5004311D
:103B200058508018083158501A60063004F08AFD49
:103B3000FF21124AA15401341D2CFBD10122002087
:103B40000F4B01001A6004230E4A0F4D1468002C1D
:103B5000FCD02C680002013B20431160002BF5D102
:103B600001220A4B1A6004F0A5FC01F025F970BD92
:103B7000C81B00200080004004050000E405002070
:103B800000D0004000D1004008D5004004D00040E3
:103B9000F8B50B4E070030000D0004F017FB0400D1
:103BA000A84200DD2C003D00EB1B9C4205DD3000EF
:103BB00004F016FB28700135F6E72000F8BDC0467A
:103BC000C81B002010B50100014804F0BFFA10BD69
:103BD000C81B002010B5054C200004F0C5FAE121F7
:103BE0002000490204F0AAFA10BDC046C81B0020FC
:103BF000C3070CD4064B1B68834208D8054B1B68CF
:103C0000984204D8031F1B68002B00D0180070478F
:103C10000C060020080600200023012210B50A48E7
:103C2000990001334250642BFAD1084C084B002113
:103C30001A602000074A08F045FC074B074A6360FA
:103C4000074B1A6010BDC046982D002010060020BA
:103C500008000020D40900003027000014060020CE
:103C60000406002010B5044B044A1A60044B054AB0
:103C70001A60FFF7D1FF10BD0C06002010060020CF
:103C800008060020E40F0020044B1B681868000998
:103C900080B20238C343DB17184070470406002087
:103CA00000B59BB00200054901A808F04FFF01A82C
:103CB00002F0AEFA02F064FDFCE7C04692E00000BC
:103CC0000B4BC20704D4042804D80A4B00D00A4B7B
:103CD000180070470F2203681A40031D042AF7D00A
:103CE000064B092AF4D0064B032AF1D0054BEFE727
:103CF0006CE0000078DB000072DB000076E0000082
:103D000086E000007DE000000020064A0649131FFF
:103D1000186013681B099BB202339B00D2188A42B9
:103D2000F5D3704714060020E40F0020F7B50F24E8
:103D30000126314B314A1968314B324D18681368EE
:103D40001F002740072F26D813681B099BB2023398
:103D50009B00D218AA42F2D300242B4EA500AD1925
:103D60002868FFF745FF01342860642CF6D1274C02
:103D70002068FFF73DFF2060254C2068002802D016
:103D8000FFF736FF20600025224B1B680093009B45
:103D90009D4214DBF7BD1B099BB29B00D3189A42CE
:103DA000D2D01F68374208D1B94206D2B84204D3F4
:103DB000043F3F68002F00D01F60043BEFE7F02373
:103DC0006B43154A9B181A78002A01D10135DEE7AA
:103DD0001F693C2300266B43DB199B0001930136CE
:103DE000BB1BF3D4019BB4001C1B0B4B1C19A0691B
:103DF000FFF7FEFEA061F2E70C060020140600208B
:103E000008060020E40F0020982D00200800002064
:103E1000E40F0020D8050020401C0020F7B5012445
:103E2000204246D1234B1B689C46984241D3224BEB
:103E30001B68019398423CD8031F1B68002B38D1A4
:103E40000200036800941B099BB2002B0FD100995C
:103E5000131F196090422CD015682B1F1B68990006
:103E600069180C68013B14600A602A00EDE79D00A8
:103E700055192968009C214219D18C4517D8019CFD
:103E80008C4214D30E1F3468002C10D10F680F34ED
:103E90003C40072C08D92F60151F2B600B680A6067
:103EA0001B099BB20A00D0E700993160CDE7013BC6
:103EB000CBE7F7BD0C060020080600200D4970B5C1
:103EC0000A000D4D1368141F1B0926689BB2981C2D
:103ED000002E0BD000238A4200D00B002360830009
:103EE000C91880001218AA42ECD370BD1B011360E0
:103EF000F7E7C04614060020E40F0020F8B5124C86
:103F000027000F223B681D09ADB213420DD06E1C75
:103F1000B600A74204D032003900200008F0BFFAF2
:103F20000022A3190436A4191A600235AD00074B0C
:103F30007F199F42E5D31B1B9B10013B1B01236094
:103F4000034B1C60F8BDC04614060020E40F00209F
:103F500004060020F0B59BB0FFF738FC00240700F2
:103F6000214AA300D0580134FFF758FF642CF7D141
:103F70001E4B1868FFF752FF1D4B1868002801D030
:103F8000FFF74CFF00261B4B1B689E4217DBFFF719
:103F900095FFFFF7CBFEFFF7B1FFFFF717FC164BBE
:103FA000C21B1B6815491B6801A81B099BB2023B79
:103FB00008F0CCFD01A802F02BF91BB0F0BDF025F4
:103FC00075430F4BED182B78002B01D10136DAE742
:103FD0002B695C1E002CF9DBA300EB189869FFF736
:103FE0001DFF013CF6E7C046982D00200800002088
:103FF000E40F0020D8050020040600204CE000005B
:10400000401C0020F7B5174D4F1C2B6806001B689D
:104010000C001B099BB201929F420BDBFFF79AFF3A
:104020002B681B681B099BB29F4203DB0A20FDF72C
:104030006BFBFEBD2868A71CBA00DB1B81181B01A7
:104040000B6029600021031F19600F231E4003002D
:104050002401264340C3083A9A189A42E9D90199A3
:1040600002C3FAE704060020F7B50300012213405B
:1040700004000D000193002B2BD1174B1B688342CA
:1040800027D8164B1B68834223D90F23144F38605F
:1040900000681840FFF7B6FF019B3C68061E3B60B6
:1040A00017D0236804301B099BB29D4200DD1D0020
:1040B000AA00211D251F08F0E9F9FFF725FE2E6053
:1040C000FFF734FE00232B602268064B1340236069
:1040D00034002000FEBDC0460C060020080600206B
:1040E000E40F0020F0FF0F000323043010B5C117C8
:1040F00019400918891000220420FFF783FF10BD22
:1041000070B5050008000C00FFF7EEFF0023002843
:1041100004D170BDE95CC21811710133A342F9DB0F
:10412000E343DB171C40002304192371F1E7F0B5CA
:104130000C009BB0022804DC1C20FDF7E5FA1BB044
:10414000F0BD01230868184206D1042804D90F26BF
:1041500001683140042901D00E20EEE761680D00AE
:104160001D40F9D10429F7D90A683240042AF3D155
:10417000A2681A4201D10D20DFE7FFF7A1FD06007A
:104180006068FFF79DFDA768010001AC7F1030005B
:10419000257003F0FDFB39006423220003F05DFC71
:1041A000200008F019FD01002000FFF7A9FFC6E775
:1041B00010B51C4CA544041E02D1FFF795FF0BE07F
:1041C00003F0FEFA0138062828D805F0A3FF0909F4
:1041D00011182904240000208023DB009D4410BD19
:1041E000200003F069FB011B2000FFF789FFF3E7C4
:1041F000200003F00FFB430001201843ECE780226E
:104200006946D200200003F01CFB684608F0E4FC7D
:1042100001006846E9E704210348E6E70020CCE70F
:104220000420D9E700FCFFFFD8E0000070B50C00C7
:10423000022803DC1C20FDF767FA70BD0123086823
:10424000184206D1042804D90F2501682940042901
:1042500001D00E20EFE761681942FAD10429F8D99C
:104260000A682A40042AF4D1A2681A4201D10D201A
:10427000E1E7FFF725FD05006068FFF721FDA46871
:1042800001006410280003F083FB210003F0C0FB51
:10429000FFF78EFFD1E770B50D00012803DC1C206D
:1042A000FDF732FA70BD01240868204206D10428C7
:1042B00004D90F2102680A40042A01D00E20EFE73A
:1042C0006A682242FAD1042AF8D913680B40042BF9
:1042D000F4D1FFF7F5FC06006868FFF7F1FC010078
:1042E000300003F055FB03F0D7FB40002043D9E733
:1042F000F8B507000C001C20012F0BDD0125086814
:10430000284206D1042804D90F2102680A40042A51
:1043100003D00E20FDF7F8F9F8BD62682A42F8D103
:10432000042AF6D913680B40042BF2D1FFF7C8FC1E
:1043300006006068FFF7C4FC0100022F14D0A468D7
:104340002C4211D06410300003F022FB050003F072
:1043500037FA012811D1002C02DD0135012C06D1DC
:104360002800FFF725FFD7E701246442EBE7280088
:1043700003F0AFFA013C0500F0E70228F0D1002C71
:10438000EEDD0135012CEBD000222800110003F0F6
:10439000D2FA03F09EFA013C0500F3E710B50124C0
:1043A0000868044016D04410200006F0DBF91549D7
:1043B00006F0A6F807F08CFF04F0DEFB0022124B9B
:1043C00007F040F904F080FB07F012FF43000120E2
:1043D000184310BD042810D90F2302681340042B82
:1043E00007D1FFF76DFC21000A2208F0BDFC040094
:1043F000DAE7032B01D10430F5E70D20FDF784F94E
:10440000D2E7C046D30237390000D040086870B503
:1044100001240500254006D1042804D90F23026891
:104420001340042B03D00E20FDF76EF970BDFFF78B
:1044300047FC03782900233B5A4253411022C018FD
:1044400008F092FC80239B05C218044B9A4201D9C4
:104450001420E9E740002043E8E7C046FFFFFF3FA4
:1044600010B5034A0621034801F042FC10BDC046C6
:10447000A8E00000A3E000000020704710B51E2057
:10448000FDF742F910BD10B51E20FDF73DF910BD36
:1044900010B51E20FDF738F910BD10B51E20FDF730
:1044A00033F910BD10B51E20FDF72EF910BD10B563
:1044B0001E20FDF729F910BD10B51E20FDF724F9C7
:1044C00010BD10B51E20FDF71FF910BD10B51E2040
:1044D000FDF71AF910BD10B51E20FDF715F910BD36
:1044E00010B51E20FDF710F910BD10B51E20FDF708
:1044F0000BF910BD10B51E20FDF706F910BD10B563
:104500001E20FDF701F910BD10B51E20FDF7FCF8C7
:1045100010BD10B51E20FDF7F7F810BD10B51E2018
:10452000FDF7F2F810BD10B51E20FDF7EDF810BD37
:1045300010B51E20FDF7E8F810BD10B51E20FDF7E0
:10454000E3F810BD10B51E20FDF7DEF810BD10B564
:104550001E20FDF7D9F810BD10B51E20FDF7D4F8C8
:1045600010BD000010B5034A1821034801F0C0FB3C
:1045700010BDC04614E10000D4E100000120034B4F
:104580001860034B1B6883401843704700100020DD
:10459000E80F0020F0B5EFF310810123194083F3F9
:1045A0001088134AA1261268124D013A9340A022A6
:1045B000114FD205F600002B17D02C6894510342FE
:1045C0000BD0C046C046C046C046C046C046C046E6
:1045D000C0462C68D4515B08EDE7D451C046C046B4
:1045E000C046C046C046C046F5E781F31088F0BD1E
:1045F00020000020F40F00200C05000030B585B02D
:1046000001AD0C220649280007F040FF0024285D78
:1046100001210134FFF7FAF80C2CF8D105B030BDB8
:1046200010E30000F7B56A463B4B01AE13800A2346
:1046300093703A4B33801C23B370FFF7C7F8384BA5
:10464000384DC0182B68984201D200232B602C688B
:10465000002C41D1375D01213800FFF7D7F8013434
:104660000021380004F064F9032CF3D10024012761
:104670006B461E5D39003000FFF7C8F80134390081
:10468000300004F055F9032CF2D1C8200138C0469F
:10469000C046C046C046C046C046C046C046C046EA
:1046A000C046C046C046F1D16B4600211878FFF7DE
:1046B000ADF86B4600215878FFF7A8F86B4600214B
:1046C0009878FFF7A3F8FFF781F8FA2300241B017D
:1046D000C01828602000FEBDFFF778F82B68002482
:1046E0009842F7D3032003F0B3FF0600042003F041
:1046F000AFFF36180A2003F0ABFF0B4B9B1B181AB9
:104700000A4BA04206DB18600023094A2B601360A5
:104710000124DFE71C60F7E7030400001A1B000018
:1047200010270000F80F0020E3030000E80F00202E
:10473000001000200022054B10B51A60044B1B68C6
:10474000934201D002F0DCFF002010BDFC0F0020DE
:10475000EC1A002010B5041E0CDA0024084BA4004B
:10476000E2581F231A401E3B9340064A1360064A34
:10477000136010BDFFF748F8A042EEDDEEE7C0463B
:10478000F8F00000F40F002018050050020008683F
:1047900010B5C3070FD540101823012A03DD4A685E
:1047A000042A00D10833054A1360FFF753F8FFF7D6
:1047B000D1FF002010BD01204042EDE72000002085
:1047C00010B50124044002D04410200010BD04287C
:1047D00010D90F2302681340042B07D1FFF770FA9A
:1047E00021000A2208F0C0FA0400EEE7032B01D1F1
:1047F0000430F5E70D20FCF787FFE6E70868F8B519
:10480000C3071AD5FFF7DCFF0300203B5E2B25D83A
:104810000520434301221D180020114E9D4219D04E
:1048200005211024F75C3C4200D080180139520069
:1048300064100029F7D10133F0E704280ED90F22C4
:1048400003681A40042A09D11B099BB2002B05D02A
:104850000379DAE7012340001843F8BD0120FCE7A3
:104860001CE3000070B508680D00FFF7A9FF040005
:104870006868FFF7A5FF621E0100042A14D8451ED0
:10488000042D11D805236B439B18012215009D4070
:104890002B00064805682B430360054B1B68002B63
:1048A00002D0200002F02DFF002070BDFC0F002080
:1048B000EC1A002070B508680D00FFF781FF0400B6
:1048C0006868FFF77DFF621E0100042A13D8451EA9
:1048D000042D10D805236B439B1801229A400748EA
:1048E000036893430360064B1B68002B03D0002230
:1048F000200002F006FF002070BDC046FC0F002023
:10490000EC1A0020F0B5050089B008680C00FFF72C
:1049100057FF0690022D36DD6068FFF751FF0190CA
:10492000A068FFF74DFF04000127231D661E0793B3
:10493000731C0293079B9E4235D005237343059356
:10494000019B019D05330493049BAB421ED0042EB2
:1049500016D86B1E042B13D80122059B2349013B5B
:104960005B199A409446224A0B681068069A3A40AE
:1049700003920DD062461A430A60012200280DD12D
:104980007F000135E0E701240194CDE7029ECFE7E7
:10499000624693430B600028F2D0039A02992800E4
:1049A00002F0AFFEECE7019B1E1D042E1AD8012C6D
:1049B00018D1002505273B0021006B439B19994026
:1049C0000B000A4A013511689943094B11601B68B5
:1049D000002B05D0019B0022581D290002F091FEFA
:1049E000052DE8D1002009B0F0BDC046FC0F002025
:1049F000EC1A0020F0B53B4B85B01B680C00002B77
:104A000003D101204042FFF7A5FE012627683E4062
:104A10003CD1042F3AD90F233A681340092B35D1E2
:104A20007B685B100293029B9E4258DAB300FB182E
:104A30009868FFF7C5FEFF23050004140012184014
:104A40001C4029492B404043019305F0F7FB030428
:104A5000200025496043039305F0F0FB039C00020E
:104A6000044301982049404305F0E8FB1F4B2043D5
:104A70001B68202B06D1AD00AD0E1D4BAD00EC58D0
:104A800000022043FFF786FD0136CCE73800FFF730
:104A900097FEFF26050007140012304012494043DC
:104AA00005F0CCFB3740040438000F49784305F08B
:104AB000C5FB2E400002044330000B49704305F053
:104AC000BDFB0A4B20431B68202B06D1AB009B0E7D
:104AD000074A9B009B5800021843FFF75BFD00202C
:104AE00005B0F0BDF40F00205906000020000020A2
:104AF000F8E40000086810B5C30703D5FFF760FEAF
:104B0000054B1860054B1B68002B03D0024B18683F
:104B100002F0F8FD002010BDFC0F0020EC1A002070
:104B20007FB5A04C2368002B0AD19F4A1268002A47
:104B300006D19E4B1B68002B01D0FFF773FD7FBD94
:104B40009B4D2A68002A26D1984A1268002A1BD059
:104B5000FFF768FD0028F2D0FFF750FD924B246864
:104B60001A681C60002A16D0002C14D101AD0C224A
:104B70009049280007F08AFC285D00210134FEF7E7
:104B800045FE0C2CF8D1DAE7874A1268002AE5D1F5
:104B9000002BE3D0E0E700211A2003F0C9FE00213A
:104BA0001B2003F0C5FE00211C2003F0C1FE2E686F
:104BB000012E5CD0022E00D1A2E0002E50D1013691
:104BC0003100794C03202368994303F0B1FE04209F
:104BD000216801404B42594103F0AAFE102123688D
:104BE0000A2019404B42594103F0A2FE802123685C
:104BF000090119404B425941062003F099FE8021DA
:104C00002368090219404B425941072003F090FEE6
:104C100080212368490219404B425941092003F081
:104C200087FE80212368890219404B42594119208F
:104C300003F07EFE80212368C90219404B4259418E
:104C4000182003F075FE802321681B0319404B4296
:104C50005941172003F06CFE31001A2003F068FE62
:104C60002B680321581C05F0CFFB296067E7022160
:104C70004D4C1720236819404B42594103F058FE10
:104C800008212368182019404B42594103F050FE77
:104C900080212368C90019404B425941042003F088
:104CA00047FE80212368490119404B4259410A209F
:104CB00003F03EFE80212368C90119404B4259414F
:104CC000032003F035FE80212368890319404B42FD
:104CD0005941092003F02CFE802321681B04194050
:104CE0004B425941192003F023FE3100062003F006
:104CF0001FFE3100072003F01BFE31001B20ADE733
:104D00002021294C1720236819404B42594103F0B8
:104D10000FFE40212368182019404B42594103F0EF
:104D200007FE80212368192019404B42594103F0A6
:104D3000FFFD80212368490019404B425941092059
:104D400003F0F6FD80212368890019404B42594148
:104D5000072003F0EDFD80212368890119404B42B3
:104D60005941062003F0E4FD8021236849031940DE
:104D70004B4259410A2003F0DBFD80212368C9031F
:104D800019404B425941032003F0D2FD8023216892
:104D90005B0419404B425941042003F0C9FD012135
:104DA0001C205BE7FC0F0020F00F0020001000200B
:104DB000EC0F002010E30000012010B54042FFF787
:104DC000C9FC10BD10B5034A0921034800F090FF4B
:104DD00010BDC046F8E5000040E600008023F0B5B5
:104DE00002255B051A690A4C0A4BA1261D510327AF
:104DF0008025F600ED00BA43884202D300221A5102
:104E0000F0BD5F59002FFCD098518018F4E7C046E0
:104E10000405000000E0014010B5002806D1C020C4
:104E2000B02140028902FFF7D9FF10BDB0208021D8
:104E30008002C902F7E7000043425841064B404256
:104E40001840B0239B02C018036800201A0E532A92
:104E500001D11B02180A704700C0FEFF30B50124C3
:104E60008025054B054AED009C505C59002CFCD078
:104E700001600021995030BD00E0014004050000B0
:104E800043425841074B40421840B0239B02C01890
:104E9000A62310B50902DB05090A1943FFF7DEFF57
:104EA00010BDC04600C0FEFFF0B5012480260D4BAA
:104EB0000D4DF6005C51002902DC00225A51F0BD74
:104EC000577814783F022743947824042743D478F2
:104ED000043224063C439F59002FFCD010C00139F6
:104EE000E9E7C04600E001400405000070B5050098
:104EF0004B680A009C1C2100A400FFF7D5FF28196D
:104F000070BD0000134B1B68002B0CD08022B02317
:104F1000D2029B0200280BD11A1D5B681B0E522B7C
:104F200000D110007047B022C02392025B02F1E76B
:104F300082420DD903681B0E522B09D143680233FC
:104F40009B00C018824203D903681B0E522BE9D084
:104F50000020E7E704110020F0B50020B7B00024DE
:104F6000FFF7D0FF270005002600002D2ED1284D89
:104F70002868FFF761FF32003B000190009425494B
:104F800004A807F0E3FD04A801F042F9224B6420D5
:104F90001C682B68A0215A425341204A5B421340AF
:104FA000B02292029B18E41A6043490205F046F9C8
:104FB000A0225202030000921949220004A807F01F
:104FC000C5FD04A801F024F937B0F0BDFF226B68DD
:104FD00029689C460233FF180B12013613409C428D
:104FE00000DA1C00FF200A140240039262460140CE
:104FF00001920091039A0B4904A807F0A7FD04A8A9
:1050000001F006F92800FFF77DFF0500ADE7C04677
:10501000041100204AE700000811002000C0FEFF34
:10502000F4E6000036E7000070B50020FFF704FF4B
:1050300004000120FFF700FF844200DA04000A4B5D
:105040001D686A42554128001D60FFF7E5FEA02259
:105050006B4252021340054A28009B18044A611C07
:105060001360FFF70DFF70BD0411002004800100E4
:1050700008110020F8B50020FFF7DEFE0700012030
:10508000FFF7DAFE3E00204D0643204C0DD1802173
:10509000C020C9024002FFF7A1FE01213000FFF746
:1050A000EFFE1B4B2E6023601DE0874209DD0023CD
:1050B000B0212B60164B8902236023680020012554
:1050C00017E0012380212B60124BC9022360F4E713
:1050D000120E522A08D0002800D023600E4801F09A
:1050E00097F8FFF7A1FFF8BD28005A680232920036
:1050F0009B188B4205D21A68561CE9D10028F2D0C1
:10510000D1E72160EFE7C04604110020081100201C
:105110000480010004C002000FE7000070B5002009
:10512000FFF7F0FEFF260500002801D1280070BD22
:1051300003681C143440FFF7E5FEDA2CF4D10500B7
:10514000F2E70000FF2270B5134CD20000212000CE
:1051500007F0B8F9FF25FFF7E1FF0026002800D18E
:1051600070BD03681A142A400A2A0AD11A122A406A
:10517000FF2A03D0D200A1180B71A050FFF7C2FE86
:10518000ECE7132AFAD11B122B40FF2BF6D0DB00E1
:10519000E2181671E650F1E7A025002010B59AB08C
:1051A000FFF768FFFFF7CEFF00231A000A48D90077
:1051B000415801334C1EA1415218FF2BF7D107492A
:1051C00001A807F0C3FC01A801F022F8044801F08F
:1051D0001FF81AB010BDC046A02500207FE70000D0
:1051E00093E700008022F0B55200A1B0002168488A
:1051F00007F068F9802200215200664807F062F942
:10520000654BFF271B681A00049353425A41100054
:105210000592FFF701FE049C0020631E9C415F4B3A
:1052200064421C405E4BE418FFF778FF0600002E36
:105230002FD10498FFF700FE411C0598FFF720FED0
:10524000059A554B574D1A602C60FFF77BFFFEF710
:10525000C1FC514B64201B68A0215A4253414F4A64
:105260005B421340B0222C6892029B18E41A604300
:10527000490204F0E3FFA0225202030000924A49CF
:10528000220007A807F062FC07A800F0C1FF21B0C8
:10529000F0BD3268131412123A403B4003921A00D8
:1052A0000A3A092A49D83A4B039A995C002931D124
:1052B00010223E4807F006F935002B6803991A12B0
:1052C0003A40914209D11A143A400B2A27D0132AA6
:1052D0002DD00A2A01D1354B1D602800FFF712FEA0
:1052E000051EEAD1314B196800290FD02000FFF7C5
:1052F000FDFD04002D4B5B195968002903D02000E7
:10530000FFF7F4FD040004350C2DF3D1204B0121EF
:10531000039A99543000FFF7F5FD060087E73B40FC
:10532000022BDADC214A9B00D3185D60D5E71022FE
:1053300000211E4807F0C6F8CFE71A00153A082AE0
:10534000E8D8144A0399525C002AE3D13500152BA2
:1053500000D01500300003681A143A40152A0FD007
:105360001D2A00D10025FFF7CDFD0028F3D1002D27
:1053700004D020002900FFF7B9FD0400054BC6E763
:10538000039A1B123B409A42EDD10500EBE7C04661
:10539000041000200C1100200411002000C0FEFFAA
:1053A00004C0020008110020D9E60000282F0020C8
:1053B00010B5FFF717FF10BDF0B585B003920322BB
:1053C0000333DC17294D1440E4182B68284F5A4248
:1053D000534180225B42D202A4103B409B18A21C86
:1053E0000291244E910000910190316800980A18B2
:1053F000934215D2FFF7F6FE2B685A4253418022A2
:105400005B421F40D202BF183368009A9B189F422C
:1054100006D2194800F0FCFE0025280005B0F0BDBA
:10542000029B356819066B461A7BA423DB051343E0
:10543000FF222F00090C1943019B12041B04134087
:1054400019432800FFF70AFD0837281D210037609F
:10545000FFF704FD002C04D00A9A21003800FFF762
:1054600023FD009B083BFF183760D6E7041100209E
:1054700000C0FEFF08110020B3E600000021094B28
:10548000094A59600131516059680029FCD0002156
:105490001961012393600222044B8131FF315A507C
:1054A0001A607047FC1000400010004000E100E06E
:1054B0000222064B0121DA670022054B5A61054A98
:1054C00011615A69002AFCD07047C04604E100E02F
:1054D000FC1000400010004010B5044C2378002B55
:1054E00001D0FFF7E5FF0020207010BD0D12002055
:1054F0000120024B1B685B0018437047901200208C
:105500000120024B1B685B001843704724000020F9
:105510001FB5064B06491A6801A807F017FB0821BA
:1055200001A8FEF7EDFD05B000BDC04694120020B5
:1055300024E800001FB580235B051A6E044901A80A
:1055400007F004FB082101A8FEF7DAFD05B000BD55
:1055500024E8000010B5044C200007F03DFB0100DA
:105560002000FEF7CDFD10BD991200200E4B10B5A6
:105570001B680E4C5A1C0FD00D4C002B0CD00D4C40
:10558000012B09D00C4C022B06D0094C042B03D064
:105590000A4C052B00D1074C200007F01DFB010031
:1055A0002000FEF7ADFD10BD2800002029E8000016
:1055B00028DF000034E800002FDF00002EE80000A4
:1055C00070B504000D001600FEF70AF980230122D1
:1055D00000215B051B6E6270E270020AA271020C70
:1055E000E2711A0A60716372000EA2721A0C1B0E2D
:1055F00026702571A1702072E272237370BD0000C5
:1056000070B5214C2278002A3DD1204B01215A60EF
:105610008022D20511605A68002AFCD0002207209F
:105620001B4B1C4901255A500439585008315A5017
:1056300019481A4958501A491A485A501A495A5082
:10564000A622D2009D50082218495A5004315850C1
:10565000022017495850174917485850174804391D
:105660005850182016495850C12189005A50053900
:10567000FF395858921802435A501249124A995009
:10568000FFF7FCFE257070BD0D120020FC000040ED
:10569000001000400C050000746962751C050000D4
:1056A00024050000200004022C0500001405000061
:1056B000340500003C050000FFFF00002110010040
:1056C000540500000E1200200405000070B50E4BBA
:1056D00006001B78002B01D1FFF792FF00200B4D35
:1056E0002C7884420ED00A4B202219780323091B00
:1056F0001940084B4901C918300006F0C7FE0120C7
:10570000013C2C7070BDC0460D1200209812002084
:105710000C1200200E120020002370B588B09842B1
:1057200035DD0D6801262C0034409C422FD123002A
:10573000042D2CD90F222B681A402300092A26D1C8
:105740006A683F2A23DD6846FFF7C0FF2300002870
:105750001DD06B4619783300A14203DB6B461B5DFD
:105760005B003343A200AA1801349360202CF2D1CD
:10577000092169444A780B7812021A438B781B047A
:105780001A43CB781B061343024A13600423180004
:1057900008B070BD9412002070B5454B8AB01B78DC
:1057A000002B01D1FFF72CFF02AC2000FFF78EFF8A
:1057B000002802D100200AB070BD23780B2BF9D944
:1057C0006378012BF6D1E378012BF3D1002311206C
:1057D000384E394D33602B7068442379374A41780D
:1057E0001360027809021143827812041143C278CF
:1057F00012060A4332490A60002B0ED11521694472
:105800004A780B7812021A438B781B041A43CB7820
:105810001B0613433360002318E0012B1AD1152116
:1058200069444A780B7812021A438B781B041A4396
:10583000CB781A211B06134333600E23627C694424
:10584000934200DD130000229A422CD10022042052
:10585000EA54B0E7022B03D1627B10331621EEE746
:10586000042B0DD1152108226944684606F00EFE6E
:105870000098019903F098F806F0BAFC3060CAE786
:10588000052BC8D1152108226944684606F0FEFDA3
:105890000098019903F088F806F0AAFC3060627D58
:1058A0000A231E21CBE7885CA8540132CCE7C0460E
:1058B0000D120020901200209912002028000020D4
:1058C0009412002010B5134B04001B78002B01D15B
:1058D000FFF796FEFFF7ECFD00200F4A0F49104B33
:1058E000545058600130106058680028FCD00020E7
:1058F00018610130906018690028FCD0094B0A48F3
:105900001B785B011B185350FFF7D2FDFFF7B6FD64
:1059100010BDC0460D12002000100040040500001C
:10592000FC1000400C1200200E12002010B588B0B0
:1059300000281DDD0A68012113000B4018D1042A3C
:1059400016D90F2014682040092811D150683F282B
:105950000EDD9800101880680024084201D0401025
:10596000C4B26846C4540133202BF2D1FFF7AAFF1A
:10597000002008B010BD000010B5002813DD0C6831
:10598000E30710D56410532C0DD8084B1B78002B5F
:1059900001D1FFF735FEFFF78BFDA123044ADB00A1
:1059A000D450FFF76BFD002010BDC0460D12002043
:1059B0000010004010B500280EDD0C68E3070BD581
:1059C0006410FF2C08D8054B1B78002B01D1FFF782
:1059D00017FE034A034BD450002010BD0D120020C7
:1059E000001000402405000013B5002814DD0C68E9
:1059F000E30711D5094B64100093094B0193072C61
:105A00000AD8084B1B78002B01D1FFF7F9FD6B4634
:105A1000054A1957054BD150002016BDE2ECF0F4B1
:105A2000F8FC00040D120020001000400C050000DE
:105A300070B588B0002820DD0124086804401CD11E
:105A400004281AD90F2302681340042B15D1FEF73E
:105A500037F9060007F0C0F80500122800D9122512
:105A60002A0002210D326846FFF7AAFD6B465D73DE
:105A7000A54205DC6846FFF725FF002008B070BD91
:105A80002300325D6B449A730134F1E7F0B50D00E9
:105A90008BB0012832DD08680122040014402DD1AA
:105AA00004282BD90F2301680B40042B26D16B68E7
:105AB000134223D0FEF704F96E68070073100193B8
:105AC00007F08AF805000E2800D90E252A000121CA
:105AD000113202A8FFF774FD6A46127902AB5A73BD
:105AE00002AA73129373019B76141B0ED673137460
:105AF0005574A54205DC02A8FFF7E4FE00200BB0B8
:105B0000F0BD3A5D02A963189A740134F1E730B52B
:105B100089B0002814DD0C68E30711D5102268460F
:105B20000021FFF74DFD6B466A4665105D736846C0
:105B300063122D0E64149373D4731574FFF7C2FEB1
:105B4000002009B030BD0000174B184A59680029E1
:105B500003D00021596001319160196900291FD0DB
:105B6000002018618023DB00D3581149012B18D184
:105B7000A923DB00D3585B420B600E490B78032B43
:105B800001D801330B7003200B490B78013303401C
:105B90000B700A495B015B1809495350012393605C
:105BA00070470860FAE7C046FC1000400010004053
:105BB00024000020981200200C1200200E12002059
:105BC0000405000010B5034A1021034800F090F8C6
:105BD00010BDC046A4E700009BE70000044A054949
:105BE0001368C85401339B059B0D13607047C04672
:105BF000C8160020C812002070B5114C114A236845
:105C0000834202DC0023236016E0155C411C2E0059
:105C1000FA3E012E05D899420FDA555C013D1F2D41
:105C200001D90800ECE70100151A565C6E540131E9
:105C30008B42FADC181A206070BD1570FAE7C04676
:105C4000D41A0020D416002010B5FDF7BFFD064B76
:105C50001A68824201D900221A601B68C31A0348DD
:105C600098428041404210BDC4120020204E0000E6
:105C700010B5094C094A23681268934200D110BD3F
:105C8000074AD05CFDF79EFF0028F8D02368013357
:105C90009B059B0D2360ECE7CC160020C816002066
:105CA000C812002010B50400064B074A1B68126892
:105CB0009B1ADB439B059B0DA34200DB10BDFFF746
:105CC000D7FFF1E7C8160020CC16002070B5FFF70B
:105CD00025FAFF250400002801D1200070BD0368CB
:105CE0001B142B401D2B00D10400FFF70BF9F2E72A
:105CF00070B5074E33680B2B08DC0C255D43054C53
:105D00000133285164196160A260336070BDC046E0
:105D1000D0160020382F0020F0B5B7B0040006F0F0
:105D20005BFF012802D8002037B0F0BD23785B2B41
:105D3000F9D1013825182B785D2BF4D101343A21A3
:105D4000200006F031FF061EEDD0071B002FEADD14
:105D5000210000243A0004A806F056FF04AB711C91
:105D6000DC556F1AA742DEDD1DAD3A00280006F0B3
:105D70004BFF134BEC551B6803950193019BA3420A
:105D8000D1DD0C2666430F4B04A9F618306806F0E7
:105D900019FF051E05D17368B6680293029B9D42E8
:105DA00001DB0134EAE73068039906F00BFF3700A6
:105DB0000836002801D17868B6E70135EEE7C0461D
:105DC000D0160020382F002010B5FBF7D5FAFEF7CB
:105DD000F9FFFBF7FBFAFDF789FEFEF741FBFEF743
:105DE000C1FBFFF7EFFE01F039F801F05FFC01F0B5
:105DF0008BFC01F0D5FE10BD962210B512010021DA
:105E0000034806F05FFB0022024B1A6010BDC0463B
:105E1000401C0020D805002070B514007F22174BCD
:105E2000C000C0580D00836813401C2B01D0002017
:105E300070BDC368190011400429F8D101690A40F6
:105E4000192AF4D11B0A01339B000C30C018FDF74E
:105E500037FF037806000120002BE9D0300006F060
:105E6000BBFE0023A042E2D1A34201DB0120DFE719
:105E7000F15CEA5C9142DAD10133F5E7A02500201C
:105E8000064B074A1B6812689B1ADB439B059B0D58
:105E90000122834200DC002210007047C816002057
:105EA000CC160020F8B505000C0016001F1E0ED100
:105EB0000320FFF7E5FF002808D0FA20FFF78EFE49
:105EC000E8B2FFF78BFEE0B2FFF788FEF8BD501D89
:105ED000FFF7D6FF0028F9D0FB20FFF77FFEE8B2DE
:105EE000FFF77CFEE0B2FFF779FEF0B2FFF776FE37
:105EF0003012C0B2FFF772FE3C00E31B9E42E5DDAC
:105F00002078FFF76BFE0134F7E7000070B500243E
:105F1000F0250B4B1B68A34202DCFFF76DFF70BD41
:105F20002B006343074A9B181A78002A05D059783A
:105F3000002311201A00FFF7B5FF0134E9E7C0463E
:105F4000D8050020401C0020F8B507000024F025EB
:105F50002B0063430C4A01349E18B74211D03178AC
:105F600000290BD00133D15C002311201A00FFF768
:105F700099FF2A000021300006F0A4FA0A2CE7D18C
:105F8000F8BD024B1C60F9E7401C0020D80500203A
:105F9000F0B5150001222F007A4C1740A54401905E
:105FA0000291002F11D005AB1A706A105A70120EB0
:105FB0001A710522691299706D140299DD70FFF74C
:105FC00071FFCF239B009D44F0BD042D2AD90F24DF
:105FD00028680440042C32D1022304AA280013713B
:105FE000FDF76EFE050006F0F7FDC82302009B00DA
:105FF000984200DD1A007C1C97420DD1984206D9C8
:10600000614804AB03226149C01806F03FFA220040
:1060100005AB02990198D2E72700611E695C05ACC7
:10602000E155E8E7042D00D0A7E0032304AA043DCE
:1060300013716B425D4105AB55710222E9E7092CF2
:106040007ED1042205AB1A706A685110009169462E
:10605000521209789A70009A59701F2A01DD202285
:1060600000926A46127806ACDA70009BBB4202DCF2
:1060700005ABE21ACDE70126BB00EB189868064095
:1060800006D1042837D90F210368194002290CD101
:10609000012323704310637042121B0E4014A27040
:1060A000E070237105340137DFE7042921D1022391
:1060B0002370FDF705FE039006F08EFDA31C0C284F
:1060C00009D86070864201D19C19ECE7039A925D71
:1060D0009A550136F6E70C226270039A925D9A5542
:1060E0000136092EF9D12E23E372237363730E3424
:1060F000D9E7012907D103230438237043425841CB
:1061000060700234CFE7092909D104232370436862
:106110005A1062705B12A370E6700434C3E703295F
:106120000BD1052323700068020992B2430F92003D
:106130000B40D31A63701B12EDE726700134B2E7EF
:10614000032C00D03DE7052205AB01091A7089B286
:10615000420F890022408A1A11125A709970642ADB
:1061600000DD64220421DA70081F824201DC04325F
:106170004FE7685C58540131F6E7002D00D020E766
:1061800053E7C046C4FCFFFF2203000082DB00008F
:1061900070B502000024F0210D4E08006043801904
:1061A0004578954203D001340A2CF6D170BDF02217
:1061B000002106F087F9074A1368013BA34200D18A
:1061C0001460002329001A001120FFF76BFEEDE791
:1061D000401C0020D805002010B5B2B002236A464A
:1061E0000400137006F0F8FCC72800D9C72000236C
:1061F000984207DC421C6B46FE211420FFF752FE3A
:1062000032B010BD694601335A1EA25CCA54EFE792
:1062100030B5B3B002236A460500137006F0DCFC0B
:106220000400C72800D9C72400239C420BDC2000AF
:106230003230FFF737FD621C6B46FF211420FFF759
:1062400031FE33B030BD694601335A1EAA5CCA54D0
:10625000EBE70000F0B5BDB005900C00012803DCB1
:106260001B20FBF751FA55E02C4B08680393C3073A
:1062700009D4042807D90F2302681340042B02D144
:10628000FDF71EFD0390254B60680493C30709D4F6
:10629000042807D90F2302681340042B02D1FDF70D
:1062A0000FFD049000261E4B1B680893089BB34209
:1062B0000BDC049B1B4A0093C821039B0AA806F031
:1062C00013FC0AA8FFF7A4FFCAE70C257543164B79
:1062D0000399ED18286806F075FC071E05D16B6858
:1062E000AD680993099B9F4201DB0136DEE7286810
:1062F0000499079506F066FC0835069000280BD136
:1063000021000598079B08315B6802389847074BC6
:10631000069A1A603DB0F0BD0137E3E7A2E0000045
:10632000D016002005E90000382F0020E40F0020DF
:10633000F7B5234B06001B68F02100930023009A59
:106340009A4211DC0024F0231A0062430192019961
:106350001C4A55182F78002F12D001340A2CF3D183
:106360001948FFF755FF29E00A005A4315488218DB
:106370005078B04202D11278002A1FD10133DEE7F3
:10638000F0223900280006F09DF802230D4A0199F9
:10639000EB6053540D4AF1008A58009B6E70AE704A
:1063A000AA602F616F61A34202DC054B01341C60BF
:1063B000002331001A001020FFF774FDF7BDC0461E
:1063C000D8050020401C00204DED0000A025002035
:1063D00010B5FFF79BFDFF24084AE3005B429B18C2
:1063E000074AD35C043B012B03D8E043C0B2FFF75C
:1063F0009FFF013C002CEFD110BDC046FC07000000
:10640000A0250020F8B505000E00FDF779FEFF2459
:106410000D4B18600D4AE3005B429B180C4AD35C9D
:10642000062B01D0032B0BD1E743FFB2320029002A
:106430003800FFF7F1FC002802D03800FFF778FFA2
:10644000013C002CE6D1F8BD08000020FC0700004C
:10645000A025002070B50500FF24084AE3005B4238
:106460009B18074AD35CAB4203D1E043C0B2FFF7AD
:106470005FFF013C002CF0D170BDC046FC0700005E
:10648000A0250020F7B5FDF7A1F9574B1A68824205
:1064900001D900221A601A685449821A8A420DD919
:1064A000FF2253491860D3005248CB1A1B181B789F
:1064B000073B022B0CD9013A002AF4D1F7BD072083
:1064C000FFF7C8FF4C4B27E00820FFF7C3FF38E079
:1064D000FDF786F9071E00D101270020FDF734FAE9
:1064E00001900020FDF744FA019B0090434C444D7D
:1064F000002B12D02368002B6ED12B682760002B55
:106500006ED0404B01261B78002BD8D10920FFF715
:10651000A1FF394B1E703B4B1E70009B002B12D00D
:106520002B68002B0FD123682F60002B1ED0324B1D
:1065300001261B78002BC7D10920FFF78BFF2E4BBC
:106540001E70304B1E702368002B0FD02A4E3278FD
:10655000002A0BD19F4200D227602368FB1A312BFF
:1065600004D90720FFF776FF012333702B68002B37
:106570000FD0244E3278002A0BD1BB4200D92F60B5
:106580002B68FF1A312F04D90820FFF763FF01237E
:1065900033702368002B0CD0019B002B09D1164EC1
:1065A0003378002B02D10720FFF754FF002323602C
:1065B00033702B68002B00D180E7009B002B00D0AC
:1065C0007CE7104C2378002B02D10820FFF742FF14
:1065D00000232B60237071E7009A002AA0D1B5E751
:1065E000009B002B9FD1AEE7C01200200F270000B8
:1065F000A0250020FC070000B4120020B0120020EB
:10660000B8120020BC12002013B50400FFF77EFC76
:10661000002301930F4B1B68002B02D101A8FDF74B
:106620007BF900210800FEF785F8FEF779FAFDF7FF
:10663000B3F9FDF737FAFDF751FAFEF7BDFBFDF7A9
:10664000F3F8002C04D0FDF7E7FA0348FFF7E0FD6C
:1066500013BDC046EC1A00203EED0000002310B52B
:1066600001001A001120FFF71DFC10BD07B56B4695
:10667000197069465A7013128B701314120ECB7076
:106680000A716B46010005221320FFF70BFC07BDC2
:1066900010B50A0001001220FFF77AFC10BD70B59A
:1066A00005000C00FDF7AAF8002809D020003230C0
:1066B000FFF7F8FA2B00220000211B20FFF7F2FB66
:1066C00070BD10B50C000300110014202200FFF76C
:1066D000E9FB10BD012370B5FF24084A41185B4255
:1066E000884201D3D84370BD06781D0A2340734009
:1066F0009B009B5801306B40F2E7C04620E9000048
:1067000013B50400FE2813D80A4BC200D058002845
:106710000ED0436808309900FFF7DCFF0190092094
:10672000FFF7C0FA01AB042221001720FFF7BAFBE4
:1067300013BDC046A0250020F7B50190FFF7C6FAAB
:1067400001250400FF276D42002C01D12800FEBD69
:10675000266833143B40152B0DD1210001980831D8
:1067600006F030FA002801D135123D402000FEF736
:10677000C9FB0400E8E71D2BF8D101256D42F5E7C0
:10678000F0B58027A1B0FFF773FAB84CB84D206878
:10679000FF00391A4019FDF7FBF923680600C318FA
:1067A0002360002B0ED121B0F0BD2068391A2818C3
:1067B000FDF7EEF9236806001B182360FDF706F8C5
:1067C000AC4B1860002EF0DC2B78FA2B00D014E1D3
:1067D0002368022B07DCFFF737FA0028E3D00120FB
:1067E000FFF70AFADFE76B78AC78981E182800D913
:1067F000F8E003F08FFC0D2024282B34F73E707A4C
:106800007E94D3E4F7F7F7F7F7F7F7F7F7F7F20027
:10681000FF2C0ED02000FFF7BBFC0022964BE100BE
:10682000CA505B181A712100009213001320FEF762
:10683000C3FD0320D4E72000FFF77AFDF9E720002D
:10684000FFF7A6FCF5E7FFF7C3FDF2E7FFF75EFBF6
:106850000020FFF7D9FE8948FFF7DAFCE9E7632C4F
:10686000E7D8874BA200D25821001520FFF790FBF4
:10687000DFE7FFF72BFAFF270400002CD9D02568AB
:106880002B143B40152B04D02000FEF73BFB0400EB
:10689000F3E72000083006F09FF906000530FFF707
:1068A00001FAFB20FFF79AF92D121D20FFF796F948
:1068B000E8B2FFF793F9F0B2FFF790F93012C0B2E7
:1068C000FFF78CF925002B1B9E42DDDD287AFFF7B0
:1068D00085F90135F7E700211D2000910B000A0022
:1068E000FEF76AFDFDF798F9A3E72000FFF708FF20
:1068F0009FE7FCF785FF07AC624A64210090624B7A
:10690000200006F0F1F802232000237006F064F95D
:106910002300020000211620FFF7C4FA89E75B4B31
:10692000FA21186803F08AFC00260490524AF3000A
:106930009B181C68002C28D01B79059363680834C9
:106940009F00B81D0393FFF7ADF9FB20FFF746F951
:1069500001207D1CFFF742F9F0B2FFF73FF9E8B2E2
:106960002D12FFF73BF9E8B2FFF738F90598FFF76A
:1069700035F9E719A7420CD8FFF77AF9049B039879
:10698000584301F0B5FDFFF773F90136FF2ECDD165
:106990004FE72078FFF722F90134EBE70024FFF7F7
:1069A000B5FA2200210000942300DA20FEF704FD4E
:1069B000FF222100D200304805F084FD92E7012C2F
:1069C00002D1FEF7C9FA34E7022C02D1FEF7F0FC3F
:1069D0002FE70120FFF718FE2BE7002321001A0004
:1069E0001A2099E71A00C83A052A00D921E700229F
:1069F00018001100FAF7F6FC1BE7FB2B00D0EEE6BF
:106A00002268042A00DCE6E62E79E878204B36027C
:106A100006439E4200DDE2E6331D9A4200DCDAE6E0
:106A2000EB5CFE2B00D0DAE66878AC78771E1B288A
:106A300000D17FE030D8072865D008283AD0012857
:106A40002FD1FF2C10D02000FFF7A2FB6D79114A47
:106A5000B31E009221002A000A20FEF7ADFC064B6F
:106A6000E400E0501B191D71701DB9E6D41A002016
:106A7000D4160020C4120020A025002020ED000024
:106A8000982D002037ED000032ED000004000020BA
:106A9000F6030000DA1600201D285DD04FD31E2813
:106AA00071D00300C83B052BDED8404A3900FAF705
:106AB00099FCD9E7632CD7D86A79022A13D0032A24
:106AC0001BD0012AD0D1E979AB79090219432B7A7D
:106AD000A4001B0419436B7A1B060B435B00134392
:106AE000334AA350C0E7002FBEDDB11E3148FDF789
:106AF00007FB2F4BA400E050B6E7AB79A4005A1E69
:106B000093419B00ECE7632FAEDC07AD3A002749C9
:106B1000280005F0BBFC00232800EB55FFF70CFE16
:106B20000028A1DB224B8000C25821001520FFF76E
:106B30002FFA99E739001D48FFF764FC94E7FF2C12
:106B400092D06A79022A8FD81A490B20009121002D
:106B5000B31EFEF731FC87E7632F00DD63270023B8
:106B600007A99F420ADCFB430022DB173B40CB18FE
:106B70001A70152000917B1C2100EAE7EA1852796F
:106B8000CA540133EDE7012C00D06DE7002F00DC83
:106B90006AE76B79002B03D01C00322B00DD322416
:106BA00064235C43044B1C605EE7C046D91600209A
:106BB000982D0020DA160020040000200122094B45
:106BC0001A60094A1368002BFCD00322074B1B688C
:106BD000D8171040C0180123801006384000184311
:106BE0007047C04600C0004000C1004008C50040DA
:106BF0000120704710B5064C200001F0E5F805496A
:106C0000200001F015F90122034B1A6010BDC046A7
:106C1000101B0020801A0600D81A00201FB5002182
:106C20000E20FCF7F3FD01210F20FCF7EFFD012101
:106C30000D20FCF7EBFD1C4C200001F023F81B4B52
:106C40001B4A1B6812681B49D2B28B420BD88023A7
:106C50009B04019301AB1A710199029A0023200051
:106C600001F02CF81FBD14498B4202D88023DB04AD
:106C7000EFE712498B4202D880231B05E9E7104950
:106C80008B4202D880235B05E3E70E498B4202D892
:106C900080239B05DDE70C498B4202D88023DB056E
:106CA000D7E780231B06D4E7F01A0020300000202D
:106CB0002C00002048E8010090D0030020A107002C
:106CC00040420F0080841E0000093D0010B50028DE
:106CD00015DD01240B68234211D023410C4A1360B7
:106CE0000C4AA04209D04B68234206D02341022B14
:106CF00009D0032B09D0A34203D002231360002044
:106D000010BD0023FAE70323F8E71460F7E7C04655
:106D1000300000202C000020F8B50125086828422A
:106D200003D10D20FAF7F0FCF8BD4010FCF792FDFE
:106D3000041E2DDBFCF768FDA04229DB00212000AA
:106D4000FCF764FDFA222900D200200001F002FCC9
:106D500000281DD0002500270726FA2201219200D5
:106D6000200001F0F7FB002812D0282802DD0123C3
:106D7000B3401F43013EF0D20D4EAF550135052DF6
:106D8000E9D1012206210920FDF73CF9002801D1B3
:106D90000020C9E70B23012443600023F25C990023
:106DA00052004118224301338A60052BF6D1BBE71C
:106DB000DC1A002070B500281EDD0D68EB071BD41F
:106DC000042D19D90F242B681C40032C14D11A0947
:106DD00092B25B0F92001C40141B2E00FFF71EFFA7
:106DE000731B06489C4205DD317900F06DFF0136CA
:106DF000F070F5E700F067FF002070BDF01A00208A
:106E00000120704710B504680D20E30703D5641016
:106E1000FF2C03D91720FAF777FC10BDFFF7FEFE11
:106E2000E1B2044C200000F04FFF200000F04BFFC7
:106E30000020F2E7F01A002070B5FFF7EFFE064DD4
:106E40000021280000F040FF0400280000F03BFF74
:106E500001206400204370BDF01A002010B5034AE1
:106E60000E210348FEF744FF10BDC04664ED00004C
:106E7000D4ED00000D4B70B51B6804000E0015002A
:106E8000002B01D1FFF7B6FEE1B2094C200001F062
:106E900066F8F1B2200000F063FFE9B2200000F0D4
:106EA0005FFF200001F0C6F870BDC046D81A002070
:106EB000101B002010B501240368234205D041684F
:106EC000214202D08268224203D10D20FAF71CFC35
:106ED00010BD5810802801D91520F7E74910FF2967
:106EE00001D91620F2E75210FF2A01D91720EDE749
:106EF000FFF7C0FF0020EBE7F7B501221400904236
:106F000026DD0D682A4223D02D4B15411B684C68A5
:106F1000002B01D1FFF76EFE2A4EE9B2300001F0DE
:106F20001EF827000122174014D01441FF2C02D96B
:106F30001720FAF7E9FBE1B2300000F011FF300052
:106F400001F078F80024A04202D02320FAF7DCFBFD
:106F50002000FEBD042CF2D90F2523681D40092D09
:106F60001CD1636801925B100093009BBB42E6DD7D
:106F7000BB00E3189D68019B1D420BD06D10FF2DD7
:106F800002D91720FAF7C0FBE9B2300000F0E8FEA2
:106F90000137EAE71720FAF7B7FBF9E7032DCED15F
:106FA00027001A0992B25B0F92001D40551B3B1B34
:106FB0009D42C4DD3979300000F0D2FE0137F6E79A
:106FC000D81A0020101B0020154B70B51B68050057
:106FD0000E00002B01D1FFF70DFE124CEDB229007F
:106FE000200000F0BCFFF1B2200000F0B9FE00214B
:106FF000200000F0BFFF002801D0404270BD72B6F3
:1070000001222900200000F0A5FF62B6200000F058
:1070100098FE0028F2D0200000F098FEEEE7C0466F
:10702000D81A0020101B002010B501240368234249
:1070300002D04168214203D10D20FAF765FB10BD53
:107040005810802801D91520F7E74910FF2901D9E8
:107050001620F2E7FFF7B8FF40002043EFE70000FB
:1070600070B50D211D20FFF7AFFF184C5A280CD129
:1070700001222A2122703D38FFF7FCFE022001F098
:1070800037FA0122124B1A6070BD0F211920FFF749
:107090009BFF332805D102238F22237020211A3829
:1070A000EAE70D211E20FFF78FFFC7280AD103252D
:1070B00000222A21A9382570FFF7DCFE2A002A21A8
:1070C0001E20D9E700232370D8E7C04634000020F3
:1070D000E41A002010B5002803DC1C20FAF714FB8A
:1070E00010BD01240B681C4001D10D20F6E75B1098
:1070F000012B2BDD022B03D00224042B00DD0134F5
:10710000194B1B68002B01D1FFF7AAFF174B1B7807
:107110005BB2022B1CD0032B1ED0012B11D1032CF0
:1071200000D1013C00222A211D20FFF7A3FE2200EE
:107130000E211D20FFF79EFE01222A211D20FFF7B0
:1071400099FE022001F0D4F90020C9E70024D7E716
:10715000220123211920F2E7032C00D1013C220057
:107160000E211E20EBE7C046E41A00203400002068
:10717000204B10B51B680400002B01D1FFF770FFF6
:107180001D4B1B785BB2022B0AD0032B29D0012B9D
:107190002CD121001D200124FFF716FF644205E0D9
:1071A000012C13D129211920FFF70EFF7F2801DDC3
:1071B0000138FF3803007F3301DA7F204042C823C3
:1071C0007F21584303F03AF8604310BD032C0BD1E4
:1071D0002B211920FFF7F8FE043CE7E72D211920A9
:1071E000D9E721001E20D6E7052CF7D00124002086
:1071F0006442E4E7E41A00203400002010B50120C6
:10720000FFF7B6FF43000120184310BD10B503205F
:10721000FFF7AEFF43000120184310BD10B5052055
:10722000FFF7A6FF43000120184310BD144B70B5B3
:107230001B68002B02D10120FFF79AFF114B1B782E
:107240005BB2013301D1FFF70BFF0120FFF790FF85
:1072500004000320FFF78CFF05000520FFF788FFDF
:107260006D43644340436419201804F0F7FF01F0B4
:10727000CBFC04F0BDFF43000120184370BDC046A5
:10728000E41A002034000020F8B5514B05001B68BB
:10729000002B01D1FFF7AEFC4E4C23787F2B00D89A
:1072A00092E007210E20FFF78FFEC42833D1012280
:1072B0000E26494B10211A70484B30001A70267068
:1072C000FFF7D8FD802211213000FFF7D3FD002108
:1072D000615600291EDB424EC9B2300000F03FFE6D
:1072E0003D4B3000197800F03BFD300000F0A2FE6D
:1072F00021780622300000F02DFEAC1D300000F099
:1073000020FD002806D0300000F020FD2870013557
:10731000A542F3D1F8BD0F211920FFF755FE332800
:107320000FD168222C4B1E261A7000222B4B602195
:107330001A7030000C322670FFF79CFD022261218A
:10734000C2E700211820FFF73FFEFA281CD1422295
:10735000214B10261A700022204B4B211A7030004E
:1073600001322670FFF786FD042001F0C1F83822B3
:107370004C213000FFF77EFD0F2251213000FFF736
:1073800079FD1B2252219FE70F211C20FFF71CFED5
:107390003D289CD128221C2600270F4B20211A7043
:1073A0000E4B263A30001F702670FFF763FD3A003F
:1073B00022213000FFF75EFD3A0023213000FFF765
:1073C00059FD402224217FE70021615683E7C04612
:1073D000D81A002035000020370000203600002099
:1073E000101B002073B5002606220021684605F018
:1073F00069F86846FFF748FFFFF7C2F91A4B6A467B
:107400009E576C466B4691781878D5785B781279E0
:107410006479002E1FD000020902034329431BB2E6
:1074200009B2120211482243007812B240B2102869
:1074300002D15210DB10C910D8171B184340C817CF
:107440000918414001205918D317D2185A408A18F8
:107450005200104376BD1B022D02034329431BB289
:1074600009B22402DEE7C0463600002035000020C5
:10747000F8B501231C0098422BDD0F683B4228D051
:107480004E6835001D4024D1042E22D90F223168C8
:107490000A40092A1DD173685C10202C00DD2024CD
:1074A000144B1B68002B01D1FFF7A4FB72B67F10B1
:1074B000F9B2114F2200380000F04CFD62B6A5422F
:1074C00014DA380000F03DFC002804D101246D00DE
:1074D0002C432000F8BD380000F038FC0122AB003E
:1074E0004000F31810439860AD18E8E764000125E8
:1074F000EEE7C046D81A0020101B002010B5054C3E
:107500002368002B02D01B20FAF7FEF80020206031
:1075100010BDC046E81A002010B5002803DC1C206E
:10752000FAF7F2F810BD0B68DA0706D4042B04D979
:107530000F221B681340032B01D02420F0E7034BDC
:1075400025201B68002BEBD01B20E9E7E81A002060
:1075500010B5002803DC1C20FAF7D6F810BD0B6824
:10756000DB0701D40D20F7E71B20FAF7CDF8002048
:10757000F4E700001D4B70B51B680C00002B03D115
:107580002520FAF7C1F870BD012801DC1C20F8E7BE
:1075900008680121084207D1042805D90F23026891
:1075A0001340DD1E8D4201D92420EAE765680D42B3
:1075B00001D11120E5E7042B0BD1FCF781FB05F08D
:1075C0000BFB63685B10013B01D4834208DB122094
:1075D000D7E7100980B252008000920F801AF0E7BE
:1075E0001B20FAF791F80120CDE7C046E81A0020E9
:1075F00010B50400802803DD2620FAF785F810BDB9
:10760000002CFCDD1B20FAF77FF8FEF73BFFFFF7AD
:10761000B7F8012000F06CFFF2E7000010B5002879
:1076200005DC1C20FAF770F80400200010BD184B90
:107630001B68002B01D12520F4E7012408680440D1
:107640000FD04010FF2801D92820EBE71B20FAF7C4
:107650005BF8FEF717FFFFF793F8012000F048FFF3
:10766000F4E70428E1D90F2102681140042906D16A
:10767000FCF726FB05F0B0FAFFF7BAFFD5E70329C0
:10768000D3D1100980B2520F80000A40801AF3E76C
:10769000E81A0020044B10B51B682520002B00D0F1
:1076A0001B20FAF731F810BDE81A002010B5034A84
:1076B00006210348FEF71CFB10BDC04670EE00001B
:1076C000A0EE0000002070470120704700207047A6
:1076D000002070470020704701207047002070474D
:1076E000002070470020704700207047002070473E
:1076F000002070470020704700207047002070472E
:10770000704770477047000010B5034A0F210348C7
:10771000FEF7EEFA10BDC046C0EE000038EF0000E4
:107720000378013B1F2B00D970470130F8E710B5F3
:10773000FFF7F6FF0378002B0BD00130222B11D17D
:107740000378002B03D0421C222B03D11000FFF73B
:10775000E7FF10BD5C2B03D14378002B00D0821CC7
:107760001000EDE73A2BF2D02C2BF0D07B2B0BD175
:10777000FFF7D6FF0378002BE9D07D2B01D1013034
:10778000E5E7FFF7D4FFF5E720225B2B14D1FFF7E5
:10779000C7FF0378002BDAD05D2BF0D0FFF7C7FFCF
:1077A000F7E7202BD3DD2C2BD3D0190091435D2993
:1077B000CFD0222BCDD001300378002BF1D1C6E7FA
:1077C000002210B5904216D0FFF7AAFF03780422DA
:1077D000222B10D0023A7B2B0DD0013A5B2B0AD022
:1077E000190030390232092905D92D2B05D14178EC
:1077F000303909290AD8100010BD0522742BFAD09F
:107800000132662BF7D001326E2BF4D0581E834123
:107810005A42F0E770B5FFF783FF037801222D2B62
:1078200001D18018023A00230A2502E06B4301309F
:10783000CB1801783039CCB2092CF7D95A43100053
:1078400070BDF8B50C001500FFF76AFF0378222B16
:1078500002D000232370F8BD0D236A1E21000825E5
:107860000C260A279C4601300378222B02D10023E4
:107870000B70F0E7002BFAD0441C5C2B0BD1437843
:10788000841C622B0ED0662B0ED06E2B0ED0722B6A
:107890000ED0742B0ED0002AE9DD0B70013A0131B5
:1078A0002000E1E72B00F6E73300F4E73B00F2E7C6
:1078B0006346F0E70923EEE710B50400FFF737FF52
:1078C000A04203D90378013B1F2B00D910BD01381A
:1078D000F6E710B5002815D00378002B13D0FFF77A
:1078E0001FFF2021037802008B4300205D2B09D06D
:1078F0001000FFF71CFF03782C3B5A425341C0187D
:10790000FFF70EFF10BD1800FCE70300002070B564
:107910000C0081420EDD1A785B2A0BD1581CFFF750
:10792000FFFE0125AC4205D0FFF7D3FF002801D0B0
:107930000135F7E770BD70B50C001500002901D0C6
:1079400000230B70002820D00378002B1ED0FFF7F7
:10795000E7FE037806002C2B03D10130FFF7E0FE91
:107960000600337800207D2B0FD0844204D02A00FB
:1079700021003000FFF765FF3000FFF7D8FE0378E5
:107980003A2B02D10130FFF7CBFE70BD1800FCE7A7
:10799000F0B50D0004009DB02E78002E35D02E21BC
:1079A000280005F001F9071E14D0431B0193303E57
:1079B000092E14D82800FFF72DFF01002000FFF743
:1079C000A4FF0400002C20D0002F1ED0019B013307
:1079D000ED18E1E7280005F0FFF80190E7E72378CC
:1079E0007B2B11D1601C642203A9FFF7A4FF041EA6
:1079F0000BD0019A290003A805F0F5F80028E1D082
:107A00002000FFF794FEEEE7002420001DB0F0BD3B
:107A100070B5050000200C0081421DDD2800FFF735
:107A2000CFFE0300681C012B14D00020022B13D1C1
:107A30000022681C1100FFF77EFF012C0CD0FFF71D
:107A400048FF00221100FFF776FF013CF5E7FFF742
:107A500040FF013C012CFAD170BDF8B505000020B3
:107A60000C0016001F0081420DDD2800FFF7A8FE64
:107A700003000020022B06D1681C3A003100FFF7FA
:107A80005AFF012C00D1F8BDFFF723FF3A00310067
:107A9000FFF751FF013CF4E710B50024A04218D0D5
:107AA000FFF73EFE03787B2B0AD101300022110044
:107AB000FFF741FF00280CD0FFF739FE0134F5E74E
:107AC0005B2B06D10130FFF704FF002801D0013401
:107AD000F9E7200010BDF8B5002816DD0D68EB07AA
:107AE00013D56D10013D0124FDF718FB0026FF277B
:107AF000644200280CD1002E21D0300005F06CF833
:107B000001003000FCF7FCFAF8BD01256D42EAE700
:107B100003681A143A40152A0BD11B123B409C42B1
:107B200000DA1C009D4201D106000836FDF7EAF993
:107B3000DFE71D2AFAD1012400266442F6E701207E
:107B4000013464002043DFE710B508680C00FCF73F
:107B5000B7F8FEF7F1FD002803DB6268024B8000F6
:107B6000C250002010BDC046982D002010B50868F6
:107B7000FCF7A6F8FEF7E0FD0123002802DB024B2C
:107B80008000C358180010BD982D002010B508685B
:107B9000FCF796F8FEF7D0FDC043C00F800010BD83
:107BA00010B5034A04210348FEF7A2F810BDC046F1
:107BB000D4EF0000CEEF000010B5FBF7A3FFFCF7F9
:107BC00051F8FEF701F90448FEF722FBFDF7E6FA4B
:107BD000FEF7FEFB10BDC04623F0000010B5FBF71A
:107BE0000DFC10BD70B5002504AC24780573A942C6
:107BF00005D10A4B0A4A25210A4804F0D9FB016045
:107C00000949920052589B0002715B58A40083718D
:107C10006358856043710223C37170BD3BF000005F
:107C20009AF0000049F00000F8F00000037B002B00
:107C300004D14373837303610133037370470000FE
:107C40001FB50191A02100240068C900D2B24450A0
:107C5000012A10D0A24209D0032A0AD0074A835031
:107C6000074B019AC250012343501FBD0222134308
:107C7000F4E70422FBE70622F9E7C04654050000BA
:107C80002405000010B50400FFF7D0FFA1222368EF
:107C9000A179D20099506179064A20009950217942
:107CA00004329950044B19685A689B68FFF7C8FF63
:107CB00010BDC0460C050000041B00201FB5FFF7D7
:107CC000BFFF05B000BD70470368074A99501A000E
:107CD000FC32D1680029FCD0A321C90058580023E8
:107CE000C0B2D3607047C0461C05000007B58022B3
:107CF000074BD2051A6000229A6002321A710F23D4
:107D00000C3200930349023B0348FFF76BFF07BDAA
:107D1000041B002000300040F01A0020F8B50500D8
:107D20000E0017000024BC4208D02B68315D1B6890
:107D300028009847002801D00134F4E72000F8BD5E
:107D4000704710B51C3000F0AFF910BD10B51C30F5
:107D500000F09CF910BD10B51C3000F0ABF910BD5F
:107D600070B5437E0D00002B01D1002070BD643042
:107D7000040000F0A8F90028F7D12000290000F045
:107D800076F90120F2E70000F7B50193FA23002508
:107D900004009B0083600B4B4560083303601C307C
:107DA0000F00160000F058F92000643000F054F97C
:107DB0006B461B79276166756576A5762000A375ED
:107DC000FEBDC046D8F00000012330B5A024C37525
:107DD000837D13499B005A58437DC132114DFF32B8
:107DE000E40592009B005B581551CC22C133FF3350
:107DF0009B001D5104690C4B5204E250052204699A
:107E0000243BE250837D04699B005A58A123DB0088
:107E1000E250437D02699B005958044BD15030BD5C
:107E2000F8F000000C060000240500000C0500001E
:107E3000A022002310B50469D200A3500A4CA1422D
:107E40000FD90A4C8C425B4109495B420B40CD2162
:107E5000C9045B18046907496350052103699950F7
:107E600010BDCC235B04F5E7A086010090D0030091
:107E7000000098FD24050000F7B5040000200D0067
:107E80000193824265D01600402A00D9402627007F
:107E90001C37380000F0F6F8B1232269DB00D5501A
:107EA00080220123216992008B50A27E002A03D1F7
:107EB00022691362226913600025731EAB4207D149
:107EC000019B002B04D0802202212369920099504B
:107ED000012223691A622369FC33DA68002A02D17D
:107EE0009A6A002AF9D09A6A002A0BD1DA60A32391
:107EF0002269DB00D1583800C9B2013500F0B7F86B
:107F0000B542DAD3019B2269002B0FD11300FC3359
:107F10009B6A002B0AD10133A376D3612369FC331A
:107F2000DA6C002AFCD00022DA640AE00023012186
:107F3000A37651611A002369FC3399680029FCD0AB
:107F40009A602369FC339A6A002A01D000229A625F
:107F5000E8B2FEBD10B50123FFF78EFF10BD030090
:107F6000AC3310B504001970643000F08BF80123B5
:107F7000637610BD0023020070B5AC3243760D006D
:107F80001178B12204000069D20081508022216959
:107F900092008B502269013313622269936026009C
:107FA0006436300000F080F8002812D0300000F075
:107FB0006DF81E4B2269D0502369FC331A6A002ADF
:107FC00002D19A6A002AF9D09A6A002A01D11A626B
:107FD000E5E723690122002D0DD11900FC31896AE2
:107FE000002908D1DA612369FC33DA6C002AFCD05D
:107FF0000022DA6407E05A612369FC339A68002A98
:10800000FCD000229A6000202369FC339A6A8242E5
:108010000BD098622169064A8B588B501800022BAE
:1080200003D0181F431E9841033070BD1C0500008B
:10803000C404000010B50121FFF79CFF10BD000033
:1080400010B51323142202490248FFF79DFE10BD0C
:1080500000400040101B002010B540220021040009
:1080600004F030FA002320002364636410BD10B5CF
:108070003F24026C531C2340446C9C4201D0815429
:10808000036410BD0023036443647047436C026CB7
:10809000934206D03F21C25C01330B404364100081
:1080A000704701204042FBE7036C406C181A00D572
:1080B00040307047436C026C934201D0C05C704703
:1080C00001204042FBE73F22036C406C0133134028
:1080D000181A43425841C0B27047000003210A48B1
:1080E00002680A430260094802680A4302600849BC
:1080F000084A094B9B1A03DD043BC858D050FBDCEF
:1081000000F012F8F8F700F824050040540500408C
:1081100048F600000000002070020020FEE7FEE7A5
:10812000FEE7FEE7FEE7FEE7014B024A1A607047F2
:10813000380000200024F4000120704710B50368C7
:108140001322DB69984710BD70470000054B026998
:10815000D1500369FC331A6A002AFCD000220120A6
:108160001A6270471C050000030010B55C331A78D2
:108170001F231A401E3B19009140114AD167C222A9
:10818000042104699200A150026953600269D3601E
:10819000A02300220169DB00CA5001230169094ABA
:1081A0005B428B500169084A8B5001690C3A8B5035
:1081B000016908328B501430FFF764FF10BDC046D0
:1081C00004E100E00C0500001405000010B51430B7
:1081D000FFF76AFF10BD10B51430FFF76BFF10BD3D
:1081E00010B51430FFF752FF10BD0000030070B54A
:1081F0005E331A780469724BE25003005D331A78DB
:108200000469704BE250030061331C7802696E4BC5
:10821000012C00D09EE005005F352E78A225ED00F0
:108220005651020060321578A1220669D200B5507D
:108230000269D4509623DB00994200D88CE0962343
:108240001B01994200D88AE096235B01994200D82D
:1082500088E096239B01994200D885E0E1239B01A9
:10826000994200D882E09623DB01994200D880E051
:10827000E123DB01994200D87DE096231B0299425D
:1082800000D87AE0E1231B02994200D877E09623D8
:108290005B02994200D874E0E1235B02994200D866
:1082A00071E0E1239B02994200D86EE0474B99426E
:1082B00000D86CE0E123DB02994200D86AE0E122B9
:1082C000002312038A425B41414A5B4213408022F1
:1082D00052059B1801693F4A8B50A0230422016973
:1082E000DB00CA5000210369FC33D9600369FC3309
:1082F0001962012301690B6001698B60C121046966
:10830000890062501F215C3002780A40934062313C
:10831000314AFF3153500021415600293CDA0F23E6
:108320000B40083B2D4C9B089B001B19032421404C
:10833000A140FC348C40DD69A5432C00C0258D4054
:1083400029002143D9611F23017819401E3B8B402E
:10835000136070BD00246CE79E23DB02BAE79D2307
:108360001B03B7E71E4BB5E71E4BB3E7EC239B039C
:10837000B0E71D4BAEE71D4BACE71D4BAAE71D4B0D
:10838000A8E71D4BA6E71D4BA4E71D4BA2E78023E2
:10839000DB049FE71B4B9DE78C080F4BA400E41800
:1083A00003230B40FF21C025DB009940AD00665937
:1083B0008E433100C0269E4033000B436351C2E719
:1083C0000C050000140500006C05000090D00300AF
:1083D00000D0BEFE2405000000E100E000ED00E05A
:1083E00000B013000050270000A04E0000F0750000
:1083F00000509D0000F0EB0000903A0100E0D70132
:1084000000B0AF0300705F07F7B5009308AB1B78AF
:1084100000250193FA2304009B0083600E4B456006
:108420000833036014300F001600FFF715FE230019
:108430005C3327611E70009B084A9B0099582300FB
:108440005D331970019B20009B009A5823005E3316
:10845000DD701A70FEBDC0467CF10000F8F000002F
:10846000036910B51A00FC32D2680400002A0AD051
:10847000A322D20099581430C9B2FFF7F8FD0022A8
:108480002369FC33DA6010BD10B50248FFF7E8FF3E
:1084900010BDC046C81B0020162307B5022200935A
:1084A0000249013B0248FFF7AFFF07BD0020004033
:1084B000C81B002010B5002801D004F0BFFA10BD81
:1084C0000849094A094B10B51B688858FA22190A4D
:1084D0001B0618439200002301F0E8FF4904C00B7B
:1084E000084310BD00100140040500002C1C0020B2
:1084F00070B5041E09D0FFF7E3FF050000F014F883
:10850000FFF7DEFF401BA042F8D370BD0022044BF2
:108510009A60044A13680133DBB213607047C046A7
:10852000FC1001402C1C00207047704710B500F073
:108530005FF8FFF7FAFF0120FFF7DAFFFFF73CFBD8
:10854000FFF74CFB024B002BFAD000E000BFF7E72F
:1085500000000000F8B54C1EA1410125104B114F41
:108560008000C3584C4238680F499D40160001F006
:10857000DBFD0A21704301F0D7FD2C4003002200EF
:1085800029000A4800F016F8FA21094C89004443F2
:10859000386801F0C9FD0100200001F0C5FDF8BDFB
:1085A000F8F000003800002040420F001005005095
:1085B0001027000030B504680C40944206D1013BFE
:1085C000002BF8D112E0013B002B0FD004680C40C7
:1085D0009442F8D1002405680D40954204D101343D
:1085E0009C42F8D1002002E0201C00E0181C30BDA5
:1085F000C420114B80001A5810491140C0221202A9
:108600000A431A50C0218022490092025A501A602F
:108610008023A3220021DB05D20099500122F930EA
:108620009A60074BFF301950C12002318000195069
:10863000403019501A60704700E100E0FF00FFFF72
:1086400000100140014B18607047C04684000020B4
:10865000F7B5002320285AD8384B8000C258042A86
:108660005BD007D8022A54D055D80423012A09D058
:1086700000234CE0062A54D051D31A2A53D00223A7
:108680001B2AF5D12E4A116808294ED909294FD045
:108690000A240226A02001252A4AC00015502A4893
:1086A0002A4D07681C20BF00074029480197006831
:1086B0005759009027481B0207401F43C0230098CA
:1086C0009B020340FF2057515759000207401F43A8
:1086D000019B1F43009B58016023184007433E4302
:1086E000565101251C4B156058680028FCD000200D
:1086F0005860A1230125DB00D3585560A025ED006B
:1087000050511BB2A14202D015D2611ACB401800C1
:10871000FEBD0823B6E71023B4E72023B2E74023C9
:10872000B0E78023AEE70123ACE708240026B1E7D9
:108730000C000126AEE7091B8B40E8E7F8F00000CB
:1087400080000020007000403C0000200405000074
:1087500040000020FF00FFFFFC700040F0B5202823
:108760005BD8364B8000C258354B1E68002E30D186
:10877000C227344BBF00D859334C03250440C020D6
:1087800000022043D851C02480206400800018518A
:108790002E4F18602E4B803CD859FF3CA043D85137
:1087A0000437D859A8432043D8510837D8590C3535
:1087B000A8438446072065462843D851A820C00016
:1087C0001E50C1208026800076021E501C601C4B6B
:1087D0001C60142500202B001E4C2E0046433659E9
:1087E000771C1BD14343E250A0230325C132FF3243
:1087F0009200DB05D550184B1A68082A14D11423AF
:108800004343E3189A6812485132FF32920059608C
:108810001150DA68C1239B00C250F0BD9642E1D0EE
:1088200001300328D9D1F8E7082A02D9083AD14003
:10883000E5E708239A1A9140E1E7C046F8F0000006
:10884000301C002000E100E0FF00FFFF04050000F5
:108850000090004044000020840000202149F0B531
:108860004A6C2148002A14D0A025A1260023012407
:10887000ED05F600C258571C06D0C7187F68002FB8
:1088800002D027009740AF5114333C2BF2D1002384
:108890004B64A0230121DB0500260F009C46142316
:1088A0004B43C3181A1F1268104C0E4D9200141936
:1088B0005219526C002A10D01A00143A1268551C32
:1088C00009D0103B1B68FF2B05D03B009340654649
:1088D0001A00074BEA50FC34666401310429DED1EA
:1088E000F0BDC046FC9000404400002000900040D5
:1088F0000C05000000B5202810D80C4A80008358D1
:1089000003290BD8A0220800C133FF33D2059B00F6
:1089100001F000FC020905070021D15000BD0C2127
:10892000FBE70421F9E70321F7E7C046F8F0000070
:1089300020280AD8074B8000C25801239340A02268
:10894000D205002902D1044953507047A121C90022
:10895000FAE7C046F8F000000C0500000300002014
:10896000202B0AD8A021A222C905D2008858034A88
:108970009B009B58D840012318407047F8F0000036
:10898000F7B506000D000C008B180193019B671BC7
:108990009C4207D0336821781B6830009847013427
:1089A0000028F3D13800FEBDF0B5C64600B5CB0FA8
:1089B0009846404A4B005B0D9A1882B00D000400A7
:1089C000132A2FDC002A49DB3B4F17413E000E40A3
:1089D000064323D07F08390029400C430AD0374989
:1089E000BD438C4663445C425C418023DB021341FF
:1089F000E4071D434146CE0031492B008E19220069
:108A0000346875682000290001F0F6FE009001919D
:108A10000098019922002B0003F086F802B004BCF4
:108A20009046F0BD332A08DD8023DB009A42F5D161
:108A300002000B0001F0E0FEF0E7224A944601221A
:108A400063445242DA400242E8D052080242D1D096
:108A500094438022D2051A411443CBE74B005B08B4
:108A60000343DBD00B031B0B1C43634223438024D3
:108A70004D0C24031B0B23406D042B43190043466C
:108A8000DA000F4B9B181C685D6802000B00200089
:108A9000290001F0B1FE0090019100980199220097
:108AA0002B0003F041F842464B005B08D6073343E6
:108AB0001900B3E701FCFFFFFFFF0F00EEFBFFFF14
:108AC000B0F10000EDFBFFFFF8B5274A4B005B0D4E
:108AD0009A180C000700132A10DC002A36DB234BFF
:108AE00013410B423AD0802424031441002064181F
:108AF0009C430600250030002900F8BD332A0EDD16
:108B000080230600DB000D009A42F4D102000B0026
:108B10003800210001F070FE06000D00EBE7144D57
:108B20000600AC46012563446D42DD40AC46634619
:108B30000D000342DFD033239A1A323B93401818BA
:108B4000874200D94C1C63469843D2E7C90FCC0733
:108B50000020531CCDD1074B1C43CAE706000D0073
:108B60000028C0D1C7E7C04601FCFFFFFFFF0F0090
:108B7000EDFBFFFF0000F03F30B5214A4B0087B00E
:108B80005B0893421EDD1F4A934205DD02000B0085
:108B900002F0CAFF07B030BD02AA00F095F8032327
:108BA0001840049A059B012813D002281DD00028E4
:108BB00014D00298039900F06FFB80231B069C469B
:108BC0006144E7E7002300220093002301F0DEF870
:108BD000E0E70298039900F05FFBDBE701240298CD
:108BE0000399009401F0D2F8D4E701240298039984
:108BF000009401F0CBF880231B069C466144C9E732
:108C0000FB21E93FFFFFEF7FF0B54746CE4680B539
:108C10008DB004000D0000F067FA294B06001B78A8
:108C20000F005BB29846013310D022002B002000C9
:108C3000290003F0C1FA8146002807D10022002351
:108C40002000290001F00AFC002806D1300039007C
:108C50000DB00CBC90469946F0BD01230293194B10
:108C60000694079503934B460A934346049405954F
:108C7000002B15D0002300221900100002F0D8F8B4
:108C8000434608900991022B0ED103F0AFFB21233C
:108C900003600A9B0193002B0CD1089E099FD5E726
:108CA000002300240893099402A801F0C1F90028C8
:108CB000EFD1EAE703F09AFB0A9B01930360ECE72C
:108CC00088000020C0F10000F0B54E464546DE4663
:108CD0005746E0B5E14B4C008FB09046894664089A
:108CE0009C4200DC87E0DE4B9C4222DCDD4A00290E
:108CF00000DC92E0DC4B02F017FFDB4B06000F00BC
:108D00009C4200D17EE1D94AD94B02F00DFF02000E
:108D10000B00414630000A604B60390002F004FF4E
:108D2000D34BD24A02F000FF434601259860D96038
:108D30006BE0D04B9C4200DC8FE0CF4B9C4200DDCF
:108D400055E1CE4A231592469A4451460905631AC5
:108D500019001D00040003F04BFA03F07FFA020033
:108D60000B00200029000892099302F0DDFE00228A
:108D7000C34B02F067FC0F00060003F039FA03F062
:108D80006DFA04000D0002000B00300039000A9457
:108D90000B9502F0C9FE0022B94B02F053FC0022F1
:108DA00000230C900D9101F053FB002800D192E1BB
:108DB000002300222000290001F04AFB43424341E6
:108DC0000133B04A41460192022208A8009252465D
:108DD00000F07CFB4B460500002B16DA8022434650
:108DE0001206944642465B68454263445360D3682A
:108DF0006344D36009E00B00020041460A604B6007
:108E00000022002300258A60CB6028000FB03CBC04
:108E100090469946A246AB46F0BD934B01F0ECFC60
:108E2000914B06000F009C4200D13DE18F4A904BD0
:108E300001F0E2FC02000B00414630000A604B608A
:108E4000390002F071FE894A894B01F0D5FC0125F9
:108E500043466D429860D960D7E701F049F88A4AE5
:108E60008A4B06000F0002F0EDFB0022884B01F058
:108E7000C3FC03F0BDF9050003F0F0F9794A7A4B21
:108E80000490059102F0DEFB02000B003000390077
:108E900002F04AFE754A06000F0004980599744BCB
:108EA00002F0D0FB029003911F2D00DCC7E0029A74
:108EB000039B3000390002F037FE83468A46534652
:108EC0005B0024155B0DE31A102B6CDD04980599EB
:108ED000D322674B520502F0B5FB02000B003000B5
:108EE00039000292039302F01FFE0A0001001300F2
:108EF0000691079202003900300002F015FE029A36
:108F0000039B02F011FE06000F0004980599614AC8
:108F1000614B02F097FB32003B0002F005FE069E1B
:108F2000079F0B000200390030000292039302F009
:108F3000FBFD4B005B0D83468A46E41A312C32DD83
:108F400004980599B822544B920502F07BFB03006C
:108F50000C000200029303940B000698079902F09C
:108F6000E3FD02000B0006000F000698079902F0CF
:108F7000DBFD029A039B02F0D7FD484A0290039161
:108F800004980599464B02F05DFB029A039B02F0A0
:108F9000CBFD02000B00300039000292039302F077
:108FA000C3FD83468A465A465346414630000A600E
:108FB0004B60390002F0B8FD029A039B02F0B4FD49
:108FC00044460B000200A260E3604B46002B00DB2E
:108FD0001BE75B46236080231B06534463608023AA
:108FE0001B069C466144A060E1606D420DE70B00EA
:108FF000020002F099FD434600259860D960186090
:10900000596002E7D3221A4B520502F08DFD214A26
:10901000214B0D00040002F087FD02000B004146C9
:1090200020000A604B60290002F07EFD1A4B194AAD
:1090300002F07AFD434601259860D960E5E602001A
:109040000B003000390002F06FFD6B1E154A9B00CB
:109050009B5883468A46A342A5D130E7FB21E93FCE
:109060007BD9024000004054FB21F93F3163621A72
:1090700061B4D03DFB213941FFFFEF7FEAFBFFFFE9
:109080000000704148F2000083C8C96D305FE43FC2
:109090000000E03F7370032E8A19A33BC1492025CD
:1090A0009A837B39C8F10000D3220C4B520501F0A2
:1090B000A3FB0B4A0B4B04000D0001F09DFB0200CB
:1090C0000B00414620000A604B60290002F02CFD95
:1090D000034A044BB9E6032373E6C04661B4D03DAE
:1090E0007370032E8A19A33BF8B54746CE46674BEB
:1090F00080B50A000F00190005003940994200D1DF
:109100009BE004000100002F69DD3F1500D1B4E0B1
:109110005F4B12039C468023120B5B0313435B00DF
:10912000CA0F67449B184A00F80703D5D20F5B00AB
:109130009B188A0079108C460021802016248946CD
:1091400080030D189D4202DC29185B1B8144D50F5A
:109150005B00013C5B1952004008002CF1D100205B
:109160008046802020250027000609E08B425CD045
:10917000D40F5B00013DE31852004008002D16D0CB
:10918000C4198B42F2DD27180E00002C49DB5B1A54
:10919000A242894149425B1A121BD40F5B00013D78
:1091A00080443100E31852004008002DE8D11343F9
:1091B0004ED143465B0837494A46884649465210D5
:1091C0004244C90702D5802109060B4361460F05B9
:1091D000BD18180029000CBC90469946F8BD7B00CC
:1091E0005B0803433900002BF5D0002F3CD1E30A84
:1091F000153A6405002BFAD08020400303423FD18A
:10920000002700E00F005B00791C0342FAD0250024
:1092100020208D40401A2900D71B2200C2401A434B
:1092200076E7FE43F60F8E19B1E79442A0D82718CF
:10923000002CF6DB1E000023AEE702003B002800F6
:10924000390002F0FFF92A003B0001F0D5FAC2E72D
:109250004346013303D0434601335B08ABE70123A8
:1092600098460023C144A6E73B00020002F05CFCE4
:1092700002000B0001F0DCFDADE713000022BBE7AC
:109280000127210020207F42C6E7C0460000F07F72
:1092900001FCFFFF0000E03FF0B54746CE4680B539
:1092A00087B000920193754B4F00814688467F0836
:1092B0009F4263DC02F09CFF002800D1D4E04A46C4
:1092C00043464846414602F0BDF904000D006C4A91
:1092D0006C4B02F0B7F96C4A6C4B01F08DFA22002E
:1092E0002B0002F0AFF96A4A6A4B02F01DFC220023
:1092F0002B0002F0A7F9684A684B01F07DFA2200C2
:109300002B0002F09FF9664A664B02F00DFC22002A
:109310002B0002F097F9644A644B01F06DFA2200C9
:109320002B0002F08FF9029003910022604B200085
:10933000290002F087F9029A039B06000F00200023
:10934000290002F07FF9009A019B04000D004846B5
:10935000414602F077F902000B002000290002F0DC
:10936000E3FB02000B003000390002F0DDFB0200DD
:109370000B0000204F4902F0D7FB70E002000B0009
:1093800002F060F904000D003D4A3E4B02F05AF92C
:109390003D4A3E4B01F030FA22002B0002F052F918
:1093A0003B4A3C4B02F0C0FB22002B0002F04AF982
:1093B000394A3A4B01F020FA22002B0002F042F920
:1093C000374A384B02F0B0FB22002B0002F03AF98A
:1093D000354A364B01F010FA2B00220002F032F928
:1093E000354B029003919F429FDD344B00229F42F8
:1093F0003DDC334900207B182E4916001F0002F087
:1094000093FB049005910022294B2000290002F0D3
:1094100019F932003B0002F087FB029A039B060019
:109420000F002000290002F00DF9009A019B0400B2
:109430000D004846414602F005F902000B002000ED
:10944000290002F071FB02000B003000390002F02D
:109450006BFB02000B000498059902F065FB07B056
:109460000CBC90469946F0BD00201249F7E7154B19
:10947000002604920593144FC5E7C046FFFF3F3E08
:10948000D43888BEE9FAA8BDC4B1B4BD9EEE213E71
:10949000AD529C804F7E923E9015CB19A001FA3EB2
:1094A0007751C1166CC1563F4C5555555555A53F82
:1094B0000000E03F0000F03F3233D33F0000E93FBF
:1094C0000000E0FF0000E73F0000D23FF0B5DE46BD
:1094D0004E4645465746E0B5DC4CA5440D91140078
:1094E0001900A49A0993DA4B9200D6584D1E0390A6
:1094F0001821E01E0696029500F0A0FEC34301006D
:10950000DB1719404B1C9A009B1ADB001B190B91AF
:1095100005934C1B771918D4A59BA5009C463F19B1
:1095200022AE6544013707E0286802F097FE013457
:1095300003C60435BC4208D0002CF5DA0020002117
:10954000013403C60435BC42F6D1069B002B01DA78
:1095500000F0FDFB069B03990133DB009A46099B53
:10956000DA00944600920022914672AA0492B94A07
:109570006144934688469AAB63449B44029B002B0C
:1095800000DABCE15D4600260027039C4D442A68B2
:109590006B6803CC02F056F802000B003000390073
:1095A00001F02AF9083D06000F004445EFD1049B65
:1095B0004B441E605F6008239C46E144D145DDD1E9
:1095C0000EA804218446494261448C46069A9300C1
:1095D0009C44614684460A910399083B63448C4647
:1095E0000C93009B009263449B46009A0498D10020
:1095F00003008C46634408911E685F68002A33DDCF
:10960000954980468C466244D300984470AB9A4694
:109610000EAB99460022914B3000390002F012F84F
:1096200002F0E6FD02F01AFE00228D4B04000D0050
:1096300002F008F802000B003000390002F074FA62
:1096400002F0D6FD4B4601C39946434620001A68F6
:109650005B68290001F0D0F808235B429C46E04497
:1096600006000F00D045D5D1059B30001A00390007
:10967000984600F0DFFCFF2300229B0504000D004C
:1096800001F0E0FF00F038FC0022764B01F0DAFF39
:1096900002000B002000290002F046FA0D00040031
:1096A00002F0A6FD814602F0D9FD02000B00200069
:1096B000290002F039FA060040460F00002800DCBD
:1096C000EEE0009B18215A1E92000EAB9B58091A1F
:1096D0001D000D41A9448D405D1B0EAB9D5017230D
:1096E0001B1A1D41002D2DDD01239C46009BE144EA
:1096F000002B00DC1CE20E9C0123002C00D0B5E006
:10970000009A012A09D099000EAA54580133002C5E
:1097100000D0ACE0009A9A42F5D1059B002B0EDDFB
:10972000012B00D1A8E1022B09D1009B0EA95A1EE2
:1097300092000EAB9B5807939B029B0A8B50022D05
:1097400000D1C1E0002300223000390000F080FE8B
:10975000009B002800D194E2069A591E8A4210DC30
:10976000414A0A9894460EAA6344944600229B00FC
:1097700063441C68043B22438342FAD1002A00D090
:10978000C0E0069B0EAA013B9B00D358002B00D0E3
:10979000B3E001220C9B043B596801320029FAD046
:1097A000009B9C466244110007921A0001338B42D1
:1097B00046DC0B9863468046A59C4344A046099C22
:1097C0009B00A1464A449844D30022AA9146049A99
:1097D00099449446089BA59A634484466144944600
:1097E0009A468B00634400934346586802F036FD66
:1097F0004B4618605960029B002B24DB4D46039CAE
:109800000026002701E0286869680CCC01F01AFFE7
:1098100002000B003000390000F0EEFF083D0600AA
:109820000F005C45EFD153469E60DF6004239C46E9
:109830000433E0449C46009BE144E2449845D3D184
:10984000079B0093D1E600260027ECE794FDFFFF7D
:1098500090F3000018FEFFFFFFFFFF1F0000703EA7
:109860000000704100002040FFFFFF3F00218022E8
:109870005204141B0EAA5450009999420EDD0EA8F2
:1098800084469B000EAA8900D25861446344CF48A5
:1098900000E01A68821A04C38B42FAD101243CE723
:1098A000059B002B06D1009B0EAA013B9B00D558BF
:1098B000ED1517E70022C64B300000F0EDFD002843
:1098C00000D024E100253DE732003B000020C149E3
:1098D00002F02AF906000F00002C00D132E7059AA9
:1098E0000020BC4900F0A6FB02000B00300039004C
:1098F00002F01AF906000F0024E7012250E70026C3
:10990000002754E64B46059A079388468B000EA91C
:10991000CB58183A08950592002B0DD18C4641463C
:10992000AD4B43449B006344043B58680139183AEB
:109930000028F9D088460592059A0020A54900F034
:1099400079FB434604000D00002B00DA05E29E007F
:109950000EAB9C464346DB0066449C46059370ABC9
:109960009946049F67440097306802F077FC220014
:109970002B0001F067FE002238607960974B2000D1
:10998000290001F05FFE083F04000D00043EB945C8
:10999000EAD14AAB03939B4600239A46069B424674
:1099A000994643460132029204934B46002B00DA5B
:1099B000AAE080208A4B009D9846C0058949002670
:1099C0000027002408E008239C460835E04454455D
:1099D00011DC4346186859682A686B6801F032FE4A
:1099E00002000B003000390000F006FF01340600D1
:1099F0000F00A145E7DA5B46C0C39B4601239C46A6
:109A0000009BE244083B0093029B9A45CDD1049B06
:109A10009846A49B022B00DD8EE0002B37DC1FD183
:109A2000059B00271D00039B00249C461E006544E7
:109A3000083E2A686B683800210000F0DDFE083D12
:109A400007000C00AE42F4D1089B002B03D080230A
:109A50001B069C4664443A0023000D990A604B6043
:109A60000720079B18409B239B009D443CBC9046CD
:109A70009946A246AB46F0BD009B0EA95A1E920025
:109A80000EAB9B5807935B025B0A8B5057E643462D
:109A9000002B00DA70E100200021DB004AAAD61872
:109AA00048AF32687368083E00F0A6FEB742F8D1AE
:109AB000089B002B00D025E10B0002004A984B992F
:109AC0000D9C2260636002F02FF8434607000C00F3
:109AD000002B13DD01254CAEB14638002E002100CD
:109AE0004C4601360CCC00F087FEA146B045F7DAB3
:109AF000089B07000C00002B00D015E13A00230062
:109B00000D998A60CB60ABE70026002773E701233D
:109B10009C46009BE1440225002B00DDEBE5320072
:109B20003B0000202B4901F0FFFF06000F0009E673
:109B30000024F2E54AAB0393A49B032B00D08FE7EC
:109B40004346002B00DC14E1039ADB009B46130024
:109B500091465B441E685F68234B43440293DB00DD
:109B6000994448AB9A464B465C681B681800210034
:109B700032003B000090019100F03EFE04000D0019
:109B800002000B000098019901F0CEFF3B0032006B
:109B900000F032FE4B469860D9601C605D6008237F
:109BA0005B429C46E14426002F00CA45DBD1434678
:109BB000012B00DCE3E0039A13005B441E685F683E
:109BC000029BDB0099464A44904610E0FFFFFF00ED
:109BD0000000E03F0000F03FFFFFFF3F0000703E4D
:109BE00050F30000FB21F93FFFFFFF1F984643465B
:109BF0005C681B681800210032003B000090019156
:109C000000F0FAFD04000D0002000B00009801991D
:109C100001F08AFF32003B0000F0EEFD4346039A5C
:109C20009860D9601C605D60083B26002F009A4256
:109C3000DCD14D469446002600244746083565444D
:109C40002A686B683000210000F0D6FD083D060050
:109C50000C00AF42F4D1039B4A9F5D689968D868B5
:109C6000089B002B65D08022120694460D9B65440C
:109C7000604464441F605D609960D8601E615C61EF
:109C8000EEE69A464B460793059B30005A42390050
:109C9000089500F0CFF900223A4B06000F0000F0C3
:109CA000FBFB002824D0384B00223000390001F0A3
:109CB000C9FC02F09DFA52460400950002F0CEFA6B
:109CC0000022304B01F0BEFC02000B0030003900D6
:109CD00001F02AFF02F08CFA0EAA50510122059BD6
:109CE000524418339046059393000EAAD45023E6AD
:109CF0005346300039009C0002F07AFA0EAB18513E
:109D0000D04619E680230D9A1B06CB1810605360CD
:109D10000B0002004A984B9901F006FF43460700EA
:109D20000C00002B00DDD5E680231B069C46644416
:109D3000E4E62B003A000D9D2A606B600A000300E8
:109D4000AA60EB60320023002A616B6188E6099B00
:109D5000DB00009372AB049332E4A49B022B00DD82
:109D6000E8E6002B00DD92E600D079E6002700242B
:109D70006AE6002600246EE70020002198E600260F
:109D8000340068E7000070410000703EF0B5CE4638
:109D9000474680B587B000920193474A4B00814601
:109DA00088465B08934207DC4146484602F020FAA9
:109DB0004146031E484666D04A4643464846414609
:109DC00001F040FC04000D0002000B004846414633
:109DD00001F038FC394A3A4B06000F0020002900F8
:109DE00001F030FC374A384B01F09EFE22002B0078
:109DF00001F028FC354A364B00F0FEFC22002B0017
:109E000001F020FC334A344B01F08EFE22002B007F
:109E100001F018FC314B324A00F0EEFC0E9B029030
:109E20000391002B34D00098019900222D4B01F0B2
:109E300009FC029A039B049005913000390001F05F
:109E400001FC02000B000498059901F06DFE220050
:109E50002B0001F0F7FB009A019B01F065FE224AFE
:109E600004000D00214B3000390001F0EBFB020033
:109E70000B002000290000F0BFFC02000B00484648
:109E8000414601F051FE07B00CBC90469946F0BD2A
:109E900002000B002000290001F0D4FB124A134BF2
:109EA00001F042FE32003B0001F0CCFB4A46434643
:109EB00000F0A2FCE7E7C046FFFF3F3E7CD5CF5A4B
:109EC0003AD9E53DEB9C2B8AE6E55A3E7DFEB1573B
:109ED000E31DC73ED561C119A0012A3F1111813F81
:109EE000A6F810110000E03F495555555555C53F9E
:109EF00049004B0819007047474AF0B54F46914654
:109F00004B005B0D99444646D6464A46C0B505000F
:109F10000C000E0088460700132A27DC002A4BDBC2
:109F20003E4B13419A460B0052461340034318D050
:109F30003B4A3C4B2800210000F05EFC002200233D
:109F400000F0A0FA002847D0002C04DA80234A460B
:109F50005B03134198444646534600279E4338000E
:109F600031001CBC90469946A246F0BD332A08DD5C
:109F70008023DB009945F4D102000B0000F03CFC8B
:109F8000EFE7294A9446012263445242DA4092465E
:109F90000242E6D0224A234B2800210000F02CFC8C
:109FA0000022002300F06EFA002815D0002C1EDBE2
:109FB000534646469F430FE0194A1A4B280021009A
:109FC00000F01AFC0022002300F05CFA002803D005
:109FD000002C04DB0027002638003100C1E76400B4
:109FE000640825430027002DF6D0104EF4E74B46B9
:109FF000142B0BD03422D21A012393405D19BD4299
:10A0000008D201239C462F00E044D1E7133B9C4635
:10A01000E044CDE72F00CBE701FCFFFFFFFF0F007F
:10A020009C7500883CE4377EEDFBFFFF0000F0BF2D
:10A03000002070474B0070B55B0D14000A00002B28
:10A040001AD14B005B08034315D0234B002201F0CB
:10A05000F9FA224B9C422DDB0A004B005B0D363B8C
:10A060001F4DE318AB422ADC002B0DDD1D4C1B05F8
:10A0700022401A43110070BD1B4DAB42F0D10200CB
:10A080000B0000F0B9FBF6E71D00353519DA174B68
:10A0900002009C4209DD0B001548164900F032F819
:10A0A000134A144B01F0CEFAE5E70B0012481349AE
:10A0B00000F028F8104A114B01F0C4FADBE7020067
:10A0C000E9E7084C363322401B05134319000022F0
:10A0D0000B4B01F0B7FACEE700005043B03CFFFF56
:10A0E000FE070000FFFF0F80FF07000050C30000C5
:10A0F0009C7500883CE4377E59F3F8C21F6EA501B9
:10A100000000903C30B54A00DB0FDB0752081A43D1
:10A11000110030BD02B4714649084900095C49008C
:10A120008E4402BC7047C046002243088B4274D361
:10A1300003098B425FD3030A8B4244D3030B8B4248
:10A1400028D3030C8B420DD3FF22090212BA030C51
:10A150008B4202D31212090265D0030B8B4219D332
:10A1600000E0090AC30B8B4201D3CB03C01A524152
:10A17000830B8B4201D38B03C01A5241430B8B429A
:10A1800001D34B03C01A5241030B8B4201D30B0383
:10A19000C01A5241C30A8B4201D3CB02C01A5241AA
:10A1A000830A8B4201D38B02C01A5241430A8B426D
:10A1B00001D34B02C01A5241030A8B4201D30B0256
:10A1C000C01A5241CDD2C3098B4201D3CB01C01A70
:10A1D000524183098B4201D38B01C01A524143097A
:10A1E0008B4201D34B01C01A524103098B4201D368
:10A1F0000B01C01A5241C3088B4201D3CB00C01AD5
:10A20000524183088B4201D38B00C01A524143084C
:10A210008B4201D34B00C01A5241411A00D2014671
:10A22000524110467047FFE701B5002000F0F0F8FA
:10A2300002BDC0460029F7D076E7704703460B43BE
:10A240007FD4002243088B4274D303098B425FD32F
:10A25000030A8B4244D3030B8B4228D3030C8B425B
:10A260000DD3FF22090212BA030C8B4202D3121241
:10A27000090265D0030B8B4219D300E0090AC30B16
:10A280008B4201D3CB03C01A5241830B8B4201D3C3
:10A290008B03C01A5241430B8B4201D34B03C01AAC
:10A2A0005241030B8B4201D30B03C01A5241C30A24
:10A2B0008B4201D3CB02C01A5241830A8B4201D395
:10A2C0008B02C01A5241430A8B4201D34B02C01A7F
:10A2D0005241030A8B4201D30B02C01A5241CDD224
:10A2E000C3098B4201D3CB01C01A524183098B426F
:10A2F00001D38B01C01A524143098B4201D34B0158
:10A30000C01A524103098B4201D30B01C01A5241BA
:10A31000C3088B4201D3CB00C01A524183088B4241
:10A3200001D38B00C01A524143088B4201D34B002A
:10A33000C01A5241411A00D201465241104670479C
:10A340005DE0CA0F00D04942031000D340425340A1
:10A3500000229C4603098B422DD3030A8B4212D361
:10A36000FC22890112BA030A8B420CD38901921193
:10A370008B4208D3890192118B4204D389013AD0D0
:10A38000921100E08909C3098B4201D3CB01C01AA5
:10A39000524183098B4201D38B01C01A52414309B8
:10A3A0008B4201D34B01C01A524103098B4201D3A6
:10A3B0000B01C01A5241C3088B4201D3CB00C01A13
:10A3C000524183088B4201D38B00C01A5241D9D22B
:10A3D00043088B4201D34B00C01A5241411A00D2AC
:10A3E0000146634652415B10104601D34042002BA8
:10A3F00000D54942704763465B1000D3404201B527
:10A40000002000F005F802BD0029F8D016E77047DB
:10A410007047C046D0400B1C1141203A03D49C46E3
:10A420001341184363465242934018437047C04655
:10A430008446101C62468C46191C634600E0C046E8
:10A440001FB501F097F8002801D40021C8421FBDB4
:10A4500010B500F0EFFF4042013010BD10B501F023
:10A4600089F8002801DB002010BD012010BDC04686
:10A4700010B501F07FF8002801DD002010BD01209B
:10A4800010BDC04610B501F011F8002801DC002015
:10A4900010BD012010BDC04610B501F007F800281E
:10A4A00001DA002010BD012010BDC046F0B5CE4637
:10A4B000474615042D0C2E0080B50704140C3F0CE4
:10A4C0009946030C7E435D43674363437F19340C15
:10A4D000E4199C46A54203D980235B029846C444F4
:10A4E0004B4643435143250C36046544360C240443
:10A4F000A4195B19591820000CBC90469946F0BD70
:10A50000F0B54E4657464546DE46E0B543025B0A87
:10A51000450083B00F1C99462D0EC60F002D57D055
:10A52000FF2D24D08020DB00C00418430023814687
:10A530009A469B467F3D7C027A00FB0F640A120E0E
:10A54000984623D0FF2A4BD0E30080240020E40467
:10A550007F3A1C43AD186B1C474601935346774026
:10A560003A000F2B48D87D499B00CB589F46002BC3
:10A5700000D085E008339A46063B9B467C027A0071
:10A58000FB0FFF25640A120E9846DBD1002C00D089
:10A5900090E0524601231A4392460120DBE74C46E5
:10A5A00058461700022824D0032800D1CFE000220B
:10A5B000002301284DD15802D205400AFF0710435D
:10A5C000384303B03CBC90469946A246AB46F0BD2A
:10A5D000002B5BD104239A46033B00259B46AAE748
:10A5E000FF35002C60D1524602231A4392460220C6
:10A5F000B1E7FF220023DEE74B461B0C9C464B468F
:10A600002604360C180461463300220C6446000C04
:10A6100043434E435043544380191A0C1218964238
:10A6200003D9802149028C4664441B041B0C10048E
:10A63000C01883015E1EB341800E1843130C1B1912
:10A640009B0103431C00230179D5012362081C40B0
:10A650001443019A7F32002A4DDD630704D00F2393
:10A660002340042B00D00434230103D53C4B019A32
:10A670001C408032FE2ABCDCA3015B0AD2B29AE7FE
:10A680000C239A46093BFF259B4654E7180001F02E
:10A6900071FE4A46431F76259A4000236D4291463B
:10A6A0002D1A9A469B4646E7524603231A43924682
:10A6B000032050E7200001F05DFE431F2D1A9C404F
:10A6C000763D002047E780230027DB03FF2272E767
:10A6D000424666E74C463200584662E780234A46C7
:10A6E000DB031A4222D01C4220D123435B025B0AC7
:10A6F0004746FF225FE701239A1A1B2A21DC230029
:10A700000199D3409E318C401A0023005C1EA34166
:10A7100013435A0704D00F221A40042A00D00433EE
:10A720005A0111D49B015B0A002244E780234A4668
:10A73000DB0313435B025B0A3700FF223BE7019513
:10A7400087E70022002336E70122002333E7802336
:10A75000DB0323435B025B0AFF222CE7A0F300002C
:10A76000FFFFFFF770B500283DD0C317C5185D4047
:10A77000C40F280001F0FEFD9E22121A962A07DC63
:10A78000D2B2082833DD083885406802400A23E049
:10A79000992A0BDD052329001B1AD94003001B331E
:10A7A0009D402B005D1EAB4119430D00052801DDC6
:10A7B000431F9D402B000F490B406E0709D00F2609
:10A7C0003540042D05D004335D0102D59F220B4096
:10A7D000121A9B01580AD2B24002D205400AE4077D
:10A7E0001043204370BD002400220020F4E76802DB
:10A7F000400AF1E7FFFFFFFBF0B54F464646D6465D
:10A800000C000903C0B5490A470F5E0039431F0316
:10A81000DB0F9C4665007B0A570F1F436D0DE40F4D
:10A82000760DA146C000B846D200AB1B64457BD074
:10A83000002B5FDD002E00D0A4E03E00164300D1C7
:10A8400012E15E1E002E00D09EE1871A4346B842F8
:10A8500080410125C91A4042091A0B0200D431E196
:10A8600049024E0A002E00D16EE1300001F082FD57
:10A870000300083B1F2B00DD61E120223900D21AC2
:10A880009E40D1409F400E439D4200DD51E15D1B43
:10A890006B1C1F2B00DD7CE12021C91A3D0030001C
:10A8A0008F408840DD40791E8F41310007222843C8
:10A8B000D940002507433A40002A09D00F233B40E6
:10A8C000042B05D03B1DBB42BF417F42C9191F006D
:10A8D0000B0200D426E26A1CC64B55056D0D9A4248
:10A8E00000D106E1C44AFF080A40530752023B4325
:10A8F000120B8EE0002B00D0B8E06B1C5B055B0DEB
:10A90000012B00DC30E1871A4346B842B641CB1A2E
:10A9100076429E1B330200D54CE13B003343A1D16C
:10A9200000220024002570E0002B00DCE5E0002E72
:10A9300000D183E0AF4EB54260D080263604374365
:10A94000B846382B00DC3EE1434613431F007A1E15
:10A9500097413F1887428041404209180B0200D4BA
:10A96000B0E0A44B01359D4200D1C3E0A24A7B0870
:10A970000A4001210F401F435108D30707221F43FC
:10A980003A4099E79B4EB54238D08026360437438B
:10A99000B846382B00DDDCE01F2B00DC30E11E0068
:10A9A0004746203EF740BC46202B04D04026F31AF1
:10A9B00046469E403243170063467A1E97411F4326
:10A9C000CCE0002B00D104E24346134300D159E10F
:10A9D0004B07C00818438023C9081B03194208D03D
:10A9E0004546ED081D4204D14346D00859070843A7
:10A9F0002900420FC9007F4D1143C0004B07CA0810
:10AA00007C49C00803438D4268D012036D05120BC8
:10AA10006D0D002112031800130B0A0D12051A43C5
:10AA2000764B2D0513402B435B00E4075B08234363
:10AA300019001CBC90469946A246F0BD3E00164344
:10AA400012D05E1E002E00D000E1871887428041A0
:10AA500041444042091801250B0233D5022585E700
:10AA600064463300414610001D00C7E7002D00D0AA
:10AA7000DAE00C000443F3D05C1C00D19FE15D4C94
:10AA8000A64200D12FE1DB43382B00DD66E11F2B0E
:10AA900000DD83E120240500E41A0F00DD40D940E9
:10AAA000A0404346A7405B1A441EA04198462F434E
:10AAB0003843171ABA42924143465242991A6446A1
:10AAC0003500CAE607223A40002A00D0F6E64B07D6
:10AAD000CA084849FF083B438D4296D119001143EB
:10AAE00000D19EE1802109030A431203120B414D5C
:10AAF0008FE71500002200238BE7002B00D0C7E072
:10AB00006B1C5F057F0D012F00DCF1E0394DAB427E
:10AB100000D1B9E085180A00854289414244494282
:10AB200051180722CF076D082F4349083A401D00EE
:10AB3000C2E607223049ED1A31403A40BCE63E00F9
:10AB40002838864000279FE6380001F013FC2030AB
:10AB50008EE6434613431F007A1E9741C71BB84237
:10AB600080414042091A78E60E003B000643134339
:10AB7000002D61D1002E00D0F4E0002B00D11BE1AC
:10AB800064463900100039E71A4FBB427AD03300CF
:10AB9000FFE630001F3DE840202B03D04021CB1AB8
:10ABA0009E4037437B1E9F41072207433A400021C6
:10ABB000002589E7171A4346BA42B641591A764228
:10ABC0008E1B64464EE61F2B00DDADE02026474677
:10ABD000F61AB740B9461700B246DF404E463E432C
:10ABE00037005646B240561EB24117434246DA403D
:10ABF0008918AEE6FF070000FFFF7FFFFFFF0F8011
:10AC000020264746F61AB740B9461700B246DF403D
:10AC10004E463E4337005646B240561EB241174399
:10AC20004246DA40891A99E77F4CA6425BD08024DD
:10AC300024045B42214327E7002E0CD1002B00D1D6
:10AC4000CBE0644639001000774DD7E6764FBB4223
:10AC500018D0330075E6002B14D04B07C0081843FA
:10AC60008023C9081B03194207D0FC081C4204D1E9
:10AC70007907D0080843E14621004C46420FC9003D
:10AC80001143C000684DB9E61D0000220023C0E654
:10AC9000002D5BD10D00054300D1E2E65D1C00D123
:10ACA000B0E0614DAE421FD0DB43382B71DC1F2B6F
:10ACB00000DD96E020250F00ED1AAF40B9460700F1
:10ACC000AA46DF404D463D432F005546A840D94097
:10ACD000451EA84188440743BF18974292415142FC
:10ACE000414435003AE6644635004146100085E6A9
:10ACF0000B000343002D00D063E6002BF5D0434644
:10AD0000134300D17AE687188742804107224144E5
:10AD1000404209183A400B0200D4D5E6434B0135B6
:10AD20001940C9E5380069E61E004746203EF74055
:10AD3000BC46202B04D04026F31A46469E403243A0
:10AD4000170063467A1E97411F4302E6364DAE4216
:10AD5000CAD080252D045B422943A6E70843411E43
:10AD60008841A6E6002B00D148E6871A4346B84240
:10AD7000B641CB1A76429E1B33024BD5171A434677
:10AD8000BA429241591A5242891A072264463A40FD
:10AD900092E501430F00791E8F419DE71C000F00D3
:10ADA000203CE740202B03D04024E31A994008437D
:10ADB000411E884138437CE60022002425E6171A0C
:10ADC0004346BA429241591A5242891A64463500A2
:10ADD00043E541461000144D10E680220024120382
:10ADE00080E61D000F00203DEF40BC46202B03D025
:10ADF0004025EB1A9940084307006346781E8741B7
:10AE00001F4369E7871897429B4141445B42C91839
:10AE10003500A3E53B003343CED0072231003A4052
:10AE200052E600231A00F4E5FF070000FFFF7FFF52
:10AE3000F0B55746DE464E464546E0B58346070028
:10AE40000E03480085B092461C00360B400DCD0F16
:10AE5000002800D19DE0954B984239D08023F60020
:10AE60001B041E43924A7B0F3343994694460300CA
:10AE70006344009300230026FF00029323031B0B6F
:10AE800098466300E40F52465B0D019400D1B3E095
:10AE900086498B4200D19EE04246D10080221204B6
:10AEA0000A435146490F11438B46814952468C460D
:10AEB00000996344CB1A0021D20000932B00634019
:10AEC0009A460F2E00D905E17A4BB6009B599F4652
:10AED0005B463343994600D0B8E00223082600279A
:10AEE00000900293CAE7CB463A0002990195019B74
:10AEF0009A46022927D0032900D180E2012944D0B3
:10AF00006D49009B8C4663441C00002C38DD5307C0
:10AF100000D013E2D2085B46DB0109D55946674BE6
:10AF200019408B468021C9008C46009B63441C005D
:10AF3000634B9C4207DC5B4664055F075B0217437B
:10AF40001B0B620D02E000230027584A00211B035F
:10AF50001C0B0B0D1B05234314055A4A38001340E4
:10AF60001C4353466400DB0764081C43210005B002
:10AF70003CBC90469946A246AB46F0BD01225242E7
:10AF800001231B1B382B00DCADE10022002300272E
:10AF9000DCE75B46334399465ED0002E00D18AE160
:10AFA000300001F0E7F903000B3B1C2B00DD7BE1D7
:10AFB0001D22D31A5A460100DA4008398E40130088
:10AFC0005F46334399468F403F4B00261B1A009340
:10AFD0000023029352E7414653460B433B499B46AD
:10AFE0008C46009B634400935B46002B3BD10223BD
:10AFF00000221E43022161E7434613439B4637D09C
:10B000004346002B00D162E1404601F0B3F9030052
:10B010000B3B1C2B00DD53E102004146083A9140F6
:10B0200088461D21CB1A5146D9400B0041460B439F
:10B030009B46534693401A00009B25499C4660441A
:10B0400003008C4663440093002137E70323B14695
:10B0500000900C26029311E700230093013304268D
:10B06000002702930AE70323C3461E43032125E773
:10B0700001331E430022012120E700239A4680234A
:10B0800000271B03094A61E7802349461B03194235
:10B0900000D1E2E05946194200D0DEE00B431B0329
:10B0A00017001B0BA246014A50E7C046FF070000ED
:10B0B00001FCFFFFE0F30000FF030000FFFFFFFEC5
:10B0C000FE070000FFFF0F800DFCFFFF01F8FFFFF0
:10B0D000F3030000D94500D9CBE000D1C6E03C0025
:10B0E00048460027009B013B00935B46160E1B025F
:10B0F0001E431302984633041B0C9946310C0191F0
:10B10000FFF798F84A4642430B04210C0500194307
:10B110008A4207D98919013D8E4203D88A4201D952
:10B12000851E8919881A0199FFF784F809048C464D
:10B130004A46210464464243090C030021438A42E3
:10B1400004D98919013B8E4200D8F1E02D041D433A
:10B15000AB464346891A4246280C12041D0C5B4636
:10B16000140C22001B041B0C5A4303946B434443EE
:10B17000029568431B19150CEB189C4203D98024D7
:10B180006402A44660441C0C15041B042D0C2018FA
:10B190005D19814277D373D00C1AA24A7D1BAF424E
:10B1A000BF419446009B7F426344E01B1C008642E3
:10B1B00000D1DBE00199FFF73DF84A4642430B041A
:10B1C000290C070019438A4207D98919013F8E4289
:10B1D00003D88A4201D9871E8919881A0199FFF775
:10B1E00029F809044A46894629044D464243090C78
:10B1F000030029438A4207D98919013B8E4203D8AB
:10B200008A4201D9831E89193F04891A3A00039F93
:10B210001A43380013041B0C584381460298150C3E
:10B220006F43434345434846000C8446DB1963445F
:10B230009F4203D9802040028446654448461F0C43
:10B2400000041B04000C7D191818A94200D284E0E8
:10B2500000D17FE001231A4357E680234A461B03AF
:10B2600013431B031B0BAA466F4A6FE6BA4200D971
:10B2700035E74B46DC0758087B081C43FF0734E7DB
:10B280000024AF4289D247444745A4415B4664420B
:10B29000A4196418013BA6421ED2A0426DD800D169
:10B2A000B6E0241A9B4678E703005A46283B9A40AA
:10B2B0000027914688E6584601F05CF8203072E697
:10B2C00003005246283B9A4093460022B4E650467B
:10B2D00001F050F820309AE6A642E2D1B845DCD918
:10B2E000341A9B4659E71F2B65DC504C0099A44645
:10B2F0005C46614408008C4011008240D940501ED9
:10B3000082410C4314435A46DA401300620709D0C5
:10B310000F222240042A05D02200141D94428941A4
:10B3200049425B181A0262D50122002300270DE66C
:10B330008A4200D80AE7831E891907E70F231340C2
:10B34000042B00D1E6E5171D9742924153429B44DE
:10B35000FA08E0E5002800D1D7E57118531EB14284
:10B3600027D3A94215D358D01A0073E7002B00DC6D
:10B3700004E6012300229B44CDE5022347444745D0
:10B3800089415B429C46494289190C19E344241ABD
:10B3900003E743465F0047459B41B8465B429E1921
:10B3A000023A8919A94200D054E7404500D051E73C
:10B3B000ABE51A00F6E71F215F4649420C1BE74048
:10B3C000202B07D01A49009B8C46634418005B462B
:10B3D00083401A43501E82413A43072700231740F7
:10B3E00009D00F21002311401400042995D1220017
:10B3F0005F075B021B0BD20817430022A6E58023E0
:10B4000059461B030B431B0317001B0B064A9DE504
:10B41000BD42B2D89B460024BFE68045B9D31A008E
:10B42000C3E7C046FF030000FF0700001E04000042
:10B430003E040000F0B54F464646D6468446C0B5A9
:10B440008046194E18030F034D00000B5C00824626
:10B450003F0B6D0DC90F9146640DDB0F0120B54206
:10B460000AD0B44203D0A54201D157450CD01CBC30
:10B4700090469946A246F0BD66463E43F7D1AC429F
:10B48000F5D154461443F2D10120C845EFD1994279
:10B4900007D0002DEBD163461F433800471EB8414B
:10B4A000E5E70020E3E7C046FF070000F0B54F46A0
:10B4B0004646D6464D00C0B50E03C90F8A462C49F4
:10B4C0001F035C008046360B6D0D91463F0B640DEB
:10B4D000DB0F8D421ED08C4216D0002D1ED1304382
:10B4E0008446002C01D13A4323D06246002A1AD068
:10B4F0009A4529D0514602200139084001381CBC28
:10B5000090469946A246F0BD39001143E5D002208D
:10B510004042F4E73043FAD1AC420FD0002C0FD1B7
:10B520003A43E7D00CE00122013B9343180001307D
:10B53000E5E763460020002BE1D0DBE73A43E6D1A4
:10B540009A45D7D1A542D5DCA54205DBBE42D1D86C
:10B5500008D00020BE42D2D2504601230138984381
:10B560000130CCE7C845C5D80020C845F4D3C6E7AC
:10B57000FF070000F0B54F464646D6464D00C0B521
:10B580000E03C90F8A462E491F035C008046360B06
:10B590006D0D91463F0B640DDB0F8D4218D08C4230
:10B5A00011D0002D18D130438446002C1ED13A43CF
:10B5B0001CD163460020002B30D0514602200139B7
:10B5C000084001382AE039001143EAD0022025E082
:10B5D0003043FBD1AC4226D0002C26D13A4324D1B3
:10B5E0005146022001390840013817E06246002A1E
:10B5F0000FD09A45E1D1A54205DBBE42DDD819D076
:10B600000020BE420AD2504601230138984301303F
:10B6100004E00122013B9343180001301CBC90461A
:10B620009946A246F0BD3A43D0D19A45C5D1A5422C
:10B63000C3DCE0E7C845C0D80020C845E3D3EDE748
:10B64000FF070000F0B55746DE464E464546E0B5DA
:10B65000834606000F03480087B092461D003F0B4B
:10B66000400DCC0F002800D16FE0DE4B984238D05F
:10B670008023FF001B041F43730F3B430193DA4BEE
:10B680000027994600239B46F60081442B0369005E
:10B690001B0B52469846490DED0F002900D185E05D
:10B6A000D04B994200D173E04346DA0080231B045B
:10B6B00013435246CC48520F84461343524600204F
:10B6C0006144D20089442100694000918C460121E7
:10B6D00049448A460F2F00D990E0C449BF00CF5992
:10B6E000BF465B463B43019300D06AE10223082733
:10B6F000002681469B46C9E732005846019B6146B9
:10B700000091022800D175E0032800D1FEE1012854
:10B7100000D02CE100230027002600253F032A0D3E
:10B720003F0BB34812053A4302401B051343009AEE
:10B730005B00D1075B080B433000190007B03CBC2D
:10B7400090469946A246AB46F0BD5B463B4301930B
:10B7500000D12FE1002F00D1A5E1380000F00AFE52
:10B7600003000B3B1C2B00DD96E11D22D31A5A4629
:10B770000100DA405E4608398F4013008E403B439B
:10B7800001939C4B00271B1A994600239B467DE79B
:10B79000414653460B4393498C46E144002B00D06D
:10B7A0001AE102220220174300228CE7134300D142
:10B7B0000DE14346002B00D181E1404600F0DAFD67
:10B7C00002000B3A1C2A00DD72E1010043460839F1
:10B7D0008B4098461D239A1A5346D3401A0043467D
:10B7E000134352468A404946081A82498946814491
:10B7F000002068E77B4B002700268EE7140C12041C
:10B80000120C1100370C3604350C794328008C4695
:10B810002E0060436044834656432100300C80462E
:10B820005846794340440291844506D98846802190
:10B8300049028C46E044414602913604010C360C24
:10B8400000048B4681191E0C1B041B0C039119006C
:10B8500079438C46280075436544A8465843050C37
:10B8600045447743A94203D9802149028C46674465
:10B87000290C8C4639000004000C2D042D1861445D
:10B88000AB4405915946049101990F043F0C080CF3
:10B89000390051434243904602008C46090C8B46C6
:10B8A00062437C4344445C44A04503D9802149025F
:10B8B00088464244210C884661460904090C8C469E
:10B8C00039005943434370437E430F0CF618240458
:10B8D000BE19644442448C46B34203D980235B02C0
:10B8E00098464044029B61469846049B3704434473
:10B8F0009B46AB45AD416B420D0405992D0C8C4622
:10B900007F196744FD18A8465D462D19A542A4413C
:10B9100093466442A446C344DC448F42BF419845E9
:10B920009B4193459241A445A4415B427F421F4302
:10B93000360C52426442BF192243BF18624638187F
:10B940004302D20D039913436A020A43501E8241F7
:10B950006146ED0D2A434E023243D90100D4B3E0D3
:10B960000126500832400243DE0732435B08224C76
:10B970005444002C62DD510709D00F2010400428E8
:10B9800005D0101D9042924152429B180200D901ED
:10B9900004D580241948E4000340544418488442E4
:10B9A00000DD27E75E075B02D2081F0B6305164325
:10B9B0005B0DB2E6002399460133042700269B461F
:10B9C00064E60323019781460C279B465EE601222D
:10B9D00001201743002276E6032303201F4343463A
:10B9E00071E6C046FF07000001FCFFFF20F40000E5
:10B9F000FFFF0F800DFCFFFFFF030000FFFFFFFEB6
:10BA0000FE0700000023802700933F030026434BDE
:10BA100083E6019B3200A446584670E6AC466EE6CB
:10BA2000802701993F0339422DD03B422BD11F4340
:10BA30003F033F0B00951600384B6EE601252D1B8A
:10BA4000382D00DD66E61F2D40DC35481C005044D3
:10BA5000160082408440EE40501E8241344314431D
:10BA6000EB40620709D00F222240042A05D02200B1
:10BA7000141D9442804140421B181A023ED50123F6
:10BA80000027002649E68027019B3F031F433F0311
:10BA90003F0B0094214B40E603005A46283B9A4056
:10BAA000002601926DE6584600F064FC203057E60F
:10BAB00003005246283B9A401300002293E650466A
:10BAC00000F058FC20307BE6CA4650E71F201E00DD
:10BAD0004042041BE640202D03D0124C5444A340A6
:10BAE0001A43501E8241324307260027164009D0D0
:10BAF0000F200023104014000428B9D122005E0753
:10BB00005B021F0BD2081643002306E680273F0383
:10BB10001F433F033F0B1600004BFEE5FF070000ED
:10BB20001E0400003E040000F8B557464E46454648
:10BB3000DE460C000903E0B5490A460F5F003143B9
:10BB40001E03DB0F760A9B46530F3343C84E650036
:10BB5000C000E40FD2006D0DA24681467F0D9C46C9
:10BB60009046B74200D1B9E05B46012673409B4640
:10BB7000EE1BA34500D183E0002E63DD002F00D033
:10BB8000B1E06346134300D123E1731E002B00D0C4
:10BB9000BAE1861A6346B04280410125C91A404283
:10BBA000091A0B0200D447E149024B0A9846434662
:10BBB000002B00D189E1404600F0DCFB0300083B8C
:10BBC0001F2B00DD7CE120223000D21A4146D040FC
:10BBD000994002009E400A439D4200DD6AE15D1BE0
:10BBE0006B1C1F2B00DD94E1202110003500C91AC9
:10BBF0008E40DA408840DD40711E8E4111000722E0
:10BC00002843002506433240002A09D00F23334041
:10BC1000042B05D0331DB342B641764289191E006C
:10BC20000B0200D43DE26A1C914B55056D0D9A4202
:10BC300000D119E18F4AF6080A40570752023743EC
:10BC4000120B9BE0002E00D0C5E06E1C7605760D31
:10BC5000012E00DC48E16746861ACB1BB042BF418B
:10BC60007F42B8461F004346FF1A3B00B8461B02FE
:10BC700000D55FE137439AD100220024002579E006
:10BC8000002E00DCFAE0002F00D18DE0784B9D42C1
:10BC900067D0802367461B041F43BC46382E00DC58
:10BCA00052E1634613435A1E93411E188642804157
:10BCB000404209180B0200D4BEE06D4B01359D4295
:10BCC00000D1D2E06B4A73080A4001210E401E43A6
:10BCD0005108D30707221E43324095E71E00164342
:10BCE00000D045E740E7624B9D423AD0802367464B
:10BCF0001B041F43BC46382E00DDEBE01F2E00DC8A
:10BD00003AE133006746203BDF403B00202E05D060
:10BD10004027BF1B6646BE40324390464646721ED1
:10BD200096413343DAE0002B00D114E2634613431B
:10BD300000D168E180234E07C008C9081B030643F1
:10BD4000194208D06046C008184204D16346010079
:10BD5000D2085E071643F3009946C900720F444D9E
:10BD600011434B46DE08424B4F073743CA089D42FA
:10BD700000D16EE012036D05120B6D0D0021120350
:10BD8000130B0A0D12051A433B4B2D0513402B4391
:10BD90005B00E4075B082343380019003CBC904675
:10BDA0009946A246AB46F8BD6346134311D0731EB5
:10BDB000002B00D007E18618864280416144404252
:10BDC000091801250B0237D502257BE73E006146A5
:10BDD00091463500C5E75C46002D00D0E1E00B0040
:10BDE0000343F3D0731C00D1ACE1214B9F4200D13F
:10BDF0003AE1F343382B00DD6FE11F2B00DD8CE1CE
:10BE000020250E00ED1AAE40B0460600AA46DE40E0
:10BE1000454635432E005546D940A8406346451E49
:10BE2000A8415B1A9C463043161AB24292416346BF
:10BE30005242991A3D00B4E607223240002A00D04F
:10BE4000E4E60B4BF6084F073743CA089D4200D083
:10BE500090E73B00134300D1A6E180231B031A4364
:10BE60001203120B024D89E715000022002785E717
:10BE7000FF070000FFFF7FFFFFFF0F80002E00D0B5
:10BE8000C7E06B1C5E05760D012E00DCF0E0C84DAE
:10BE9000AB4200D1B9E085180A008542894162446D
:10BEA000494251180722CE076D082E4349083240F7
:10BEB0001D00A9E6BF49ED1A114007223240A3E652
:10BEC000320028388240002686E6300000F052FA20
:10BED000203073E6634613435A1E9341C61AB0429C
:10BEE00080414042091A5CE60E006746064317434C
:10BEF000002D5ED1002E00D0F3E0002F00D11EE116
:10BF00005C46614691462CE7A94FBE427BD01E009D
:10BF1000F1E610001F3DE840202B03D04021CB1A52
:10BF20009A401643731E9E41072206433240002169
:10BF3000002583E7161A6346B2428041591A4042EF
:10BF40000B1A98465C4632E61F2E00DDABE0202738
:10BF5000BB1B9A4663465746BB40994613004F4663
:10BF6000F3401F433B005746BA40571EBA411343A4
:10BF70006246F240891898E62027BB1B9A46634622
:10BF80005746BB40994613004F46F3401F433B00C2
:10BF90005746BA40571EBA4113436246F240891AC7
:10BFA0009CE7834B9F425FD080252D047342294339
:10BFB00020E7002E0CD1002F00D1D0E05C46614676
:10BFC00091467B4DCDE67A4FBE421CD01E0065E601
:10BFD000002F18D0C0084E0706438020C908000370
:10BFE000014208D06346DC08044204D12100DA464D
:10BFF000D2085E071643F300994601245346C90050
:10C00000720F11431C406A4DABE61D000022002751
:10C01000B4E6002D59D10B00034300D1D6E6731CC2
:10C0200000D1B2E0624B9F421ED0F343382B6FDC4D
:10C030001F2B00DD97E020250E00ED1AAE40B04624
:10C040000600AA46DE40454635432E005546A84028
:10C05000D940451EA8418C440643B61896429241E9
:10C06000514261443D0025E63D006146914678E637
:10C070000B000343002D00D055E6002BF5D063469E
:10C08000134300D16DE686188642804161444042E8
:10C09000091800220B0200D4D0E6464B01351940A6
:10C0A000B2E5B1465DE633006746203BDF403B002A
:10C0B000202E05D04027BF1B6646BE403243904627
:10C0C0004646721E96413343EFE5394B9F42CBD033
:10C0D00080252D0473422943A8E70843411E884167
:10C0E000A2E6002F00D13CE66346861ACF1AB04282
:10C0F0009B415B42FB1A98461B024ED5161A6346BB
:10C10000B2429241591A5242891A5C4600227BE59A
:10C1100001430E00711E8E419FE71D000E00203D61
:10C12000EE40B046202B04D04025EB1A994008433E
:10C13000814648464346411E8841184374E6002222
:10C14000002417E6161A6346B2429241591A524227
:10C15000891A3D0025E561469146154D01E680228C
:10C160000024120379E61D000E00203DEE40B0468B
:10C17000202B04D04025EB1A9940084381464E46B7
:10C180004346711E8E411E4367E7861896429B41C7
:10C1900061445B42C9183D008CE547463743CED029
:10C1A00007224146324049E600273A00E6E5C0460C
:10C1B000FF070000FFFF7FFF70B50C4E0D031C034F
:10C1C00049005B002D0B490D240B5B0DB14208D0DB
:10C1D000064900208B4203D114432000441EA04195
:10C1E00070BD05430120002DFAD1F1E7FF070000E3
:10C1F00030B5144D0A034B00120B5B0DC90F002420
:10C20000AB4211DD104CA34210DC802464032243B6
:10C210000E4CE41A1F2C0CDD0D48C31ADA40130033
:10C220005C42002900D11C00200030BD094BCC1815
:10C23000FAE7094DE040AC4663449A4013000343DB
:10C24000EEE7C046FE0300001D04000033040000BA
:10C2500013040000FFFFFF7FEDFBFFFF70B5002818
:10C260002DD0C317C5185D40C40F280000F082F818
:10C27000154B1B1A5B055B0D0A2815DD0B38854035
:10C2800000222D032D0B002110002D030A0D2D0B74
:10C2900012052A430D4D1B052A4013435B00E4079A
:10C2A0005B082343190070BD02002900153291403C
:10C2B0000A000B21081AC5402D032D0BE3E70024CB
:10C2C000002300250022DEE71E040000FFFF0F8090
:10C2D0004100090E4B1C70B5DBB24602750AC40F53
:10C2E000012B14DDE0239B006D07360BCB180021DA
:10C2F0000A0D280012051C4D32435B052A405B08DD
:10C3000013435B00E4075B082343190070BD002959
:10C3100014D1002D1ED0280000F02CF80A281CDCB7
:10C320000B232A001B1ADA40030015339D400F4BE4
:10C3300012031B1A5B05160B5B0DD8E7002D06D008
:10C34000320B802636036D071643094BCFE7084BA7
:10C350000026CCE700230026C9E703002A000B3B98
:10C360009A400025E3E7C046FFFF0F8089030000E5
:10C37000FF0700001C2101231B04984201D3000C7D
:10C3800010391B0A984201D3000A08391B09984248
:10C3900001D30009043902A2105C40187047C0465E
:10C3A000040302020101010100000000000000007E
:10C3B00030B51C00094B05001B6885B0D868084BD8
:10C3C000002A01D1074B1A000292019300912B0021
:10C3D0002200054900F026F800F0A6FD8C000020A0
:10C3E00060F40000A2E000006DF40000014B18684A
:10C3F0007047C0468C000020084B10B50400002B8D
:10C4000002D0002100E000BF054B1868836A002BB2
:10C4100000D09847200001F05DFBC04600000000FE
:10C420009CF400000EB403B5010003AB044804CB38
:10C430000068019300F076F802B008BC03B018471A
:10C440008C00002070B500260C4D0D4C641BA41010
:10C45000A64209D1002601F03FFB0A4D0A4C641B9D
:10C46000A410A64205D170BDB300EB589847013621
:10C47000EEE7B300EB5898470136F2E75C02002084
:10C480005C0200205C0200206C020020002310B53A
:10C490009A4200D110BDCC5CC4540133F8E710B50A
:10C4A000884202D98B18984203D3002307E08B5CA3
:10C4B0008354013AFBD210BDCC5CC45401339A4280
:10C4C000FAD1F8E703001218934200D170471970AF
:10C4D0000133F9E7936810B5013B9360002B04DA50
:10C4E0009469A34207DB0A2905D01368581C106021
:10C4F0001970080010BD00F04BFC0100F9E7F8B519
:10C5000006000F001400D518AC4201D1002007E04E
:10C5100021783A003000FFF7DDFF0134431CF3D1EE
:10C52000F8BD0000F0B59FB002900F001600059313
:10C53000002805D083690493002B01D100F0F4FD9D
:10C540007B4B9F425BD1029B5F68BB891B0762D517
:10C550003B69002B5FD0002306AC63612033637618
:10C560001033A37635002B78002B01D0252B5CD11E
:10C57000AB1B04930CD0320039000298FFF7BFFFC9
:10C58000431C00D1C4E06269049B94466344636128
:10C590002B78002B00D1BBE00122002352426260C5
:10C5A00002A9543252186E1C2360E360A36013701A
:10C5B000A365317805225F4800F0D4FE751C002881
:10C5C00035D12268D30604D5532302A95B18202154
:10C5D0001970130704D5532302A95B182B21197076
:10C5E00033782A2B2CD0350000210A20E3682A78E2
:10C5F0006E1C303A092A64D900292ED026E04E4B11
:10C600009F4202D1029B9F689FE74C4B9F429CD167
:10C61000029BDF6899E73900029800F00FFC0028C0
:10C6200099D0012040421FB0F0BD01359BE7414B3E
:10C630002268C01A01238340134323602E00B8E709
:10C64000059B191D1B680591002B01DB099304E074
:10C650005B42E3600223134323602B782E2B0AD125
:10C660006B782A2B35D1059B02351A1D1B68059264
:10C67000002B2BDB0793324E29780322300000F089
:10C6800071FE002806D04023801B834022680135BC
:10C6900013432360297806222A486E1C217600F075
:10C6A00061FE00283AD0284B002B25D10722059B9C
:10C6B00007339343083305936369039A9B186361B7
:10C6C00050E7434301219B18350090E701235B426B
:10C6D000D0E700230A201A000135636029786E1C18
:10C6E0003039092903D9002BC5D00792C3E742434B
:10C6F000012352183500F1E705AB00933A00134BC4
:10C700002100029800E000BF0390039B0133D3D1C6
:10C71000BB895B0600D584E70B9884E705AB0093E3
:10C720003A000A4B2100029800F080F8ECE7C0467E
:10C73000F4F40000A0F4000014F50000D4F40000AC
:10C74000A6F40000AAF4000000000000FFC40000EE
:10C75000F7B5150001938A680B6900900C009342AD
:10C7600000DA130022002B6043321278002A01D035
:10C7700001332B6023689B0602D52B6802332B60A4
:10C78000062723681F4027D0230043331B785A1EF7
:10C7900093412268920630D42200019943320098D6
:10C7A000089EB047431C25D0062320682A68E1680C
:10C7B00003400025042B03D18D1AEB43DB171D40EA
:10C7C000A3682269934201DD9B1AED180027BD4240
:10C7D00020D1002010E00137E3682A689B1ABB4291
:10C7E000D2DD22000123193201990098089EB0473A
:10C7F000431CF0D101204042FEBD3020E1184331FE
:10C80000087021005A1C45310978A21843320233BE
:10C810001170C1E7220001231A3201990098089E85
:10C82000B047431CE6D00137D1E70000F0B589B02E
:10C8300004920A0043320593039002920A7E0C0090
:10C840000E9B6E2A00D186E01FD8632A33D008D809
:10C85000002A00D18CE0582A4DD0250042352A709C
:10C8600030E0642A01D0692AF7D1196825680A1DC9
:10C87000280629D508681A60002803DA2D23029AB1
:10C88000404213706B4E0A274FE0732A74D008D8C9
:10C890006F2A1FD0702AE0D1202209680A43226043
:10C8A00003E0752A16D0782AD7D1220078214532A4
:10C8B0001170614E22E025001A684235111D196081
:10C8C00013682B70012365E008681A606906D3D5E8
:10C8D00000B2D1E719682568081D186008682E069F
:10C8E00005D5544E08276F2A1BD00A2719E06D067C
:10C8F000F7D580B2F5E745314E4E0A7018682268C8
:10C90000011D00681960150621D5D30702D5202323
:10C910001A4322601027002803D1202322689A435B
:10C9200022602300002243331A706368A360002B47
:10C9300058DB0422216891432160002854D1029DD4
:10C94000002B5AD02500337842352B7055E0550620
:10C95000DBD580B2D9E71A680D68101D49691860E7
:10C9600013682E0601D5196002E06D06FBD519800B
:10C970000023029D23614FE01A68111D196015689C
:10C9800000216268280000F0EDFC002801D0401B67
:10C990006060636823610023029A13703CE023699E
:10C9A0002A0004990398059DA847431C3ED023689C
:10C9B0009B0715D4079BE068984239DA180037E0E6
:10C9C00022000123193204990398059EB047431CA5
:10C9D0002CD00135E368079A9B1AAB42F0DCE9E7FB
:10C9E0000025F7E70028ADD0029D3900FDF722FCB5
:10C9F000735C013D2B700028F7D1082F09D1236803
:10CA0000DB0706D563682269934202DC3023013DCF
:10CA10002B70029B5B1B2361059B07AA00932100DF
:10CA2000049B0398FFF794FE431CB8D101204042B9
:10CA300009B0F0BDB1F40000C2F400000D4B70B5B8
:10CA40001C680500A36B002B0FD1182000F06EFCB2
:10CA5000094BA0630360094B01224360084B8360CC
:10CA60000B2383810023026143610022A36B1D61BC
:10CA70005A6170BD8C0000200E33CDAB34126DE6D0
:10CA8000ECDE0500124B10B51C68A36B002B0FD118
:10CA9000182000F04BFC0F4BA06303600E4B0122EB
:10CAA00043600E4B83600B2383810023026143614B
:10CAB000A46B0B4A206961690A4BFDF7F7FC012260
:10CAC000002380185941206161614800400810BD71
:10CAD0008C0000200E33CDAB34126DE6ECDE050089
:10CAE0002D7F954C2DF451580CB430B5164B9DB09C
:10CAF0000C1E1D6808DA8B2301202B6040421DB0FC
:10CB000030BC08BC02B01847822302A99B008B816D
:10CB10000023029008619C4200D0631E8B604B6131
:10CB200001235B42CB81209A21AB2800019300F0C6
:10CB300055FD431C01DA8B232B60002CDFD0002332
:10CB4000029A1370DBE7C0468C0000200EB400B5DB
:10CB50000B499CB01DAB02900690079104910948C7
:10CB6000094904CB0591006802A9019300F036FD44
:10CB70000023029A13701CB008BC03B01847C046CB
:10CB8000FFFFFF7F8C0000200802FFFF020010B5AE
:10CB90001378541C002B05D1CC5CD4540133002CE9
:10CBA000FAD110BD2200F3E7C9B20378002B04D0FC
:10CBB0008B4200D170470130F7E74B42594149425F
:10CBC0000840F7E702780B78002A03D001300131E2
:10CBD0009A42F7D0D01A70470023C25C0133002A72
:10CBE000FBD1581E7047002330B59A420AD0013A53
:10CBF000C45CCD5CAC4204D1934202D00133002C22
:10CC0000F6D1631B180030BD30B50500002A00D1F5
:10CC100030BD0C78013A6B1C2C700131002C05D111
:10CC20009A189A42F4D01C700133FAE71D00EDE720
:10CC300010B50378002B0FD10B785A4253415B4259
:10CC4000184010BD0023CA5C002AFAD0C45C94428C
:10CC500001D10133F7E701300378002BF2D118003E
:10CC6000EFE70000F0B51F000E0087B005900191BE
:10CC700002920C98347800F0EAFA082200194378FE
:10CC8000751C134036D12D2C36D1B51C7478012675
:10CC9000002F62D0102F09D1302C07D120222B7801
:10CCA0009343582B54D110276C7802352D4B390003
:10CCB000F31818000393FDF7BDFA04910121002336
:10CCC000494202008C4618002100303909291AD83F
:10CCD0000C00A74223DD591C09D06346824206D3CB
:10CCE00002D10499A14202DB0123784320182C7859
:10CCF0000135E9E72E00BCE72B2C01D01E00C7E769
:10CD0000B51C7478FAE721004139192901D8373C5C
:10CD1000DFE721006139192901D8573CD9E75A1CAE
:10CD200008D1059A23331360029B0398002B09D185
:10CD300007B0F0BD002E00D04042029A002AF7D082
:10CD4000002B01D06B1E0193029B019A1A60EFE742
:10CD50003024002FAAD10827A8E7302C9ED00A271C
:10CD6000A4E7C046FFFFFF7F37B51300064A050062
:10CD70001068046A002C00D1044C0A0000942900B9
:10CD8000FFF770FF3EBDC0468C000020F000002081
:10CD9000F8B505000E001400002804D08369002BAC
:10CDA00001D100F0C1F9224B9C422DD16C68A369DE
:10CDB000A360A3891B0731D52369002B2ED02368DC
:10CDC0002269F7B2981A6369F6B2834205DC210042
:10CDD000280000F03BF9002826D1A3680130013B70
:10CDE000A36023685A1C22601F706369834204D0C9
:10CDF000A389DB071AD50A2E18D12100280000F0DC
:10CE000025F9002812D00FE00A4B9C4201D1AC68F2
:10CE1000CDE7094B9C42CAD1EC68C8E72100280045
:10CE200000F00CF80028CAD0012676423000F8BD88
:10CE3000F4F4000014F50000D4F40000364B70B593
:10CE40001D6806000C00002D05D0AB69002B02D137
:10CE5000280000F069F9314B9C420FD16C680C231B
:10CE6000E25E93B219072DD4D90611D4092301200B
:10CE7000336037331343A381404270BD284B9C423B
:10CE800001D1AC68EBE7274B9C42E8D1EC68E6E7C0
:10CE90005B0713D5616B002908D023004433994206
:10CEA00002D0300000F06AFA002363632422A389D1
:10CEB0009343A38100236360236923600823A2892D
:10CEC0001343A3812369002B0BD1A0218022A389C6
:10CED000890092000B40934203D02100300000F003
:10CEE000E1F90123A289134011D00023A3606369F3
:10CEF0005B42A361002023698342BED10C23E25E22
:10CF00001306BAD540231343A3810138B5E792072E
:10CF100000D46369A360EDE78C000020F4F4000006
:10CF200014F50000D4F4000010B5062000F090FCC9
:10CF3000012000F0CFFD0000F7B58A8905000C0044
:10CF4000130760D44B68002B04DC0B6C002B01DC56
:10CF50000020FEBDE76A002FFAD000232E682B6068
:10CF600080235B01216A1A4034D0606DA3895B077E
:10CF700006D56368C01A636B002B01D0236CC01AFE
:10CF80000200216A00232800E76AB847A189431CF0
:10CF900006D12B681D2B30D82B4ADA40D3072CD56D
:10CFA0000023636023692360CB0405D5431C02D1B1
:10CFB0002B68002B00D16065616B2E600029C7D003
:10CFC00023004433994202D0280000F0D7F9002012
:10CFD0006063BEE701232800B847431CC6D12B6815
:10CFE000002BC3D01D2B01D0162B01D12E60AFE733
:10CFF0004023A2891343A381ABE740230B430120C5
:10D00000A3814042A5E70F69002FA1D00B680F60F4
:10D01000DB1B01930023920700D14B69A360019BA6
:10D02000002B00DC94E7019B3A00216A2800A66AE5
:10D03000B047002803DC4023A2891343DFE7019BAC
:10D040003F181B1A0193EAE7010040200B6970B5F5
:10D0500005000C00002B01D1002070BD002804D079
:10D060008369002B01D100F05FF80B4B9C4209D182
:10D070006C680C22A35E002BEED021002800FFF785
:10D080005BFFEAE7054B9C4201D1AC68F1E7044B3A
:10D090009C42EED1EC68ECE7F4F4000014F50000DB
:10D0A000D4F40000002310B50400036043608360E3
:10D0B00081814366C2810361436183611900082253
:10D0C0005C30FFF7FFF9054B24626362044BA362F7
:10D0D000044BE362044B236310BDC04691D80000AB
:10D0E000B9D80000F1D800001DD9000010B50249E0
:10D0F00000F08CF810BDC0464DD0000070B568251A
:10D100004A1E55430E002900743100F081F9041EB7
:10D1100008D000212A00016046600C30A06068320F
:10D12000FFF7D0F9200070BD836913B50400002B10
:10D1300028D18364C3640365134B144A1B6882625D
:10D140000193984201D101238361200000F020F86F
:10D150006060200000F01CF8A060200000F018F8CB
:10D160000022E06004216068FFF79CFF0122092192
:10D17000A068FFF797FF02221221E068FFF792FFF5
:10D180000123A36113BDC0469CF40000EDD0000054
:10D19000F8B51C4B07001E68B369002B02D13000A4
:10D1A000FFF7C2FF4836B4687368013B04D53368A3
:10D1B000002B07D03668F6E70C22A55E002D0DD0B7
:10D1C0006834F2E704213800FFF798FF3060002848
:10D1D000F0D10C2304003B602000F8BD20000A4B76
:10D1E000656625606560A560E36025616561A56190
:10D1F000082229005C30FFF765F96563A563A56423
:10D20000E564E9E79CF400000100FFFFF7B50400C6
:10D210000700002601914834002C01D13000FEBDEA
:10D220006368A5680093009B013B009301D52468C7
:10D23000F2E7AB89012B08D90E22AB5E013304D093
:10D2400029003800019B984706436835EBE7EC302E
:10D250000068704770B50E001D000E23C95E96B0C1
:10D260001400002907DA00232B60B3891B0611D4B0
:10D270008023DB000FE06A4600F088FB0028F2DB29
:10D28000F022019B12021340054A9B185A42534157
:10D290002B60EDE740230020236016B070BDC04630
:10D2A00000E0FFFFF7B502268B8905000C00334232
:10D2B00006D0230047332360236101236361F7BD58
:10D2C00001AB6A46FFF7C6FF00990700280000F08F
:10D2D0009FF8002808D10C22A35E9A05EFD4032200
:10D2E00093431E43A681E4E70F4BAB628023A289E0
:10D2F00020601343A381009B20616361019B002B8D
:10D300000DD00E23E15E280000F052FB002806D06D
:10D310000322A38993431A0001231343A381A08905
:10D320003843A081CBE7C046EDD0000010B5034BD9
:10D330000100186800F06CF810BDC0468C00002099
:10D3400082B0002900D101A9101E06D0002B06D002
:10D3500013780B601078431E984102B0704702208A
:10D360004042FAE7C9B28218904201D100207047CA
:10D3700003788B42FBD00130F6E7000070B5050062
:10D38000002910D00C1F2368002B00DAE4182800B5
:10D3900000F034FB1D4A1368002B05D16360146054
:10D3A000280000F02CFB70BDA34209D92168601849
:10D3B0008342F3D118685B6841182160EEE71300DF
:10D3C0005A68002A01D0A242F9D919685818A04217
:10D3D0000BD120680918581819608242E0D11068F2
:10D3E0005268411819605A60DAE7A04202D90C234A
:10D3F0002B60D5E721686018824203D1106852681B
:10D400004118216062605C60CAE7C046341C00209D
:10D41000032370B5CD1C9D43083506000C2D1ED28C
:10D420000C25A9421DD8300000F0E8FA254A1468FE
:10D430002100002919D1244C2368002B03D130008E
:10D4400000F0CAF920602900300000F0C5F9431C43
:10D450002BD10C233000336000F0D1FA03E0002D13
:10D46000DFDA0C233360002070BD0B685B1B19D41E
:10D470000B2B03D90B60CC18256003E04B688C4262
:10D480000DD11360300000F0BAFA200007220B30F3
:10D49000231D9043C31AE7D05A42E250E4E7636089
:10D4A0000C00EFE70C004968C3E70323C41C9C434E
:10D4B000A042E1D0211A300000F08EF9431CDBD1EC
:10D4C000C7E7C046341C0020381C0020F8B5070010
:10D4D0000D001600002905D11100FFF799FF040087
:10D4E0002000F8BD002A03D1FFF748FF3400F7E71A
:10D4F00000F086FA2C00B042F2D231003800FFF77B
:10D5000087FF041EECD029003200FEF7BFFF290080
:10D510003800FFF733FFE3E7F0B58E6885B007000A
:10D520000C00039201939E423CD890238A89DB0031
:10D530001A4234D00325096923685B1A0293636990
:10D5400002985D43EB0F5D19019B6D1001331B18B1
:10D55000AB4200D91D00530532D529003800FFF732
:10D5600057FF061E09D10C233B6040230120A289EE
:10D5700040421343A38105B0F0BD029A2169FEF732
:10D5800085FFA389144A1A4080231343A381029B79
:10D590002661F61826606561019EED1AA560019B63
:10D5A0009E4200D9019E320003992068FEF777FF62
:10D5B000A36800209B1BA36023689E192660DAE7FE
:10D5C0002A003800FFF782FF061EE0D121693800EB
:10D5D000FFF7D4FEC7E7C0467FFBFFFFF0B59FB063
:10D5E000029005938B890F0016001B0611D50B695D
:10D5F000002B0ED14021FFF70BFF38603861002867
:10D6000005D10C23029A013813601FB0F0BD4023EE
:10D610007B61002306AC6361203363761033A3760D
:10D6200035002B78002B01D0252B46D1AB1B049362
:10D630000CD0320039000298FFF76EFF431C00D176
:10D64000AEE06269049B9446634463612B78002BCF
:10D6500000D1A5E0012200235242626002A95432A7
:10D6600052186E1C2360E360A3601370A3653178C9
:10D6700005225448FFF776FE751C00281FD122684A
:10D68000D30604D5532302A95B1820211970130770
:10D6900004D5532302A95B182B21197033782A2B48
:10D6A00016D0350000210A20E3682A786E1C303A33
:10D6B000092A4ED9002918D010E00135B1E7414BB5
:10D6C0002268C01A01238340134323602E00CEE753
:10D6D000059B191D1B680591002B01DB099304E0D4
:10D6E0005B42E3600223134323602B782E2B0AD185
:10D6F0006B782A2B35D1059B02351A1D1B680592C4
:10D70000002B2BDB0793304E297803223000FFF7E4
:10D7100029FE002806D04023801B83402268013563
:10D72000134323602978062228486E1C2176FFF7D0
:10D7300019FE00283CD0264B002B25D10722059B43
:10D7400007339343083305936369039A9B18636116
:10D7500066E7434301219B183500A6E701235B429E
:10D76000D0E700230A201A000135636029786E1C77
:10D770003039092903D9002BC5D00792C3E74243AA
:10D78000012352183500F1E705AB00933A00114B25
:10D790002100029800E000BF0390039B0133D3D126
:10D7A000BB890B985B0600D42FE7012040422CE791
:10D7B00005AB00933A00074B21000298FFF736F8BB
:10D7C000EAE7C046A0F40000A6F40000AAF40000B6
:10D7D0000000000019D50000002370B5064C0500BC
:10D7E0000800236000F060F9431C03D12368002B7C
:10D7F00000D02B6070BDC046C82F002070B504005B
:10D800000D001F2904D9162303600120404270BD7A
:10D81000436C002B04D08A009B181A68002A08D198
:10D82000200000F031F82A000100200000F01AF872
:10D83000EDE70020012AEAD0511C03D11623013064
:10D840002360E4E7002428001C6090472000DEE706
:10D8500010B5034B01001868FFF7D0FF10BDC0469C
:10D860008C000020002370B5064C05000800110054
:10D87000236000F001F9431C03D12368002B00D082
:10D880002B6070BDC82F002010B500F0E5F810BD6A
:10D8900070B50C000E25495F00F0BAF8002803DBD4
:10D8A000636D1B18636570BDA389024A1340A38191
:10D8B000F9E7C046FFEFFFFFF8B51F008B890500B1
:10D8C0000C001600DB0505D50E23C95E00220223DD
:10D8D00000F080F8A389054A28001340A381320094
:10D8E0000E23E15E3B0000F02BF8F8BDFFEFFFFFD9
:10D8F00070B50C000E25495F00F06CF8A389421C3E
:10D9000003D1054A1340A38170BD80225201134305
:10D91000A3816065F8E7C046FFEFFFFF10B50E2357
:10D92000C95E00F021F810BD0B1E04D0FF2A04D9F7
:10D930008A2303608B3B180070470A700123FAE7C3
:10D9400070B50500080011000022064C22601A0084
:10D9500000F0B8F8431C03D12368002B00D02B60E3
:10D9600070BDC046C82F0020002370B5064C0500CE
:10D970000800236000F060F8431C03D12368002BEB
:10D9800000D02B6070BDC046C82F0020002370B5AA
:10D99000064C050008001100236000F055F8431CF8
:10D9A00003D12368002B00D02B6070BDC82F00204E
:10D9B000002370B5064C05000800236000F054F801
:10D9C000431C03D12368002B00D02B6070BDC046E0
:10D9D000C82F002070B50500080011000022064C79
:10D9E00022601A0000F050F8431C03D12368002B7A
:10D9F00000D02B6070BDC046C82F00207047704714
:10DA00000B1F1B68181F002B01DA0B58C01870473A
:10DA100070B50500080011000022064C22601A00B3
:10DA200000F03AF8431C03D12368002B00D02B6090
:10DA300070BDC046C82F002058220120014B404233
:10DA40001A607047C82F002058220120014B404225
:10DA50001A607047C82F002058220120014B404215
:10DA60001A607047C82F00205822024B00201A600D
:10DA70007047C046C82F002058220120014B404269
:10DA80001A607047C82F002058220120014B4042E5
:10DA90001A607047C82F002058220120014B4042D5
:10DAA0001A607047C82F0020044A1368002B00D169
:10DAB000034B1818106018007047C0463C1C00202B
:10DAC000D02F002058220120014B40421A6070479D
:10DAD000C82F0020FEE7C046F8B5C046F8BC08BC19
:10DAE0009E467047F8B5C046F8BC08BC9E467047D5
:10DAF000646174610000000086DB0000EF0100003B
:10DB00008FDB0000E302000097DB0000090B000040
:10DB10009EDB0000450C0000A3DB000009050000AF
:10DB2000A9DB0000F5060000B4DB00005303000091
:10DB3000B9DB00009D0E0000C5DB00001F020000E5
:10DB4000CFDB0000D5090000DDDB000095060000FA
:10DB5000EADB000081080000F6DB0000550600004B
:10DB600072616E646F6D00616C6C006C6173740047
:10DB7000300066616C7365007472756500252E3126
:10DB800035732E2E2E006D616B654C6973740061C8
:10DB900064644C6173740064656C657465006A6FDD
:10DBA000696E0073706C697400636F707946726F90
:10DBB0006D546F0066696E64006A6F696E537472AB
:10DBC000696E677300756E69636F64654174007593
:10DBD0006E69636F6465537472696E67006E657712
:10DBE000427974654172726179006173427974653A
:10DBF000417272617900667265654D656D6F72790B
:10DC00000000000071DC00009113000076DC0000D1
:10DC1000AF13000097DB0000B31300007CDC0000B2
:10DC20009513000086DC0000B71300008FDC0000B5
:10DC3000BB13000099DC0000BF130000A2DC000051
:10DC4000C3130000ADDC0000C7130000B9DC000006
:10DC500099130000C2DC0000A7130000CCDC000018
:10DC60009D130000D7DC0000AB13000066696C65F3
:10DC7000006F70656E00636C6F736500656E644F56
:10DC80006646696C6500726561644C696E65007218
:10DC900065616442797465730072656164496E748C
:10DCA0006F00617070656E644C696E6500617070C4
:10DCB000656E6442797465730066696C6553697A50
:10DCC000650073746172744C697374006E65787466
:10DCD000496E4C6973740073797374656D496E662F
:10DCE0006F0000008817000098170000B2170000AE
:10DCF0002E180000661800009A180000D2180000C4
:10DD0000F81800003C1900007E190000D21900002C
:10DD1000161A0000781A0000C01A0000E61A000067
:10DD20001E1B0000641B00008A1B0000B81B0000C3
:10DD3000E61B0000DE3200009E1C0000701D00008B
:10DD4000E61D0000561E0000A21E0000C21E0000BC
:10DD5000E41E00003C20000080200000F8200000AD
:10DD600026210000582100008A2100000A2200001C
:10DD700072220000CE2200002C2300009E2300000F
:10DD8000102400006C240000C6240000FC240000C5
:10DD90004C25000092250000DA2500002E26000008
:10DDA00082260000C0260000462700007C270000D5
:10DDB000C42700000C280000542800008E28000012
:10DDC000D6280000282900008A2A0000B81B00007D
:10DDD0001E1B00009029000088170000C6290000C3
:10DDE000F2290000282A0000542A000088170000A9
:10DDF000881700008817000088170000062B000015
:10DE0000482B00008E2B0000DE2B00000A2C0000A7
:10DE1000822C0000D42C0000382D00008817000050
:10DE2000881700005C2D00008C2D0000BC2D000028
:10DE3000F22D00001C2E0000522E00007C2E00004F
:10DE4000A42E0000CC2E0000FC2E00002C2F000081
:10DE5000562F0000802F0000B02F0000DA2F0000A6
:10DE60008817000088170000881700008817000036
:10DE7000881700000A3000003630000062300000D1
:10DE80008E300000BA300000F03000003031000069
:10DE9000663100009C310000C8310000F431000000
:10DEA0002A32000088170000881700008817000039
:10DEB00088170000881700008817000088170000E6
:10DEC00088170000881700008817000088170000D6
:10DED00088170000563200005632000078330000E8
:10DEE000AE3300005B2564206974656D206C697336
:10DEF000745D002825642062797465732900286F99
:10DF0000626A65637420747970653A20256429001B
:10DF1000537461636B20756E646572666C6F770015
:10DF2000626F6F6C65616E006E756D626572007315
:10DF30007472696E67006C6973740062797465202D
:10DF400061727261790000000700000003000000A8
:10DF5000D2DF0000D5340000DADF00008535000094
:10DF6000E3DF0000AF370000ECDF0000D934000031
:10DF7000F5DF0000B3370000FDDF00009D37000033
:10DF800006E00000CD36000011E000003D39000041
:10DF90001CE000001536000027E00000B13800004A
:10DFA00033E00000793600003FE000000D3900004A
:10DFB000000000000100000002000000030000005B
:10DFC000040000000A0000006D6963726F3A626924
:10DFD0007400686173546F6E6500706C6179546F82
:10DFE0006E6500686173536572766F007365745374
:10DFF0006572766F00646163496E69740064616381
:10E0000057726974650073717561726557617665E1
:10E0100000736574557365724C454400616E616CA4
:10E020006F675265616400616E616C6F67577269FA
:10E030007465006469676974616C52656164006449
:10E0400069676974616C577269746500474320742D
:10E050006F6F6B2025642075736563733B20667258
:10E06000656520256420776F726473003C496E7487
:10E07000656765723E003C4C6973743E003C4F62BC
:10E080006A6563743E003C427974654172726179DD
:10E090003E000D0A564D2050616E69633A2025738B
:10E0A0000D0A006D69736300DDE000000D4400009F
:10E0B000E6E000009D430000EAE00000F1420000BD
:10E0C000F2E0000097420000FCE000002D4200005A
:10E0D00008E100002F4100006E756C6C00686578E7
:10E0E000546F496E740073696E006A736F6E476592
:10E0F00074006A736F6E436F756E74006A736F6E2F
:10E1000056616C75654174006A736F6E4B65794139
:10E1100074000000D8E1000079440000E0E1000054
:10E120007D440000EAE100009B440000F3E10000B0
:10E13000A5440000FEE10000AF4400000AE2000038
:10E14000B944000018E20000C344000020E20000CF
:10E15000CD44000026E20000D74400003BE200006E
:10E16000E144000050E20000EB4400005CE20000EB
:10E17000F54400006CE20000FF44000078E200007B
:10E180000945000085E200001345000094E200000C
:10E190001D450000A7E2000027450000BDE2000089
:10E1A00031450000C9E200003B450000D9E2000013
:10E1B00045450000E8E200004F450000F6E200009F
:10E1C00059450000FEE200008744000006E300001D
:10E1D000914400006E657400686173576946690078
:10E1E0007374617274576946690073746F7057690C
:10E1F00046690077696669537461747573006D7957
:10E20000495041646472657373007374617274532E
:10E210005349447363616E00676574535349440006
:10E220006D794D4143006874747053657276657200
:10E230004765745265717565737400726573706FAC
:10E240006E64546F487474705265717565737400B0
:10E2500068747470436F6E6E656374006874747074
:10E260004973436F6E6E656374656400687474709F
:10E27000526571756573740068747470526573705B
:10E280006F6E736500776562536F636B657453746B
:10E2900061727400776562536F636B65744C617370
:10E2A000744576656E7400776562536F636B657451
:10E2B00053656E64546F436C69656E74004D5154C0
:10E2C00054436F6E6E656374004D515454497343EB
:10E2D0006F6E6E6563746564004D51545444697388
:10E2E000636F6E6E656374004D5154544C6173746A
:10E2F0004576656E74004D515454507562004D5111
:10E300005454537562004D515454556E73756200E8
:10E310001A1B1C03040607090A171819000000003D
:10E320000008080800080A4A4000000A5FEA5FEA9D
:10E330000ED92ED36E19324489330C924C924D086B
:10E340000800000004880808040804848488000A7F
:10E35000448A4000048EC480000000048800000E3F
:10E36000C000000000080001224488100C925252A4
:10E370004C048C84848E1C824C901E1EC244924C91
:10E3800006CA525FE21FF01EC13E02448ED12E1F0C
:10E39000E24488100ED12ED12E0ED12EC488000852
:10E3A00000080000048004880244880482000EC033
:10E3B0000EC008048244880ED126C0040ED135B3A5
:10E3C0006C0C925ED2521C925C925C0ED010100EBD
:10E3D0001C9252525C1ED01C901E1ED01C90100E1F
:10E3E000D013712E12525ED2521C8808081C1FE2F4
:10E3F00042524C1254981492101010101E113B757A
:10E40000B131113935B3710C9252524C1C925C905F
:10E41000100C92524C861C925C92510ED00C825C75
:10E420001FE4848484125252524C1131312A441117
:10E430003135BB7112524C9252112A4484841EC44D
:10E4400088101E0EC808080E10080482410EC24231
:10E45000424E048A400000000000001F08048000B3
:10E4600000000ED2524F10101C925C000ED0100E05
:10E4700002424ED24E0C925C900E06C81C88080ECA
:10E48000D24EC24C10101C925208000808080240DC
:10E4900002424C10149814920808080806001B75D4
:10E4A000B131001C925252000C92524C001C925CF2
:10E4B00090000ED24EC2000ED010100006C8049874
:10E4C00008080EC807001252524F0011312A4400AA
:10E4D000113135BB00124C8C9200112A4498001E59
:10E4E000C4881E06C48C8486080808080818080C0E
:10E4F000881800000C83600000000000010000008C
:10E5000002000000030000000400000005000000FD
:10E5100006000000070000000800000009000000DD
:10E520000A0000000B0000000C0000000D000000BD
:10E530000E0000000F00000010000000120000009C
:10E540001400000016000000180000001A0000006F
:10E550001C0000001E00000020000000230000003E
:10E5600026000000290000002C0000002F00000001
:10E5700032000000360000003A0000003E000000BB
:10E5800042000000460000004B0000005000000068
:10E59000550000005A000000610000006800000003
:10E5A0006F000000760000007D0000008400000085
:10E5B0008B0000009200000099000000A000000005
:10E5C000A7000000AE000000B5000000BC00000085
:10E5D000C3000000CA000000D1000000D800000005
:10E5E000DF000000E6000000ED000000F400000085
:10E5F000FB000000FF00000048E600007D45000031
:10E6000053E60000F54A00005DE6000035470000D3
:10E610006AE600006548000071E60000B5480000A9
:10E620007AE600000549000086E60000FD4700008C
:10E6300097E60000F5490000A4E600008D470000C1
:10E64000646973706C6179006C696768744C657695
:10E65000656C006D62446973706C6179006D624431
:10E660006973706C61794F6666006D62506C6F748F
:10E67000006D62556E706C6F74006D6244726177EC
:10E680005368617065006D625368617065466F72B2
:10E690004C6574746572006E656F506978656C5373
:10E6A000656E64006E656F506978656C5365745073
:10E6B000696E004E6F7420656E6F75676820726FAB
:10E6C0006F6D206576656E20616674657220636F7C
:10E6D0006D70616374696F6E00436F6D7061637418
:10E6E000656420466C61736820636F646520737491
:10E6F0006F72650A2564206279746573207573658D
:10E700006420282564252529206F66202564004281
:10E710006164207265636F726420666F756E642039
:10E72000647572696E6720696E697469616C697A73
:10E730006174696F6E00256420256420256420289B
:10E74000256420776F7264732900256420726563E5
:10E750006F7264732C20256420776F7264732C2091
:10E760006D617849442025642C20636F6D7061636E
:10E7700074696F6E206379636C6573202564005241
:10E780006573746F726564202564207363726970A9
:10E790007473005374617274656400726164696FAC
:10E7A0000000000039E80000D954000046E80000ED
:10E7B0009957000056E800001957000064E800006F
:10E7C0002D5900006FE80000F15400007FE80000C0
:10E7D0006D55000093E8000055550000A2E80000C8
:10E7E0000F5B0000AEE800008D5A0000B7E80000A3
:10E7F000315A0000C2E8000079590000CDE800005D
:10E80000B5590000D6E80000E9590000DFE8000033
:10E8100001550000EEE8000035550000F7E8000063
:10E820001155000025303878006E6F6E65006F74EA
:10E8300068657200706169720064697361626C6519
:10E84000526164696F006D657373616765526563DA
:10E850006569766564007061636B657452656365B4
:10E86000697665007061636B657453656E640072F0
:10E8700065636569766564496E7465676572007283
:10E88000656365697665644D657373616765547921
:10E890007065007265636569766564537472696E4C
:10E8A000670073656E64496E7465676572007365B1
:10E8B0006E64506169720073656E64537472696E40
:10E8C00067007365744368616E6E656C0073657490
:10E8D00047726F757000736574506F77657200735F
:10E8E00069676E616C537472656E67746800646505
:10E8F000766963654944006C6173744D6573736137
:10E900006765494400556E6B6E6F776E2070726953
:10E910006D6974697665205B25733A25735D000027
:10E9200000000000963007772C610EEEBA5109996D
:10E9300019C46D078FF46A7035A563E9A395649EC9
:10E940003288DB0EA4B8DC791EE9D5E088D9D297ED
:10E950002B4CB609BD7CB17E072DB8E7911DBF9049
:10E960006410B71DF220B06A4871B9F3DE41BE846D
:10E970007DD4DA1AEBE4DD6D51B5D4F4C785D383C9
:10E9800056986C13C0A86B647AF962FDECC9658A6D
:10E990004F5C0114D96C0663633D0FFAF50D088DC9
:10E9A000C8206E3B5E10694CE44160D5727167A26D
:10E9B000D1E4033C47D4044BFD850DD26BB50AA5C9
:10E9C000FAA8B5356C98B242D6C9BBDB40F9BCACED
:10E9D000E36CD832755CDF45CF0DD6DC593DD1AB49
:10E9E000AC30D9263A00DE518051D7C81661D0BF6D
:10E9F000B5F4B42123C4B3569995BACF0FA5BDB8C9
:10EA00009EB802280888055FB2D90CC624E90BB16C
:10EA1000877C6F2F114C6858AB1D61C13D2D66B6C8
:10EA20009041DC760671DB01BC20D2982A10D5EF2C
:10EA30008985B1711FB5B606A5E4BF9F33D4B8E888
:10EA4000A2C9077834F9000F8EA8099618980EE12C
:10EA5000BB0D6A7F2D3D6D08976C6491015C63E688
:10EA6000F4516B6B62616C1CD83065854E0062F2AC
:10EA7000ED95066C7BA5011BC1F4088257C40FF508
:10EA8000C6D9B06550E9B712EAB8BE8B7C88B9FC2C
:10EA9000DF1DDD62492DDA15F37CD38C654CD4FB88
:10EAA0005861B24DCE51B53A7400BCA3E230BBD42C
:10EAB00041A5DF4AD795D83D6DC4D1A4FBF4D6D388
:10EAC0006AE96943FCD96E34468867ADD0B860DA2C
:10EAD000732D0444E51D03335F4C0AAAC97C0DDD88
:10EAE0003C710550AA41022710100BBE86200CC9AC
:10EAF00025B56857B3856F2009D466B99FE461CE08
:10EB00000EF9DE5E98C9D9292298D0B0B4A8D7C72B
:10EB1000173DB359810DB42E3B5CBDB7AD6CBAC087
:10EB20002083B8EDB6B3BF9A0CE2B6039AD2B174A3
:10EB30003947D5EAAF77D29D1526DB048316DC73FF
:10EB4000120B63E3843B64943E6A6D0DA85A6A7AA3
:10EB50000BCF0EE49DFF099327AE000AB19E077DFF
:10EB600044930FF0D2A3088768F2011EFEC2066923
:10EB70005D5762F7CB67658071366C19E7066B6E7F
:10EB8000761BD4FEE02BD3895A7ADA10CC4ADD67A3
:10EB90006FDFB9F9F9EFBE8E43BEB717D58EB060FF
:10EBA000E8A3D6D67E93D1A1C4C2D83852F2DF4FA3
:10EBB000F167BBD16757BCA6DD06B53F4B36B248FF
:10EBC000DA2B0DD84C1B0AAFF64A0336607A0441A3
:10EBD000C3EF60DF55DF67A8EF8E6E3179BE6946FF
:10EBE0008CB361CB1A8366BCA0D26F2536E2685223
:10EBF00095770CCC03470BBBB91602222F2605557F
:10EC0000BE3BBAC5280BBDB2925AB42B046AB35CA2
:10EC1000A7FFD7C231CFD0B58B9ED92C1DAEDE5BFE
:10EC2000B0C2649B26F263EC9CA36A750A936D02E2
:10EC3000A906099C3F360EEB85670772135700053E
:10EC4000824ABF95147AB8E2AE2BB17B381BB60C62
:10EC50009B8ED2920DBED5E5B7EFDC7C21DFDB0BBE
:10EC6000D4D2D38642E2D4F1F8B3DD686E83DA1FE2
:10EC7000CD16BE815B26B9F6E177B06F7747B7183E
:10EC8000E65A0888706A0FFFCA3B06665C0B0111E2
:10EC9000FF9E658F69AE62F8D3FF6B6145CF6C163E
:10ECA00078E20AA0EED20DD75483044EC2B30339E2
:10ECB000612667A7F71660D04D476949DB776E3E3E
:10ECC0004A6AD1AEDC5AD6D9660BDF40F03BD83762
:10ECD00053AEBCA9C59EBBDE7FCFB247E9FFB530BE
:10ECE0001CF2BDBD8AC2BACA3093B353A6A3B424E2
:10ECF0000536D0BA9306D7CD2957DE54BF67D9233E
:10ED00002E7A66B3B84A61C4021B685D942B6F2AE1
:10ED100037BE0BB4A18E0CC31BDF055A8DEF022D3D
:10ED2000416C6C207461736B732073746F707065C9
:10ED300064007631353500202573202573004D653C
:10ED40006D6F727920636C6561726564004E6F202F
:10ED500066726565207461736B20656E7472696597
:10ED600073000000DCED00002D720000E9ED0000F2
:10ED7000BD6B0000F5ED0000FD710000FBED000033
:10ED80000D72000001EE00001D72000007EE000091
:10ED9000D57000001DEE0000E57300002BEE0000B2
:10EDA000F16B000035EE0000717400003DEE0000D4
:10EDB000F96E000046EE0000B56D000052EE000056
:10EDC000CD6C00005BEE0000196D000063EE0000EA
:10EDD000016E000073656E736F727300616363652B
:10EDE0006C65726174696F6E0074656D70657261D7
:10EDF000747572650074696C74580074696C745928
:10EE00000074696C745A00736574416363656C6562
:10EE1000726F6D6574657252616E6765006D6167D2
:10EE20006E657469634669656C6400746F756368C8
:10EE300052656164006932635265616400693263DE
:10EE400057726974650073706945786368616E67AD
:10EE50006500737069536574757000726561644410
:10EE60004854006D6963726F70686F6E65000000D2
:10EE700071DC00005175000076DC0000FD740000BC
:10EE8000A7EE00009576000099DC000019750000DF
:10EE9000ACEE00001D760000B2EE000075750000BB
:10EEA00073657269616C0072656164007772697480
:10EEB00065007772697465427974657300000000BB
:10EEC0003CEF0000C57600004AEF0000D576000058
:10EED00057EF0000C976000060EF0000D97600000F
:10EEE0006AEF0000DD76000073EF0000E1760000BD
:10EEF00078EF0000E57600007DEF0000E976000085
:10EF000089EF0000ED76000090EF0000F176000040
:10EF100099EF0000F57600009EEF0000F976000002
:10EF2000A9EF0000FD760000B3EF0000CD760000F1
:10EF3000BDEF0000D176000074667400656E6162FA
:10EF40006C65446973706C617900736574426163C8
:10EF50006B6C6967687400676574576964746800EE
:10EF6000676574486569676874007365745069788B
:10EF7000656C006C696E65007265637400726F7514
:10EF80006E6465645265637400636972636C6500E6
:10EF9000747269616E676C6500746578740074667C
:10EFA00074546F756368656400746674546F756338
:10EFB000685800746674546F756368590074667499
:10EFC000546F75636850726573737572650076610E
:10EFD00072730000F4EF00008D7B0000FEEF000074
:10EFE0006D7B000007F00000497B000013F000007B
:10EFF000D77A000076617245786973747300766120
:10F00000724E616D6564007365745661724E616D18
:10F010006564007661724E616D65466F72496E641B
:10F0200065780057656C636F6D6520746F204D695E
:10F0300063726F426C6F636B732100705F737069F2
:10F0400020213D204E554C4C002F686F6D652F6779
:10F0500069742F2E706C6174666F726D696F2F709A
:10F0600061636B616765732F6672616D65776F723F
:10F070006B2D61726475696E6F6E6F726469636E19
:10F080007266352F6C69627261726965732F5350B5
:10F09000492F5350492E63707000535049436C619F
:10F0A00073733A3A535049436C617373284E524616
:10F0B0005F5350495F547970652A2C2075696E74CE
:10F0C000385F742C2075696E74385F742C207569F4
:10F0D0006E74385F7429000000000000000000001A
:10F0E000617D00001D7D0000437D00004D7D00001E
:10F0F000577D0000417D0000030000000200000079
:10F1000001000000040000000500000011000000E4
:10F110000C0000000B000000120000000A000000BC
:10F12000060000001A000000140000001700000094
:10F13000160000001500000010000000FFFFFFFF98
:10F14000FFFFFFFF000000001E000000190000008C
:10F15000180000000700000008000000090000007F
:10F160000D0000000E0000000F0000001C00000059
:10F170001B0000001D000000130000000000000044
:10F18000000000004D81000081890000CD81000059
:10F19000E1810000D7810000498100003D8100002D
:10F1A000ED8100006981000039810000000000004D
:10F1B000000000000000304300000000000030C3E9
:10F1C0007371727400000000FB21F93FFB210940BC
:10F1D0007CD91240FB2119407A6A1F407CD9224019
:10F1E000BBFD2540FB2129403A462C407A6A2F403E
:10F1F0005C4731407CD932409C6B3440BBFD35408C
:10F20000DB8F3740FB2139401BB43A403A463C4043
:10F210005AD83D407A6A3F404C7E40405C4741406E
:10F220006C1042407CD942408CA243409C6B4440CD
:10F23000AC344540BBFD4540CBC64640DB8F474024
:10F24000EB584840FB21494083F9A200444E6E0030
:10F25000FC291500D1572700DD34F50062DBC00022
:10F260003C999500419043006351FE00BBDEAB002A
:10F27000B761C5003A6E2400D24D42004906E00055
:10F2800009EA2E001C92D100EB1DFE0029B11C00E2
:10F29000E83EA700F535820044BB2E009CE98400BF
:10F2A000B4267000417E5F00D69139005383390047
:10F2B0009CF439008B5F840028F9BD00F81F3B00E7
:10F2C000DEFF97000F980500112FEF000A5A8B0000
:10F2D0006D1F6D00CF7E360009CB2700464FB7006B
:10F2E0009E663F002DEA5F00BA277500E5EBC70078
:10F2F0003D7BF100F739070092528A00FB6BEA0070
:10F300001FB15F00085D8D00300356007BFC460096
:10F31000F0AB6B0020BCCF0036F49A00E3A91D00CF
:10F320005E619100081BE60085996500A0145F00EE
:10F330008D40680080D8FF0027734D00060631001D
:10F34000CA561500C9A873007BE260006B8CC00030
:10F3500000000040FB21F93F000000002D44743EF6
:10F36000000000809846F83C0000006051CC783BDB
:10F3700000000080831BF0390000004020257A380F
:10F38000000000802282E336000000001DF3693592
:10F39000020000000300000004000000060000005E
:10F3A000F8A50000A2A50000A2A50000D0A60000BC
:10F3B0009EA500009EA50000C6A60000D0A60000E5
:10F3C0009EA50000C6A600009EA50000D0A60000D5
:10F3D000D4A60000D4A60000D4A60000DCA600003D
:10F3E000D4B0000046AF00008AAF0000EEAE0000CF
:10F3F0008AAF00007AB000008AAF0000EEAE0000D5
:10F4000046AF000046AF00007AB00000EEAE00004C
:10F41000E6AE0000E6AE0000E6AE000088B00000F8
:10F42000FCB70000FEB60000FEB600001CBA0000EB
:10F43000F8B60000F8B6000004BA00001CBA0000DC
:10F44000F8B6000004BA0000F8B600001CBA0000CC
:10F4500012BA000012BA000012BA000020BA00006E
:10F460002C2066756E6374696F6E3A200061737349
:10F47000657274696F6E2022257322206661696C43
:10F4800065643A2066696C6520222573222C206C05
:10F49000696E65202564257325730A00900000209D
:10F4A000232D302B2000686C4C006566674546476D
:10F4B00000303132333435363738394142434445F0
:10F4C000460030313233343536373839616263645F
:10F4D0006566000000000000000000000000000061
:10F4E000000000000000000000000000000000001C
:10F4F000000000000000000000000000000000000C
:10F5000000000000000000000000000000000000FB
:10F5100000000000000000000000000000000000EB
:10F5200000000000000000000000000000000000DB
:10F5300000000000504F5349580000202020202098
:10F540002020202028282828282020202020202093
:10F550002020202020202020202020881010101083
:10F5600010101010101010101010100404040404D7
:10F570000404040404101010101010104141414103
:10F5800041410101010101010101010101010101EB
:10F5900001010101010110101010101042424242FD
:10F5A00042420202020202020202020202020202BB
:10F5B00002020202020210101010200000000000DF
:10F5C000000000000000000000000000000000003B
:10F5D000000000000000000000000000000000002B
:10F5E000000000000000000000000000000000001B
:10F5F000000000000000000000000000000000000B
:10F6000000000000000000000000000000000000FA
:10F6100000000000000000000000000000000000EA
:10F6200000000000000000000000000000000000DA
:10F6300000000000000000000000000000000000CA
:08F64000C80AFF7F0100000071
:10F64800FFFFFFFFE803000001000000E803DC05FE
:10F65800DC05DC05DC050000FFFFFFFFFFFFFFFF07
:10F668001800000019FCFFFFFFFFFFFF0200000069
:10F6780040420F00FFFF01FF0024F40002000000D9
:10F6880003000000FFFFFFFF000000000100000072
:10F698000000020001000000FFFFFFFF0000000063
:10F6A800020000000000040002000000FFFFFFFF4E
:10F6B8000000000003000000000008000300000034
:10F6C8000A0000000800000001000000900000206F
:10F6D80000000000F4F4000014F50000D4F4000069
:10F6E8000000000000000000000000000000000012
:10F6F8000000000000000000000000000000000002
:10F7080000000000000000000000000000000000F1
:10F7180000000000000000000000000000000000E1
:10F7280000000000000000000000000000000000D1
:10F73800430000000000000000000000000000007E
:10F7480000000000000000000000000000000000B1
:10F75800430000000000000000000000000000005E
:10F768000000000000000000000000000000000091
:10F77800430000000000000000000000000000003E
:10F788000000000000000000000000000000000071
:10F79800430000000000000000000000000000001E
:10F7A8000000000000000000000000000000000051
:10F7B80043000000000000000000000000000000FE
:10F7C8000000000000000000000000000000000031
:10F7D80043000000000000000000000000000000DE
:10F7E8000000000000000000000000000000000011
:10F7F80043000000000000000000000000000000BE
:10F8080000000000000000000000000000000000F0
:10F8180029D9000041D30000000000003AF500009B
:10F8280084DB0000A2E00000A2E00000A2E00000EB
:10F83800A2E00000A2E00000A2E00000A2E00000B8
:10F84800A2E00000A2E00000FFFFFFFFFFFFFFFFB4
:10F85800FFFFFFFFFFFF000001004153434949003C
:10F868000000000000000000000000000000000090
:10F878000000000000000000000041534349490017
:10F888000000000000000000000000000000000070
:10F89800000000000000000000000000E900000077
:10F8A800ED7C00004180000099840000C100000048
:04000003000080DD9C
:00000001FF
